:100000000C94DA100C940B110C940B110C940B1132
:100010000C940B110C940B110C940B110C940B11F0
:100020000C940B110C940B110C940B110C940B11E0
:100030000C940B110C940B110C940B110C940B11D0
:100040000C940B110C940B110C940B110C940B11C0
:100050000C940B110C940B110C940B110C9496A88E
:100060000C940B110C9482820C9458820C940B11FA
:100070000C940B110C940B110C940B110C940B1190
:100080000C940B110C940B110C940B110C940B1180
:100090000C940B110C940B110C940B110C94042464
:1000A0000C940B110C940B110C940B110C940B1160
:1000B0000C940B110C940B110C940B110C940B1150
:1000C0000C940B110C940B110C940B110C940B1140
:1000D0000C940B110C940B110C940B110C940B1130
:1000E0000C940B1107634236B79BD8A71A39685690
:1000F00018AEBAAB558C1D3CB7CC5763BD6DEDFD4A
:10010000753EF6177231BF000000803F0800000006
:10011000BE922449123EABAAAA2ABECDCCCC4C3EFC
:1001200000000080BEABAAAAAA3E00000000BF00EB
:100130000000803F0000000000084178D3BB4387E7
:10014000D1133D190E3CC3BD4282AD2B3E68EC82FB
:1001500076BED98FE1A93E4C80EFFFBE01C4FF7F80
:100160003F00000000000C94AB130C9408330C9477
:1001700025110C9448B50C9478110C94E8340C9427
:10018000B2420C948F150C9449790C94B9400C949C
:10019000AB780C94BA9E0C94919E0C9450840C9461
:1001A0004C1D0C946E770C94CA4A0C9415110C9447
:1001B00066330C9411350C943A6E0C944D110C94DA
:1001C0000D110C9468330C9442B50C94CB110C9423
:1001D0002D5E0C94B69E0C944B530C94E7120C9429
:1001E000BE120C94CD930C94827A0C94846E0C9471
:1001F000E6310C9491880C9408140C94A7120C947A
:10020000C7340C9468810C943C530C9467790C941B
:100210000E4A0C94A3B70C942F410C941E7A0C94A4
:10022000367A0C944F5D0C9467BA0C9467840C94E6
:1002300059530C9455110C943D770C94CA5C0C9452
:10024000001B0C94FE120C94C07B0C9424940C9410
:100250000F770C945D340C94CE350C94ADBF0C9498
:10026000BB880C9410580C9481130C9465780C94F2
:10027000A39E0C94DD310C9498350C949FBF0C9484
:10028000412E0C9484BF0C949F570C94CC9E0C94DC
:1002900029170C94EF350C94B5120C94E5420C948C
:1002A000835D0C94A6770C947B5E0C94BC110C942B
:1002B0006C330C94B7B10C94622F0C9412120C9402
:1002C0002A6E0C94FC840C94D1150C94DA350C94A1
:1002D000C3840C94B6120C94FE520C94032F0C940D
:1002E00070330C945D360C946DA60C947B140C94B6
:1002F000FE790C9475150C94B2650C9464330C94CF
:1003000046A40C9460770C94F24C0C949F9E0C9431
:1003100071150C94231A0C94E8790C9456530C9490
:1003200026380C94F8BE0C94979E0C9443350C948C
:1003300076110C9473A60C9479C10C9452860C948B
:100340002E760C947D360C94E5110C9447840C9415
:10035000E7150C9478A60C9468780C94365D0C9490
:100360002C110C942E7C0C944A6B0C94B1840C943C
:10037000172E0C94C8400C94FD640C940F340C940C
:100380009B9E0C948F350C941E410C946AA60C9481
:10039000081F0C94B9120C9409420C94BB4B0C949A
:1003A0006F350C94BC1A0C946E330C944E150C944F
:1003B00062330C9447340C9413350C9459350C94D7
:1003C0002A480C940B5E0C94C2130C9412530C9498
:1003D00039200C940A940C9426360C94B9790C9418
:1003E00044340C94C51F0C945E330C9465530C94E8
:1003F00036840C94E7930C942D310C9461B90C94D1
:1004000072880C9411590C9415390C9472330C9415
:10041000B2790C94465E0C94BB110C94EE140C94BF
:10042000BF130C9460330C94B09E0C94EC4C0C9461
:100430002F2E0C94A74A0C94CC7A0C94631E0C9427
:10044000EBBD0C94BA500C94814A0C9425530C9437
:10045000D8410C94D69E0C94D65E0C94A69E0C9417
:100460003F490C94F6120C944C770C943DA40C94D8
:1004700004350C94F87B0C94D2340C9410770C94C3
:10048000204B0C9492470C94D4930C94514B0C94A5
:1004900056110C94A5570C94C95D0C94DA400C9439
:1004A00076790C94B05D0C94BA110C9467520C944C
:1004B0007D2F0C94EC2F0C942A340C94D35E0C9466
:1004C000D19E0C9470A60C9427BF0C945E780C946B
:1004D000FD190C942D8F0C94DE120C94C7190C94FA
:1004E000A1130C947A6A0C9444780C94BE9E0C94DC
:1004F000BCAF0C946E780C94BD130C94A4520C9465
:1005000003150C9433350C94FE150C9413A40C9421
:1005100042110C94AD4B0C94101A0C94F32D0C94C6
:10052000A4A50C94DE780C94F3770C94C0350C944D
:10053000D7170C94F0350C94D0310C9405130C940F
:10054000C9870C94EE4C0C9406BF0C945C6C0C9414
:100550006F130C949DA50C94962E0C946A330C94F6
:10056000DE110C94992F0C94C89E0C94A0790C94D5
:10057000F2BE0C94FA5E0C949C1E0C94B2350C9452
:10058000132F0C94AE490C94F7780C94AC9E0C94F9
:1005900078420C94EB930C942B170C94F5310C943B
:1005A000E66B0C9496570C94DF350C94F2130C9474
:1005B000FD760C94B9130C94B3480C9411110C945F
:1005C000D95E0C94D29E0C94D7310C946B1D0C9474
:1005D000005D0C949E7B0C947E1D0C945B260C9409
:1005E00040A40C9448530C94C49E0C9424360C9450
:1005F0006C114E414E494E495459494E46CDCCCCD2
:100600003D0AD7233C17B7D13877CC2B329595E6E6
:10061000241FB14F0A000020410000C84200401CC6
:100620004620BCBE4CCA1B0E5AAEC59D746364699D
:100630006E6F70737578585B00454F46002F004908
:100640006E3A20003D00494E3A003D004C4547417E
:10065000435920494E3A000000200023002600297B
:10066000002C002F003200000100000301060109E8
:10067000012D3E00200023002D3E00200050656E1D
:100680006465643A2023007261770076616C0074BF
:10069000656D7000736174006875650066616E0059
:1006A00052474200485356006D6F646500536574AD
:1006B000436D643A0053746F726564204558543A30
:1006C00000737566666978436F64653A0020666FEB
:1006D0007220286D73293A004354524C3A205363D8
:1006E000686564756C6520636D642000206D7320FF
:1006F0003A0041726D656420666F72200020446983
:100700007361726D656400584F4E0048414C54004F
:100710002074696D653A004354524C3A2052657317
:100720003A002054533A0020543A003D0050696E7C
:100730003A004354524C3A20436F6D6D616E642011
:10074000626C6F636B6564206279206472697665A0
:1007500072206F72206368616E6E656C2066726FC6
:100760007A656E004354524C3A204F4E3A416C72B7
:1007700065616479204163746976650A0043545267
:100780004C3A2048414C543A416C7265616479207E
:10079000496E6163746976650A004354524C3A208D
:1007A000584F4E3A2044697361626C65640A004395
:1007B00054524C3A20584F4E3A416C7265616479FC
:1007C000204163746976650A004354524C3A2058BC
:1007D0004F464620736B69707065642E20507265B9
:1007E0007620636D643A004354524C3A205475723B
:1007F0006E6564206F66662066726F6D3A004354C2
:10080000524C3A20526573746F7265642066726F41
:100810006D3A004354524C3A2049676E6F726564DA
:100820002C206368616E6E656C20636D643D0020F2
:10083000457865633A004354524C3A2041637469E9
:1008400076653A004354524C3A2048414C543A4160
:100850006C726561647920496E6163746976650ABA
:10086000004354524C3A20584F4E3A204469736129
:10087000626C65640A004354524C3A20584F4E3A19
:10088000416C7265616479204163746976650A0020
:100890004354524C3A20584F464620736B6970704F
:1008A00065642E205072657620636D643A0043546F
:1008B000524C3A205475726E6564206F66662066ED
:1008C000726F6D3A004354524C3A20526573746F04
:1008D0007265642066726F6D3A004354524C3A2040
:1008E0004E6F7420656E6F756768206D656D6F72F1
:1008F0007920666F722067726F7570206F706572F5
:100900006174696F6E00496E76616C696420617212
:100910006700496E76616C696420617267004354B8
:10092000524C3A20556E6B6E6F776E20737566660B
:10093000697800536B697070656420686F6D6965D4
:10094000207374756666002000205375623D002098
:100950004974656D3D004354524C3A2052414D3D1F
:10096000004354524C3A204F75744F664D656D6F7D
:1009700072793A2000282D292000282B29200020D8
:1009800076616C7565206973200020756E6B6E6FE3
:10099000776E0A005D3D005B0020696E76616C69D0
:1009A00064002000206F6B003A00206661696C656E
:1009B00064003A005265747279696E67206D6F64E5
:1009C00062757320434D440A004354524C2F706F9C
:1009D0006C6C3A204F75744F664D656D6F72793A45
:1009E0002000207365632072656D61696E696E67B2
:1009F000005374617475732064656666657265641E
:100A00000A00444D58000000000000444D58524771
:100A100042570000444D5852474200000050574D85
:100A20000000000000004D42555344494D00005461
:100A30004845524D4F00000052454C4159000000BE
:100A40000047524F555000000000564354454D504A
:100A50000000004D425553564300000041434841B9
:100A600049455200005350494C45440000004D4F49
:100A7000544F5200000000504944000000000000A4
:100A80004D4255530000000000554152544252441B
:100A9000470052454C415950574D00444D5852471C
:100AA0004257570056454E545300000000454C45F0
:100AB0005641544F5200434F554E54455200004842
:100AC000554D0000000000004D455243555259005D
:100AD0000020002D3E00436F6E76657274696E676C
:100AE00020002D3E0057726F6E6720417373696757
:100AF0006E6D656E742000524742783A200048536C
:100B0000562064697361626C65640020764C65767A
:100B1000656C3A0020436F6E76563A0020436F6E44
:100B200076533A0020486F743A00436F6C643A0081
:100B300020436F6E76657274656420563A00436F89
:100B40006E76657274656420533A002D3E005772CC
:100B50006F6E672041737369676E6D656E742000F8
:100B60002D3E0057726F6E672041737369676E6D1B
:100B7000656E74200053617665643A002053756693
:100B8000663A002041543A00436F6E6669672063FD
:100B900068616E676564206C6F63616C6C792C2092
:100BA000706F7274616C2064697361626C6564005B
:100BB0002F636F6E6669672E6A736F6E007265626F
:100BC0006F6F742000436D643A20002F636F6D6D6A
:100BD000616E642F002F72616D2F002F6974656D37
:100BE0002F002F6974656D2F004C6F636174696FFE
:100BF0006E3A20687474703A2F2F6C617A79686F3E
:100C00006D652E72752F707761003F6D61633D00D9
:100C10002669703D0026706F72743D00266E616D0E
:100C2000653D002F002000436F6D706C6574652E6C
:100C30002052656D6F766520746F706963200024A3
:100C4000636F6D6D616E6400536B697070696E6780
:100C50002E2E00436C65616E55702072657461695B
:100C60006E656420746F7069632000220022004F5B
:100C700075744F664D656D6F727921005D20003A85
:100C80005B000A005D00456D7074793A205B000AD4
:100C9000003A004D41433A00554450205379736C5B
:100CA0006F6720696E697469616C697A65642E0A80
:100CB000005379736C6F6720706172616D733A00D5
:100CC0003E003C00543A0043757272656E74204CCD
:100CD000414E20636F6E6669672869702C646E737D
:100CE0002C67772C7375626E6574293A000A557308
:100CF0006520746865736520636F6D6D616E6473E4
:100D00003A202768656C7027202D2074686973204D
:100D1000746578740A276D61632064653A61643A8A
:100D200062653A65663A66653A30302720736574C5
:100D300020616E642073746F7265204D41432D6194
:100D400064647265737320696E20454550524F4D3F
:100D50000A276970205B69705B2C646E735B2C677B
:100D6000775B2C7375626E65745D5D5D5D27202D0C
:100D700020736574207374617469632049500A2775
:100D80007361766527202D20736176652063757207
:100D900072656E7420636F6E66696720696E204E9F
:100DA0005652414D3B204F4E7C4F4646202D2065EC
:100DB0006E61626C652F64697361626C6520617538
:100DC000746F736176650A2767657427205B636FAC
:100DD0006E66696720616464725D27202D206765F7
:100DE0007420636F6E6669672066726F6D20707223
:100DF000652D636F6E666967757265642055524C28
:100E000020616E642073746F726520616464722C5B
:100E1000204F4E7C4F4646202D20656E61626C65EA
:100E20002F64697361626C6520646F776E6C6F61AB
:100E300064206F6E20737461727475700A276C6F12
:100E4000616427202D206C6F616420636F6E66697A
:100E5000672066726F6D204E5652414D0A2770779B
:100E60006427202D20646566696E6520616E6420AC
:100E700073746F7265204D51545420706173737791
:100E80006F72640A276F746170776427202D206465
:100E90006566696E6520616E642073746F7265208B
:100EA00048545450204150492070617373776F72D9
:100EB000640A276C6F67205B73657269616C5F6C95
:100EC0006F676C6576656C5D205B7564705F6C6FD9
:100ED000676C6576656C5D27202D20646566696E9C
:100EE00065206C6F67206C6576656C2028302E2E2F
:100EF00037290A276B696C6C27202D207465737461
:100F0000207761746368646F670A27636C65617238
:100F100027202D20636C65617220454550524F4D4E
:100F20000A277265626F6F7427202D207265626FC9
:100F30006F7420636F6E74726F6C6C657200536FA8
:100F40006674207265626F6F74696E672E2E2E0054
:100F500052414D3D000A5379736C6F6720000A318E
:100F60002D7769726520000A6D71747420000A691A
:100F70006E7075747320000A6974656D7320000AC1
:100F8000436F6E666967757265643A0020416464F8
:100F9000723A0064657623000944533234383220B3
:100FA0006572726F720009526573657420646F6EAA
:100FB000650009436865636B696E6720666F722020
:100FC000312D5769726520646576696365732E2ECD
:100FD0002E004453323438322D3130302070726557
:100FE00073656E74004572726F7220312D772069BF
:100FF0006E697420233220467265653A00777374F7
:1010000061742E20467265653A005465726D2E201B
:10101000467265653A004572726F7220312D7720F5
:10102000696E697420233100467265653A00445345
:10103000323438325F3130305F4932435F544F5F72
:1010400031575F42524944474520696E6974003BFD
:10105000003D0050696E3A003B003D4C4F57005434
:101060006865726D6F3A004F6E6520776972652012
:1010700052656164790A004170706C79696E67200D
:10108000636F6E666967004C6F61646564204554E8
:1010900041473A004E6F2073746F72656420636F2E
:1010A0006E666967004C6F616465642066726F6D7F
:1010B00020454550524F4D006C6F61642066616958
:1010C0006C6564004A534F4E2064657465637465B3
:1010D00064004C6F6164696E6720436F6E66696778
:1010E0002066726F6D20454550524F4D00436F6E24
:1010F000666967206175746F736176653A000A539B
:1011000079736C6F67206465627567206C657665BE
:101110006C3A0053657269616C2064656275672082
:101120006C6576656C3A0053617665640A005365B8
:10113000742064796E616D69632049500A004545E9
:1011400050524F4D20636C65617265640A004D51C9
:1011500054542050617373776F72642075706461AA
:101160007465640A004F54412050617373776F7245
:101170006420757064617465640A00636F756C64E3
:10118000206E6F742070617273653A200055706430
:10119000617465640A004E6F204950206164726575
:1011A00073730052656C656173696E6720736F635A
:1011B0006B657420616E64207265747279002053CF
:1011C00061766564004C6F6164696E6720485454B1
:1011D0005020636F6E666967206F6E207374617252
:1011E0007475703A004F4646004F4E002B002D009C
:1011F000455461673A200047657420455441473A99
:101200002000485454502F312E310025733A2025A8
:10121000730D0A0020485454502F312E310D0A48C6
:101220006F73743A2025730D0A4163636570743AD5
:10123000202A2F2A0D0A436F6E6E656374696F6EE4
:101240003A20636C6F73650D0A0025730020000D52
:101250000A00474554006661696C656420746F201C
:10126000636F6E6E6563740A004552524F523A20A6
:101270005365727665722072657475726E6564204E
:1012800000436F6E666967206E6F74206368616EDD
:101290006765640A00446F6E652E0A00436F6E66D0
:1012A00069672070617273696E67206661696C6539
:1012B000640A00676F7420436F6E6669670A00688E
:1012C00074747020726574636F6465200066726563
:1012D000652000436F6E666967205552493A206861
:1012E0007474703A2F2F002044656661756C742009
:1012F000636F6E66696720736572766572207573B9
:1013000065643A20006C617A79686F6D652E72753C
:10131000000A282D294D554C544956454E54000A73
:10132000282B2950574D5F52454C4159000A282D12
:10133000294D444E53000A282D29554152544252FA
:1013400049444745000A282B295359534C4F47001D
:101350000A282D29504944000A282D294D4350328E
:1013600033303137000A282D294152544E4554005C
:101370000A282B294F5441000A282D29535049206F
:101380004C4544000A282D294D4F544F52204354B8
:1013900052000A282D294143204841494552000A5C
:1013A000282D2943435338313120262048444331E6
:1013B000303830000A282B29524553544152545F8B
:1013C0004C414E5F4F4E5F4D5154545F4552524F0A
:1013D0005253000A282D294841524452455345543E
:1013E0002C207573696E6720736F6674000A282D50
:1013F00029434F554E544552000A282D294448543C
:10140000000A282B294453323438322D3130300031
:101410000A282B294F57495245000A282D2949509F
:101420004D4F44425553000A282D294D4F444255F3
:1014300053000A282D29444D58000A282B295769A2
:101440007A6E657435313030000A282B2946726572
:101450006552616D207072696E74696E67000A284A
:101460002B295741544348444F47006C617A7968AF
:101470006F6D652E7275000A436F6E666967207323
:1014800065727665723A003230313130334C00206B
:10149000432B2B2076657273696F6E3A0066366156
:1014A000353733345F323032332D31302D32310025
:1014B0000A4C617A79686F6D652E7275204C696788
:1014C000687448756220636F6E74726F6C6C6572BD
:1014D0002000204F464600204F4E002042595041E8
:1014E000535300757074696D650066726565686553
:1014F0006170002054696D65723A00204C6F636B17
:10150000733A002000204C6F636B733A000A52411B
:101510004D3D0020457870697265640A00202D7485
:101520006172676574207A6F6E652D0020416C6171
:10153000726D20457870697265640A0020636D647D
:101540003A00204375723A00205365743A005361A3
:1015500076656420746F20454550524F4D005361AD
:1015600076696E6720636F6E66696720746F2045C9
:101570004550524F4D2E2E00206973200044656C5B
:101580006574696E6720636F6E662E2052414D2030
:101590007761733A0053746F707065640053746FB1
:1015A0007070696E67206368616E6E656C73202E63
:1015B0002E2E004E6F7420756E6C6F636B65642009
:1015C000696E20313073202D20636F6E74696E75E3
:1015D00065202E2E2E00556E6C6F636B696E672032
:1015E000636F6E666967202E2E2E0020696E697407
:1015F0000052656C61792D4F75742023002073743F
:101600006F700052656C61792D4F75742023003D19
:101610003E003A0070756220616374696F6E20004D
:1016200069646C65006F66660068656174696E6701
:101630000066616E00647279696E6700636F6F6C3B
:10164000696E670020697320004F75742000556E25
:101650006B6E6F776E207375666669782000556EC5
:101660006B6E6F776E20636D642000616374696FC9
:101670006E0072656C61794374723A200020416497
:1016800064723A00646576230020616C69766500B7
:10169000204E6F64653A00312D7769726520636F63
:1016A000756E743A2000312D776972652073686F0A
:1016B00072746564005B305D3A2000202D202D207F
:1016C0002D20EFBBBF003E003E31202D200020002A
:1016D0002E00696E00735F6F7574006D79686F6DB1
:1016E00065004354524C2F657865633A204F7574FA
:1016F0004F664D656D6F72793A2000202D3E2000B7
:10170000456D69743A2000202D3E20004974656DB6
:10171000436D643A2000202D3E20004974656D3AE7
:101720002000005EBCE2613FDD83C29C7E20A3FD01
:101730001F419DC3217FFCA2401E5F01E3BD3E60AF
:1017400082DC237D9FC1421CFEA0E1BF5D0380DEE1
:101750003C62BEE0025CDF81633D7C22C09E1D4393
:10176000A1FF4618FAA427799BC584DA3866E5BB41
:101770005907DB856739BAE406581947A5FB78266F
:10178000C49A653BD987045AB8E6A7F91B45C698A1
:101790007A24F8A6441A99C7257B3A6486D85B0553
:1017A000E7B98CD2306EEDB3510F4E10F2AC2F7101
:1017B00093CD114FADF3702ECC92D38D6F31B2EC2F
:1017C0000E50AFF1134DCE90722C6D33D18F0C5261
:1017D000B0EE326C8ED0530DEFB1F0AE4C1291CF13
:1017E0002D73CA947628ABF517490856B4EA6937C1
:1017F000D58B5709EBB536688AD495CB2977F4AAEF
:101800004816E9B7550B88D6346A2B7597C94A1420
:10181000F6A8742AC896154BA9F7B6E80A54D789D2
:101820006B35436F6E6E65637465642E00436F6E37
:101830006E2E2061626F72746564003E3E20004926
:101840006E76616C696420636F6D6D616E64003EDD
:101850003E3E004E6F204D414320636F6E666967C8
:10186000757265643A20736574206669726D77617C
:1018700072652773204D41430A00454550524F4D34
:10188000207369676E6174757265206F6B00496EB5
:10189000697469616C697A696E6720454550524F79
:1018A0004D2E00476F742049502061646472657347
:1018B000733A00276970205B69705B2C646E735B00
:1018C0002C67775B2C7375626E65745D5D5D5D275B
:1018D000202D2073657420737461746963204950EE
:1018E0000A004661696C656420746F20636F6E66E0
:1018F00069677572652045746865726E65742075D8
:1019000073696E6720444843502E20596F752063D9
:10191000616E20736574206970206D616E75616CF5
:101920006C792100204D41534B3A002047573A0033
:1019300020444E533A004C6F616465642066726FB8
:101940006D20666C6173682049503A000A757365B2
:101950007320444843500A005374617274696E677F
:10196000206C616E004142434445464748494A4B1A
:101970004C4D4E4F505152535455565758595A6129
:1019800062636465666768696A6B6C6D6E6F7071BF
:1019900072737475767778797A30313233343536BC
:1019A0003738392B2F3D0042617369632000617223
:1019B0006475696E6F3A004F544120696E697469AD
:1019C000616C697A65640A0044454641554C54206F
:1019D00070617373776F726420666F72204F544129
:1019E000204150492E20557365206F7461707764D3
:1019F00020636F6D6D616E6420746F207365740079
:101A000070617373776F726400546F6F206D616ED5
:101A100079204D51545420636F6E6E656374696F05
:101A20006E206572726F72732E20526573746172CC
:101A300074204C414E002074727920616761696E98
:101A400020696E2035207365636F6E647300666174
:101A5000696C65642C2072633D004177616974692B
:101A60006E6720666F722072657461696E656420AE
:101A7000746F7069637300636F6E6E656374656421
:101A80002061732000202E2E2E0020757365723A7F
:101A9000003A000A417474656D7074696E67204D78
:101AA00051545420636F6E6E656374696F6E207459
:101AB0006F2000646973636F6E6E656374656400A4
:101AC0005573696E67204D5154542070617373775C
:101AD0006F72642066726F6D20636F6E6669670057
:101AE000446576696365204E616D653A00417420F6
:101AF0006C6561737420646576696365206E616DE1
:101B00006520616E642062726F6B6572204950209F
:101B10006D75737420626520636F6E666967757298
:101B2000656400757074696D652C667265656865BD
:101B300061700024737461747300663661353733E5
:101B4000345F323032332D31302D3231004C696701
:101B500068744875622000246E616D65007265616D
:101B600064790024737461746500526562696E64FF
:101B700020737563636573732E204950206164641C
:101B8000726573733A004572726F723A20726562C1
:101B9000696E64206661696C0052656E6577656484
:101BA00020737563636573732E20495020616464EC
:101BB000726573733A004572726F723A2072656E85
:101BC00065776564206661696C000A4E6F206C69F8
:101BD0006E6B00526573746F72696E6720636F6E0F
:101BE0006669672066726F6D20454550524F4D0003
:101BF000416363657074696E6720636F6D6D616EBC
:101C000064732E2E2E0A004E6F204D5154542063C3
:101C10006F6E66696775726564004C6F6164696EAA
:101C20006720636F6E6669672066726F6D20706FE4
:101C30007274616C2064697361626C65642E2075D6
:101C4000736520676574204F4E20746F20656E6148
:101C5000626C6500436F6E66696720697320766108
:101C60006C696400436F6E74696E75652077697482
:101C7000682070726576696F75736C79206C6F611E
:101C800064656420636F6E6669670000002200254A
:101C90000028002B002E0031003400020100000556
:101CA0000108010B0100000A0B02090C0D0E0807C8
:101CB000030401000000000000000000000000001C
:101CC0000000000000000000000000000000000014
:101CD00000121110000000000000000000000000D1
:101CE00000000000000000000000000000210024AF
:101CF0000027002A002D00300033000101000004FD
:101D00000107010A010102102020080810204010DC
:101D100020408002010201080402010102040810AF
:101D200020408080402010080402018004020180CD
:101D300040201008040201080402010102040810F6
:101D40002040800102040810204080050505050799
:101D50000508080808020202020A0A080804040426
:101D60000401010101010101010303030303030352
:101D700003040707070C0C0C0C0C0C0C0C020202E1
:101D80000206060606060606060B0B0B0B0B0B0BD4
:101D90000B2F64617461002F736B6574636800417D
:101DA00063636573732D436F6E74726F6C2D526530
:101DB00071756573742D507269766174652D4E6509
:101DC00074776F726B3A2074727565004163636556
:101DD00073732D436F6E74726F6C2D416C6C6F77E3
:101DE0002D486561646572733A202A00416363651A
:101DF00073732D436F6E74726F6C2D416C6C6F77C3
:101E00002D4D6574686F64733A20504F53542C47BE
:101E100045542C4F5054494F4E53004163636573F2
:101E2000732D436F6E74726F6C2D416C6C6F772DD8
:101E300043726564656E7469616C733A207472757F
:101E400065004F5054494F4E530044454C4554454E
:101E5000005055540047455400504F53540061758D
:101E600074686F72697A6174696F6E3A20004175A7
:101E700074686F72697A6174696F6E3A2000436F9B
:101E80006E74656E742D4C656E6774683A20006FD1
:101E9000637465742F73747265616D00696D616739
:101EA000652F6A70656700696D6167652F67696690
:101EB00000746578742F68746D6C006170706C6963
:101EC000636174696F6E2F6A736F6E0074657874E6
:101ED0002F706C61696E00436F6E74656E742D5463
:101EE0007970653A2000436F6E6E656374696F6E3A
:101EF0003A20636C6F7365004163636573732D43B0
:101F00006F6E74726F6C2D416C6C6F772D4F7269B0
:101F100067696E3A202A00556E6B6E6F776E004EC1
:101F20006F74204D6F646966696564004F4B004DA6
:101F30006F766564207065726D616E656E746C7924
:101F400000496E7465726E616C20536572766572BD
:101F5000204572726F72005061796C6F6164205419
:101F60006F6F204C61726765004E6F7420666F75ED
:101F70006E64005757572D41757468656E746963B8
:101F80006174653A204261736963207265616C6DAA
:101F90003D22416363657373207265737472696374
:101FA0007465642200556E617574686F72697A6534
:101FB00064005061796C6F61642073697A65207781
:101FC000726F6E670042616420726571756573742B
:101FD00000485454502F312E3120002000000000C2
:101FE0000000000000004F4E000000000000004F05
:101FF0004646000000000000524553540000000017
:1020000000544F47474C4500000048414C540000E5
:10201000000000584F4E000000000000584F464698
:102020000000000000494E435245415345004445DD
:1020300043524541534500454E41424C4500000046
:1020400044495341424C450000554E465245455A7D
:102050004500465245455A450000004155544F0041
:102060000000000046414E5F4F4E4C590048494722
:102070004800000000004D454449554D0000004C0B
:102080004F57000000000000484541540000000088
:1020900000434F4F4C000000000044525900000024
:1020A00000000053544F500000000000524742000F
:1020B0000000000000485356000000000000577266
:1020C0006F6E67207061796C6164004354524C2FCD
:1020D0007478743A204F75744F664D656D6F7279E0
:1020E0003A2000202D3E2041543A004368616E2082
:1020F000747970653A004E6F2073746F7265642056
:1021000076616C756573202D2064656661756C74ED
:102110003A20002D3E005075623A20006374726CC4
:1021200000454E41424C4500465245455A45004403
:10213000495341424C45002D3E005075623A200003
:10214000636D640046414E5F4F4E4C5900445259F6
:1021500000434F4F4C0048454154004155544F00F7
:102160002D3E005075623A20007365740064656C02
:10217000002D3E005075623A20002D3E00507562E1
:102180003A2000556E6B6E6F776E20636D64200A87
:10219000004F4646004F4E0053617665642045541B
:1021A00041473A0053657420455441473A200000A6
:1021B00079C1BCAF11241FBECFEFD1E2DEBFCDBFCE
:1021C00000E00CBF15E0A0E0B2E0E8E8FCEA01E0C6
:1021D0000BBF02C007900D92A239B107D9F72AE0D0
:1021E000A2E9B5E001C01D92A437B207E1F710E102
:1021F000C9EDD0E100E006C021970109802FFE0162
:102200000E9414CEC83DD10780E00807A9F70E94BC
:10221000CEAF0C9432D60C940000FC01818D928DCF
:102220000895FC018489958908952DEA33E0FC0125
:1022300031832083FB014089518962897389FC01C4
:1022400042835383648375830895DC01ED91FC918F
:10225000048CF58DE02D1994CF93DF931F92CDB7A9
:10226000DEB76983DC01ED91FC910280F381E02D02
:1022700041E050E0BE016F5F7F4F19950F90DF91F5
:10228000CF910895FC019485FB018485981303C0C8
:1022900081E0943009F480E0089521E0FC01848518
:1022A000843009F420E0822F08950895CF93DF93BE
:1022B0001F92CDB7DEB76983DC01ED91FC910280FE
:1022C000F381E02D41E050E0BE016F5F7F4F199533
:1022D0000F90DF91CF910895DC01ED91FC91068C78
:1022E000F78DE02D199591E089270895862F08959F
:1022F00081E086270895DC0180E0615038F0ED919F
:10230000E827F0E0EE5DF84E8491F7CF0895FC01E8
:10231000818191E09093E007809302081092E10799
:1023200010920308089520913F06260F3327331F8C
:1023300021323105ECF42091DA07FC0190E080E0D5
:10234000243069F082E00895A0913F062191AC010C
:10235000435E594FA40FB52FB11D2C9301968617DC
:1023600098F380913F06680F60933F0680E00895E0
:1023700081E0089508950895E091650680916406CE
:10238000E81730F4F0E0EA59F94F808190E00895C1
:102390008FEF9FEF089590916506809164062FEF6F
:1023A0003FEF981748F4E92FF0E0EA59F94F208100
:1023B00030E09F5F90936506C9010895809164069F
:1023C00090916506891B990B0895CF92DF92EF9249
:1023D000FF920F931F93CF93DF937C01CB018A0170
:1023E0002091E007222389F0EB016B01C40ED51E7A
:1023F000CC15DD0569F06991D701ED91FC91019053
:10240000F081E02DC7011995F3CF642F0E9493113D
:10241000C801DF91CF911F910F91FF90EF90DF9056
:10242000CF900895CF93DF931F92CDB7DEB7698326
:102430002091E0072223F9F020910308203258F080
:1024400021E030E0FC013383228390E080E00F90B4
:10245000DF91CF9108958091E107E82FF0E0EE51F0
:10246000F84F998190838F5F8093E10780930308F1
:1024700081E090E0ECCF61E0CE0101960E949311E3
:10248000F7CF90E0FC01E55BF24EE491F0E0EE0F57
:10249000FF1FE557F34EA591B4912C918B5F924E9F
:1024A000FC018491822391E009F490E0892F089542
:1024B000FC01DC018D918111FDCF30E020E050E086
:1024C00040E08AE09191992301F1443051055CF597
:1024D0009E3271F42F3F310509F02CF5DB01A40F7A
:1024E000B51F12962C934F5F5F4F30E020E0EACF8C
:1024F000829FD001839FB00D1124292F990F330B98
:10250000205331092A0F3B1FDDCF2F3F310509F042
:1025100054F4443051053CF4640F751FFB012283D1
:1025200081E090E0089590E080E008959FE9980FA1
:10253000963010F4875508959FEB980F963010F45D
:102540008753089580538A3008F080E00895DC01B5
:1025500015968D919C91009739F0DC01ED91FC91DD
:102560000680F781E02D19940895089583E090E0A6
:1025700008958091B5059091B6050895FC01848178
:1025800095810895DC011196EC911197E295EF7019
:10259000E150EB3008F039C0F0E08827ED52FD4EF5
:1025A0008F4F0C9414CEF612F6120513DE12DE12C3
:1025B000E712FE12FE12FE12DE12DE1214966D916A
:1025C0007D918D919C9117970E9446CC0895149609
:1025D0006D917D918D919C91179724E630E040E0BC
:1025E00050E00E94ABCDCA01B901EECF14966C91B8
:1025F00070E090E080E00E9444CC089514966D91C4
:102600007D918D919C911797089560E070E0CB01CA
:102610000895FC01A7812A2F2E7FD1F08181829518
:102620008F7081508330A0F4A695A150BB0B2BE591
:1026300031E00E942BCE24E630E040E050E00E94E2
:10264000ABCDDA01C90187569F4FAF4FBF4F0895F9
:102650008FEF9FEF0895DC01ED91FC91309729F009
:102660009085977081E0953009F080E00895FC0135
:10267000A481B581109721F118969C9118979770B5
:102680008EEF890F823010F091111AC019964D9378
:102690005D936D937C931C97A481B58118969C9152
:1026A0001897987F926018969C930480F581E02D8E
:1026B0008085982F987F903319F487708065808784
:1026C0000895DC0119968D919C91009739F0DC01F9
:1026D000ED91FC910280F381E02D19940895CF9340
:1026E000DF93EC01E881F9810484F585E02D1995EB
:1026F00029893A892F5F3F4F3A8B298BDF91CF9100
:102700000895CF93DF93EC018E8581110DC081E098
:1027100090E049895A892C853D854217530708F076
:1027200080E0DF91CF910895E881F9810484F585F7
:10273000E02DCE0119958F3F910549F780E090E09B
:10274000F0CFFC01848595856817790708F4CB01E3
:10275000928B818B0895DC011E962C911E9722236B
:1027600039F0ED91FC910190F081E02D6FEF19941B
:102770000895FC0187859089089581E0089590E08F
:1027800080E00895CF93DF93CDB7DEB760970FB6A3
:10279000F894DEBF0FBECDBF19821A821B821C8245
:1027A0001D821E821F8218868A818F7080618A83B3
:1027B0006FEF3E819F81888529817A815B814C8181
:1027C0004C873E87888B372F452F5C857E85892FE8
:1027D000988960960FB6F894DEBF0FBECDBFDF912B
:1027E000CF9108950F931F93CF93DF9300D000D024
:1027F0001F921F92CDB7DEB781E028960FB6F894EE
:10280000DEBF0FBECDBFDF91CF911F910F91089515
:10281000CF92DF92EF92FF920F931F93CF93DF93AC
:10282000CDB7DEB7AF970FB6F894DEBF0FBECDBF02
:102830007C016A010DEA13E01A8309831C861B865A
:1028400088EE93E0A0E0B0E08D879E87AF87B88BDD
:1028500085E893E09A878987188F0F8B198E1A8ED7
:102860001B8E1C8E84E089A31BA70AA71CA61DA68D
:102870001EA61FA68091330890913408A0913508B8
:10288000B09136088EA39FA3A8A7B9A78B839C837A
:10289000AD83BE8318861F82AE01465D5F4FCE01B9
:1028A00001960E94158981309105B1F4D701ED910F
:1028B000FC910488F589E02D1DA30CA38CA59DA592
:1028C000AEA5BFA58EA39FA3A8A7B9A7A601BE01C9
:1028D0006C5D7F4FC7011995AF960FB6F894DEBFB8
:1028E0000FBECDBFDF91CF911F910F91FF90EF9061
:1028F000DF90CF900895CF92DF92EF92FF920F93E7
:102900001F93CF93DF93CDB7DEB7AF970FB6F89491
:10291000DEBF0FBECDBF7C016A010DEA13E01A8352
:1029200009831C861B8688EE93E0A0E0B0E08D87CB
:102930009E87AF87B88B85E893E09A878987188F41
:102940000F8B198E1A8E1B8E1C8E84E089A31BA7F9
:102950000AA71CA61DA61EA61FA68091330890914B
:102960003408A0913508B09136088EA39FA3A8A77C
:10297000B9A78B839C83AD83BE8318861F82AE016B
:10298000465D5F4FCE0101960E9415898130910509
:10299000B1F4D701ED91FC910684F785E02D1DA3DC
:1029A0000CA38CA59DA5AEA5BFA58EA39FA3A8A78C
:1029B000B9A7A601BE016C5D7F4FC7011995AF96FF
:1029C0000FB6F894DEBF0FBECDBFDF91CF911F9140
:1029D0000F91FF90EF90DF90CF900895CF93DF930A
:1029E000EC01888D843061F00E94DB8EE88DF0E090
:1029F000EE0FFF1FE157F94F1182108284E0888F9C
:102A0000DF91CF910895EF92FF921F93CF93DF93C1
:102A1000FC01208D243039F080E0DF91CF911F91AF
:102A2000FF90EF9008957B01EC0110E0812F0E9450
:102A30009E8F81110FC0188F888D843069F3FD86B9
:102A4000EC861A8E198E20E0A70162E00E94EF8EBC
:102A500081E0E3CF883179F31F5F143039F7ECCF91
:102A60000F931F93182F0E94BEA204C096958795BE
:102A7000779567951A95D2F78B019C010150110942
:102A8000210931090E3F1F4F2F4F3F4F20F061E0CA
:102A900070E080E090E01F910F9108950F931F93D5
:102AA000CF93DF931F92CDB7DEB78C01DC01ED91A0
:102AB000FC910084F185E02D1995892B79F0BE01F8
:102AC0006F5F7F4FF80184850E94A087898190E025
:102AD0000F90DF91CF911F910F9108958FEF9FEF8E
:102AE000F7CFFC0184850C940388CF93DF931F926A
:102AF000CDB7DEB741E050E0BE016F5F7F4FFC0114
:102B000084850E9403881816190634F4898190E0A0
:102B10000F90DF91CF9108958FEF9FEFF9CFFC01D8
:102B20008485843011F00C94E18790E080E0089572
:102B3000CF93C62F0E94871161EE89E398E00E942F
:102B400012126C2F89E398E00E941212CF910C941C
:102B500076A01092DA0781E08093D9071092B4072B
:102B600061E084E10E94DA9E61E085E10E94DA9EE4
:102B7000E9EBF0E080818E7F808380818D7F808390
:102B800088E48093B80085E48093BC0008956CEEDF
:102B900071E1811102C06EEE71E186EC98E00C9457
:102BA0000C826EE37FE086EC98E00E940C82F0E0FD
:102BB000E0E0199584EF91E008956AE779E08111EA
:102BC00002C065E779E087E799E00C940C82DC01AC
:102BD00055962C915597273781F4ED91FC91008CF7
:102BE000F18DE02D199569E376E087E799E00E9481
:102BF0000C8287E799E00C94158108954F925F92BB
:102C00006F927F92AF92BF92DF92EF92FF920F93FB
:102C10001F93CF93DF9300D000D0CDB7DEB77C01F8
:102C2000D62E80911906882309F4BEC0D7011496C8
:102C30009C9180910402891708F4B6C08091170610
:102C400090911806BAE06B13F0C089539A4FFC01BB
:102C50001082D70118960D911C910115110509F4E8
:102C60009FC0F801618572856115710591F44580F9
:102C70005680678070848091270890912808A091E1
:102C80002908B0912A08481659066A067B0609F4F5
:102C900087C0D8011B964D915C911C974115510539
:102CA00009F47EC0F701248153968C91539790E0EC
:102CB000322F377002C0959587953A95E2F780FFDD
:102CC0006FC0A22EB12CC501887F9370892B39F477
:102CD00051968D919C91887F9370A82AB92AD8012A
:102CE0008D919C91DC01ED91FC916115710509F4C8
:102CF00086C00688F789E02D1995019709F050C024
:102D00006CE3F801808191810E941981A50170E036
:102D100060E02AE0D8018D919C910E94C980F80161
:102D200022818081918168EC76E1222311F066ECAA
:102D300076E10E940C82D8011D966D917C911E97C0
:102D40008D919C910E94A68160E2F8018081918121
:102D50000E941981D8011F966D917C9150978D9199
:102D60009C910E94A681F8012281808191816BEB68
:102D700076E1222311F065EB76E10E940C8267EC8C
:102D800075E0D8018D919C910E94A681F801808107
:102D90009181DC01ED91FC91008CF18DE02D199574
:102DA0001092180610921706D70115968D919C91D6
:102DB0001697009771F014963C9120910502231705
:102DC00040F0DC01ED91FC910190F081E02D6D2D42
:102DD000199581E090E026960FB6F894DEBF0FBEFD
:102DE000CDBFDF91CF911F910F91FF90EF90DF90BA
:102DF000BF90AF907F906F905F904F900895048840
:102E0000F589E02D2DEA33E03A832983D801159620
:102E10004D905D906D907C9018974B825C826D8296
:102E20007E82BE016F5F7F4F67CF8F3491050CF0BC
:102E3000BBCFBDE06B1709F4B7CF9C012F5F3F4FAD
:102E4000309318062093170689539A4FFC0160832C
:102E5000ABCF0C94ADC4CF93C1E068EE73E080E0DB
:102E600090E00E9479A06C2F86EC98E00E94C797B2
:102E7000CF5FC43191F784EF91E0CF910895CF9364
:102E8000DF93009709F490C0FC012081222309F40C
:102E90008BC0EC0169E671E20E944AC6892B09F4F5
:102EA0005FC06CE171E2CE010E944AC6892B09F431
:102EB0005AC060E471E2CE010E944AC6892B09F42F
:102EC00055C068EA76E0CE010E944AC6892B09F413
:102ED00050C064EA76E0CE010E944AC6892B09F40C
:102EE0004BC060EA76E0CE010E944AC6892B09F405
:102EF00046C06CE976E0CE010E944AC6892B09F4EF
:102F000041C068E976E0CE010E944AC6892BE9F10A
:102F100064E976E0CE010E944AC6892BC9F16FE8C8
:102F200076E0CE010E944AC6892BA9F16BE876E0D3
:102F3000CE010E944AC6892B89F16DE671E2CE016D
:102F40000E944AC6892B69F167E876E0CE010E94AB
:102F50004AC6892B49F58DE090E0DF91CF91089525
:102F600082E090E0FACF89E090E0F7CF81E090E056
:102F7000F4CF88E090E0F1CF85E090E0EECF86E0FE
:102F800090E0EBCF87E090E0E8CF8AE090E0E5CFFB
:102F90008BE090E0E2CF8CE090E0DFCF83E090E048
:102FA000DCCF84E090E0D9CF90E080E0D6CFCF9323
:102FB000DF93EC0163E076E187E799E00E940C8201
:102FC0006C817D8187E799E00E94CE976DEF75E176
:102FD00087E799E00E940C8287E799E00E941581BB
:102FE00060E08C810E94089F1092B6051092B50592
:102FF00081E090E0DF91CF910895EF92FF921F93CF
:10300000CF93DF93192F7B01C82FD92FD7FF03C090
:10301000D195C195D10961E08C2F0E94089F82E073
:10302000E816F10499F460E08C2F0E94DA9E6BEDB3
:1030300074E187E799E00E940C8287E799E0DF91CD
:10304000CF911F91FF90EF900C941581612FEF2885
:1030500051F46095661F6627661F8C2F0E94DA9ECA
:1030600067ED74E1E6CF661F6627661F8C2F0E940E
:10307000DA9E62ED74E1DDCFCF93DF9300D000D014
:103080001F921F92CDB7DEB7E0EBF8E0128A118AEB
:1030900080E090E19587848784E890E0948B838B2F
:1030A00081E0868780E090E2908B878787E7858B39
:1030B0001C821B828FE792E09A838983FE83ED83D3
:1030C0008FEF9FEF98878F836EE575E186EC98E030
:1030D0000E940C826091B0057091B105CE010196FD
:1030E0000E940F8480EB98E00E94E7156EE475E182
:1030F00086EC98E00E940C8286EC98E00E94158194
:103100000E944FA928960FB6F894DEBF0FBECDBF20
:10311000DF91CF91089565E0FC01808191810E944B
:103120009F93009751F0FC018085982F987F29F09C
:1031300086958695869590E0089590E080E00895C4
:10314000FC0186819781009799F0FC01208527700A
:10315000223029F461857285838594850895253010
:1031600039F460E00E949F93009711F0FC01F2CFC8
:1031700060E070E0CB010895CF93C62F63E0FC01BF
:10318000808191810E949F93FC01892B11F1908590
:10319000892F8570F1F4987F926090878185928560
:1031A000A385B4858827BB278C2B81879287A3872B
:1031B000B4876DEA76E087E799E00E940C826C2F75
:1031C00087E799E00E94C79787E799E0CF910C9431
:1031D0001581CF91089563E0FC01808191810E9467
:1031E0009F93009719F0FC01818508958FEF089552
:1031F000FF920F931F93CF93DF93CDB7DEB7649702
:103200000FB6F894DEBF0FBECDBF8C01F62E8FE255
:1032100090E09A838983FE01339688E0DF011D9256
:103220008A95E9F7F8016681FF2011F081E06827AF
:10323000D80114968C910E94DA9EF80187819085BE
:10324000A185B285883E9340A105B10508F48BC0E5
:1032500069E476E187E799E00E940C82D801149630
:103260006D917C9187E799E00E94CE9764E476E1C6
:1032700087E799E00E940C826F2D70E087E799E064
:103280000E94CE9787E799E00E9415816BE676E170
:10329000CE0101960E943FC6F801828193810E946F
:1032A000EB18FF2009F46BC06CE376E1843151F038
:1032B00065E376E1853131F069E276E18F3011F432
:1032C00061E376E1CE010B960E9453C664E176E19C
:1032D00087E799E00E940C82D8011296ED91FC914B
:1032E00013970190F081E02D60817181ED91FC9147
:1032F0000288F389E02D9E012F5F3F4FAE01455FAD
:103300005F4FC8011995BC0187E799E00E94CE97ED
:1033100062E176E187E799E00E940C82D80112967B
:10332000ED91FC910190F081E02D6081718187E742
:1033300099E00E94A681BE016F5F7F4F87E799E009
:103340000E94A6816FE076E187E799E00E940C82F7
:10335000BE01655F7F4F87E799E00E94A68187E7FE
:1033600099E00E94158164960FB6F894DEBF0FBEF7
:10337000CDBFDF91CF911F910F91FF90089565E22E
:1033800076E1823009F49ECF60E276E19BCFCF9266
:10339000DF92EF92FF920F931F93CF93DF93CDB7FE
:1033A000DEB760970FB6F894DEBF0FBECDBF7C01CD
:1033B0006B01CA01B9012AE0AE014F5F5F4F0E9465
:1033C000EEC6D701ED91FC910288F389E02D9801BA
:1033D000AE014F5F5F4FB601C701199560960FB6FA
:1033E000F894DEBF0FBECDBFDF91CF911F910F913B
:1033F000FF90EF90DF90CF900895892B71F0FB0143
:10340000828193810E94469565E671E186EC98E0A1
:103410000E940C8288EC90E0089590E080E0F2CF6A
:10342000892B71F0FB01828193810E94F8946EE4F4
:1034300071E186EC98E00E940C8288EC90E008959F
:1034400090E080E0F2CFEF92FF920F931F93CF9323
:10345000DF93CDB7DEB72C970FB6F894DEBF0FBE63
:10346000CDBF8C017B018DEA93E09A8389831B8217
:103470001C821D821E8298878F8319861A861B865E
:103480001C8605301105ECF0BE01695F7F4FF70126
:10349000808591850E945812892B99F0CE0107965C
:1034A0000E94E995BE01695F7F4FF7018681978190
:1034B0000E945812892B61F0CE0107960E949396C4
:1034C0000EC0CE0101960E94E9950430110554F713
:1034D000CE0101960E94939603301105A4F1BE011E
:1034E000695F7F4FF701848195810E945812892B73
:1034F00051F1CE0107960E943E96BE01695F7F4F53
:10350000F701828193810E945812892B19F1CE0113
:1035100007960E94949567E271E186EC98E00E941C
:103520000C8280E00E947D9788EC90E02C960FB68C
:10353000F894DEBF0FBECDBFDF91CF911F910F91E9
:10354000FF90EF900895CE0101960E943E960230C2
:1035500011059CF6CE0101960E949495013011054B
:10356000D1F6CE0101960E9494956EE271E186EC4F
:1035700098E00E940C82CFCF0F931F93CF93DF93DD
:103580008C01EB010297C4F08A819B810E94DEC509
:103590008093050299270E9490970230110549F007
:1035A0008C819D810E94DEC58093040299270E9430
:1035B0009A97C8ECD0E002C0C0E9D1E063E171E1C4
:1035C00086EC98E00E940C826091050286EC98E0FF
:1035D0000E94C7976EEF70E186EC98E00E940C8223
:1035E0006091040286EC98E00E94C79786EC98E010
:1035F0000E941581CE01DF91CF911F910F91089507
:10360000CF93DF93EB010297A4F169EE71E18A8118
:103610009B810E942CC6892B29F40E94E8966F7723
:103620000E942D9765EE71E18A819B810E942CC6D4
:10363000892B29F40E94E89660680E942D976DEE10
:1036400070E186EC98E00E940C820E94E8966095FA
:10365000661F6627661F70E086EC98E00E94CE9792
:1036600086EC98E00E94158188EC90E0DF91CF9184
:1036700008950E943C18F8CFCF92DF92EF92FF920C
:103680000F931F93CF93DF93EC016A017B018E812F
:103690009F81892BD9F4888199810E94D697082F20
:1036A00010E00530110594F40E941F86009721F068
:1036B000FC012085287F20879F838E83BC01888121
:1036C00099810E94A6970F5F1F4FEBCFEE81FF817C
:1036D000309749F18085982F977019F5887F82601F
:1036E0008087EE81FF81C186D286E386F48665EB12
:1036F00076E087E799E00E940C822AE030E0B7018B
:10370000A60187E799E00E94208187E799E0DF9191
:10371000CF911F910F91FF90EF90DF90CF900C947D
:1037200015819230F1F2DF91CF911F910F91FF90AF
:10373000EF90DF90CF9008958F929F92AF92BF92BB
:10374000CF92DF92EF92FF920F931F93CF93DF936D
:10375000EC01888199810E94D697082F10E00430EF
:10376000110584F40E941F86009721F0FC0120853A
:10377000287F2087BC01888199810E94A6970F5FCE
:103780001F4FEDCF60E0888199810E949F937C015B
:10379000009751F1FC0180858770843039F5C18430
:1037A000D284C114D10401F1F60180818823E1F0B3
:1037B00082E0882E8AE0982EB12CA12C1A2DC4010B
:1037C0000E945AC6AC01B401C6010E9473C6892B7F
:1037D00009F4AAC0FFEFAF1ABF0A89E0880E911C56
:1037E000E7E1AE16B10451F71FEF03C08230E1F7F5
:1037F00011851887C880D98061E0C6010E949F9317
:103800007C019B838A8362E0C6010E949F939D8313
:103810008C8364E0C6010E949F939F838E83103146
:1038200009F057C08BE090E00E9411C48C01FC01AC
:10383000D383C28384E392E0918380831682CE0196
:103840000E94E69797FD52C0F80195838483F801A2
:1038500084819581009719F0863491052CF080E2DF
:1038600090E0F80195838483E114F10409F44EC0DB
:10387000F70180858770853009F048C0C7010E9434
:10388000D697823008F442C061E0C7010E949F933E
:10389000FC01892BD9F180858770823081F56185A3
:1038A0007285838594850E9446CC20E030E04AE70B
:1038B00054E40E94A5CC0E9418CF611571058105C2
:1038C000910541F1F80167837087818792871A8794
:1038D0000987DF91CF911F910F91FF90EF90DF90BB
:1038E000CF90BF90AF909F908F90089591958195C4
:1038F0009109F8019583848381E08683A8CF833082
:1039000029F46185728583859485CFCF60E070E06E
:10391000CB01CBCF88E893E1A0E0B0E0F80187834A
:103920009087A187B287D3CFC6010E949D838A2D3D
:1039300090E0B0E0A0E0F70181879287A387B48789
:103940008085887F8260808754CFCF93DF93EC019E
:10395000798368831A8619861B861C8E1B8E0E94AB
:103960002B13882329F0CE01DF91CF910C949C1B5F
:10397000DF91CF910895EF92FF920F931F93CF9312
:10398000DF93EC018B011D821C821A821B82E8806E
:10399000F980E114F10409F472C08091B0059091AE
:1039A000B105892B09F46BC0672B09F48701F80175
:1039B000808587708630A9F46FEA73E0C8010E94A1
:1039C0002793009719F0FC0181858A8364E875E0EC
:1039D000C8010E942793009709F458C0FC01818513
:1039E0008B8361EB73E0C7010E942793009709F076
:1039F00043C06FE376E087E799E00E940C826B8119
:103A000087E799E00E94C7976DE376E087E799E042
:103A10000E940C826A8187E799E00E94C79787E736
:103A200099E00E941581E880F9800E941F868C0130
:103A30000097D1F0FC018085887F826080871186A5
:103A400012861386148680819181009711F00E945E
:103A50009D8381EB93E00E94CC83F8019183808366
:103A6000B801C7010E94A69761EB73E08881998134
:103A70000E942793009719F009969D838C83DF910C
:103A8000CF911F910F91FF90EF900895F8018081E1
:103A900091810E94DEC5A4CF1F93CF93DF93FC01D9
:103AA000162FC389D489818992899C012F5F3F4F4A
:103AB000328B218BC80FD91FCE010E9463CD1817FE
:103AC00021F0612FCE010E946BCD81E090E0DF916B
:103AD000CF911F910895FC018189928924853585B4
:103AE0008217930740F423893489820F931F0E9421
:103AF00063CD90E008958FEF9FEF08952F923F924E
:103B00004F925F926F927F928F929F92AF92BF92ED
:103B1000CF92DF92EF92FF920F931F93CF93DF9399
:103B2000CDB7DEB762970FB6F894DEBF0FBECDBF3C
:103B30005C014B0129013A01CA01B9010E9411CF70
:103B40001B013F926F938FEE93E09F938F93CE0173
:103B500001967C019F938F930E94FAD20F900F9051
:103B60000F900F900F900F9020E030E0A901C3015B
:103B7000B2010E9447CF181624F077FA709477F8B4
:103B80007094F70101900020E9F731976F01CE188A
:103B9000DF088EE28083A2E0B0E0AC0FBD1FAC0D69
:103BA000BD1DBA8BA98BB10137FE03C0719561951C
:103BB0007109072E000C880B990B0E9446CC9B01C3
:103BC000AC01C301B2010E9432CE20E030E040E2FD
:103BD00051E40E94A5CC0E9411CF605DE989FA8969
:103BE0006083FE01EC0DFD1D1382D501ED91FC916A
:103BF0000288F389E02D9801A701B401C501199548
:103C000062960FB6F894DEBF0FBECDBFDF91CF91A5
:103C10001F910F91FF90EF90DF90CF90BF90AF90EA
:103C20009F908F907F906F905F904F903F902F90DC
:103C300008959B0190E00496982F8827642F820FA7
:103C4000931F0C948587CF93DF93C82FD0E02496E1
:103C5000DC2FCC27C60FD71F0E940A878FE00E9457
:103C60001F878D2F0E941F878C2F0E941F8780E047
:103C70000E941F87C82F0E9408878C2FDF91CF9149
:103C80000895CF93DF93C82FD62F472F60E170E0C0
:103C90000E94191E4D2F61E170E08C2FDF91CF91B2
:103CA0000C94191E90E0982F882744E050E0845F20
:103CB0009B4F0C945687FC018485843011F00C9442
:103CC0009E8F80E00895CF93DF93FC0124852430FC
:103CD000D9F0EC010E945B1E843189F0882379F0D1
:103CE000883169F021E08C3159F4E881F981008450
:103CF000F185E02DCE01199521E0892B09F420E012
:103D0000822FDF91CF91089580E0FBCF44E050E017
:103D1000BC018FE090E00C94568744E050E0BC0179
:103D200085E090E00C94568744E050E0BC0181E0CF
:103D300090E00C94568708958F929F92AF92BF9215
:103D4000CF92DF92EF92FF920F931F93CF93DF9367
:103D5000CDB7DEB72D970FB6F894DEBF0FBECDBF3F
:103D60007C0110E000E038EE832E33E0932EA12C8E
:103D7000B12C45E3C42E43E0D42E1C821B828D82DD
:103D80009E82AF82B886DA82C9820D87CE01019603
:103D90000E945B1E811135C0F7014481558120E0EE
:103DA00061E0802F0E94EF8E80E590E00E94E59C0C
:103DB00063E070E0802F0E94231E833129F462E0CB
:103DC00070E0802F0E94449DF70184819581000F4F
:103DD000111FF801E157F94F918380832D960FB69B
:103DE000F894DEBF0FBECDBFDF91CF911F910F9131
:103DF000FF90EF90DF90CF90BF90AF909F908F900B
:103E000008950F5F1F4F0430110509F0B6CFE6CFBC
:103E1000CF92DF92EF92FF921F93CF93DF93FC013B
:103E20001485143089F1EC0180E590E00E94E59C56
:103E300068E070E0812F0E94449D0E94BEA26B0149
:103E40007C01CE010E945B1E8823A1F062E370E03A
:103E500080E090E00E9479A00E94BEA26C197D09CA
:103E60008E099F09683E73408105910550F38C854A
:103E70000E94DB8EEC85F0E0EE0FFF1FE157F94F5B
:103E80001182108284E08C87DF91CF911F91FF9087
:103E9000EF90DF90CF9008954F925F926F927F9254
:103EA0008F929F92AF92BF92CF92DF92EF92FF924A
:103EB0001F93CF93DF93CDB7DEB72D970FB6F8944E
:103EC000DEBF0FBECDBF7C019FE8A92E96E0B92EC4
:103ED00010E0D12CC12C28EE422E23E0522E612C72
:103EE000712C35E3832E33E0932E1C821B824D828E
:103EF0005E826F8278869A8289821D87D5012D9194
:103F00003D915D01F7018481958128173907B1F44E
:103F1000CE0101960E945B1E843199F1CE0101967B
:103F20000E945B1E8C3151F4CE0101960E948F15C8
:103F3000892B21F4CE0101960E94081F1F5F1430C7
:103F4000A1F6CD2841F4D701ED91FC910084F185D3
:103F5000E02DC70119952D960FB6F894DEBF0FBE60
:103F6000CDBFDF91CF911F91FF90EF90DF90CF9069
:103F7000BF90AF909F908F907F906F905F904F9089
:103F80000895CC24C394D12CD9CF8F929F92AF9215
:103F9000BF92CF92DF92EF92FF920F931F93CF9336
:103FA0006C015B017A01FC01C485C430A1F481E09D
:103FB00090E0F60193838283F12CE12CC701CF912D
:103FC0001F910F91FF90EF90DF90CF90BF90AF9037
:103FD0009F908F9008958A014130584010F000E082
:103FE00018E080E590E00E94E59C8C2F0E94FC9DEB
:103FF0004C0163E070E08C2F0E94231E873111F08A
:104000008C3129F58016910660F380E590E00E94DE
:10401000E59C9801A50170E060E08C2F0E949C9DBA
:1040200060E270E08C2F0E94449D62E070E08C2F73
:104030000E94231E84FD13C063E070E08C2F0E9459
:10404000231E811107C08C2F0E94DB8EB0CF10E0A1
:1040500000E0DBCF80E590E00E94E59CE6CF40E108
:1040600062E070E08C2F0E94191E012B09F0A6CF90
:104070009ECF3F924F925F926F927F928F929F92CC
:10408000AF92BF92CF92DF92EF92FF920F931F9366
:10409000CF93DF93CDB7DEB72D970FB6F894DEBF81
:1040A0000FBECDBF6C015B014A010E944C1F8FE81F
:1040B000E82E86E0F82E312C10E000E098EE492E34
:1040C00093E0592E612C712C1C821B824D825E82E2
:1040D0006F82788685E393E09A8389833D86F70132
:1040E000219131917F01F60184819581281739074B
:1040F00071F4CE0101960E945B1E873141F4A40148
:10410000B501CE0101960E94C51F080F191F3394F7
:10411000F4E03F12D9CFC8012D960FB6F894DEBF58
:104120000FBECDBFDF91CF911F910F91FF90EF9008
:10413000DF90CF90BF90AF909F908F907F906F90C7
:104140005F904F903F900895CF93DF9391E09093CD
:104150001C068823B9F0C091B800D091BA008091B4
:10416000BC008A7B8093BC0060E084E10E94DA9E00
:1041700060E085E10E94DA9E0E94A915D093BA0002
:10418000C093B800DF91CF910895CF92DF92EF9264
:10419000FF920F931F93CF93FC01C1810E94619FF7
:1041A0006B017C018091DA07811164C081E080930A
:1041B000DA078093D9079FEF9093D8071092D7071B
:1041C0001092D6078093B5078091B507CC0FC82B06
:1041D000C093B5078091B407813009F081C0109277
:1041E000B4070E94619F6B017C018091B5078093A9
:1041F000BB008091DC079091DD07A091DE07B091B4
:10420000DF07892B8A2B8B2BA1F00E94619F0091E5
:10421000DC071091DD072091DE073091DF076C1974
:104220007D098E099F09061717072807390708F423
:1042300042C08091BC0083FDD8CF85EC8093BC0048
:104240000E94619F6B017C018091DA07813009F443
:1042500049C08091D707811167C08091D707E6EBED
:10426000F7E0A6E6B6E090E0981751F121912D9382
:104270009F5FFACF8091DC079091DD07A091DE0768
:10428000B091DF07892B8A2B8B2B09F48BCF0E94EF
:10429000619F0091DC071091DD072091DE073091CE
:1042A000DF076C197D098E099F0906171707280774
:1042B000390708F077CF8091DB070E94A42080E0C7
:1042C000109265068093640689E398E00E94CB1102
:1042D000CF911F910F91FF90EF90DF90CF900895B5
:1042E00085EEACCF8091DC079091DD07A091DE07D1
:1042F000B091DF07892B8A2B8B2B09F4A5CF0E9465
:10430000619F0091DC071091DD072091DE0730915D
:10431000DF076C197D098E099F0906171707280703
:10432000390708F091CFC7CF81E099CFAF92BF9204
:10433000CF92DF92EF92FF921F93CF93DF93EC0126
:104340000E94BEA26B017C0128EEC20E23E0D21EA9
:10435000E11CF11C10E08BE4A82EB12C0E94BEA23F
:104360006C157D058E059F0598F460EFCE010E94C7
:104370009815CE010E94C520182F80FF0BC0ED8537
:10438000FE85309709F01995C5010197F1F7E6CF41
:1043900081E08A83812FDF91CF911F91FF90EF9071
:1043A000DF90CF90BF90AF9008951F93CF93DF938E
:1043B000EC01162F0E949621CE010E94871162ED1A
:1043C00089E398E00E941212612F70E06095709569
:1043D00084E0660F771F8A95E1F7612B89E398E007
:1043E0000E9412120E9476A0CE010E94C520811761
:1043F00011F084E08A83DF91CF911F910895CF93CC
:10440000DF93EC0163EC0E949815CE01DF91CF9110
:104410000C94C5200F931F93CF93DF93EC010E9460
:10442000962180FD36C0CE010E94FF2160E0CE01C2
:104430000E94D521CE010E949621CE010E948711B3
:1044400064EB89E398E00E9412120E9476A0CE01EC
:104450000E949621082F10E082FF16C082E08A8316
:104460008881882341F0CE010E94FF21682F61607E
:10447000CE010E94D52115950795802F8170DF917F
:10448000CF911F910F9108958A81823049F71A8246
:10449000E7CF80E0F4CFCF93DF93EC010E94FF21C0
:1044A000682F6460CE01DF91CF910C94D5210F93DA
:1044B0001F93CF93DF93EC01162F042F0E949621B8
:1044C000002319F0CE010E944B22CE010E948711D9
:1044D00065EA89E398E00E941212612F89E398E06F
:1044E0000E941212DF91CF911F910F910C9476A030
:1044F0006F927F928F929F92AF92BF92CF92DF92F4
:10450000EF92FF920F931F93CF93DF93FC012485CB
:1045100021118CC0872E762EEC010E940A2288235E
:1045200009F486C0CE010E94962140E060EFCE01E2
:104530000E94572210E000E066246A94AA24A39403
:10454000B12CE02EE694E694E694F12C802F87704F
:10455000650101C0CC0C8A95EAF78B85082E000C0A
:10456000990B0817190734F5FE01EE0DFF1D938016
:104570009C20CE010E949621CE010E94871168E7FF
:1045800089E398E00E941212992011F080E8982E99
:10459000692D89E398E00E9412120E9476A0CE0154
:1045A0000E949621982F907485FF0BC0992369F083
:1045B0008EEF2AC09924939408171907D1F2912CF1
:1045C000D8CF911102C087FF602EFE01EE0DFF1DB6
:1045D000938187FF28C0C92AC3820F5F1F4F003411
:1045E000110509F0AECF6B86FFEF6F1202C081E0BC
:1045F0008C872396E72DF82DCF01089629912193DA
:10460000E817F907D9F781E0DF91CF911F910F915A
:10461000FF90EF90DF90CF90BF90AF909F908F90E2
:104620007F906F900895C094C922D6CF80E0ECCFE0
:104630008FEFEACFEF92FF920F931F93CF93DF9309
:104640008C017B0140E065E50E945722E70188E08C
:10465000E80EF11C699140E0C8010E945722CE1576
:10466000DF05C1F7DF91CF911F910F91FF90EF9080
:104670000895CF92DF92EF92FF920F931F93CF9303
:10468000DF938C01EB017A01FC01858196810E9408
:104690000A228823C1F1BE01F801858196810E941A
:1046A0001A2340E06EEBF801858196810E94572223
:1046B000E7016701F9E0CF0ED11CF801E580F68033
:1046C000C7010E949621C7010E94871166E989E30C
:1046D00098E00E9412120E9476A0C7010E949621C3
:1046E00061EEC7010E949815C7010E94C5208993F9
:1046F000CC16DD0611F7F801858196810E940A2209
:1047000091E0813009F090E0892FDF91CF911F91E6
:104710000F91FF90EF90DF90CF900895CF93DF93AC
:10472000EA010E943923982F882341F068E0CE01E6
:104730000E947B1191E02885281390E0892FDF915A
:10474000CF910895CF93DF9300D000D000D0CDB7A4
:10475000DEB7AE014F5F5F4F0E948E23882331F09A
:104760008D818F33A9F020F48F31A1F080E007C054
:104770008F3521F08F37D1F78CE001C08BE029967F
:104780000FB6F894DEBF0FBECDBFDF91CF91089575
:104790008AE0F5CF89E0F3CF85ED8093BC0080916E
:1047A000DC079091DD07A091DE07B091DF07079647
:1047B000A11DB11D23E0B695A795979587952A95DC
:1047C000D1F72091BC0024FD03C01092DA070895B0
:1047D0004091DC075091DD076091DE077091DF07A3
:1047E000452B462B472B69F30097A105B10541F0F6
:1047F00025E32A95F1F700000197A109B109E1CF5E
:104800008091DB070C94A4201F920F920FB60F9299
:1048100011240BB60F922F933F934F935F936F9397
:104820007F938F939F93AF93BF93EF93FF93809169
:10483000B900887F803609F44DC008F040C0883246
:1048400009F4A9C028F5803109F49DC0C8F4882373
:1048500009F4FBC0883009F496C0FF91EF91BF9135
:10486000AF919F918F917F916F915F914F913F9108
:104870002F910F900BBE0F900FBE0F901F901895A9
:10488000883109F488C0803241F78093D80714C07A
:10489000803409F49DC040F48033B9F38833E9F6DD
:1048A0008093D80785ECB0C0803509F485C0883581
:1048B00009F496C0883489F60E94CC23CECF88397B
:1048C00009F48CC038F5883729F050F4883611F097
:1048D000803719F683E08093DA071092630657C099
:1048E000883809F47BC0803919F0803809F0B5CFD9
:1048F00080916306803208F071C0E091630681E028
:104900008E0F809363068091BB00F0E0ED5BF94F62
:1049100080833DC0803B39F0E0F4803A09F479C0EF
:10492000883A09F09ACF84E08093DA071092400623
:1049300010923F06E0913D06F0913E061995809158
:104940003F0681110FC081E080933F0610921D0643
:1049500009C0803C09F4A6CF883C09F4A3CF883B6A
:1049600009F07BCFE091400681E08E0F80934006F6
:10497000F0E0E35EF94F80818093BB0090914006A8
:1049800080913F0629C08091B5078093BB0085ECDC
:104990008093BC0062CF9091D7078091D60798177B
:1049A00058F5E091D70781E08E0F8093D707F0E0AC
:1049B000EA54F84F8081E9CFE091D70781E08E0F6C
:1049C0008093D7078091BB00F0E0EA54F84F8083D2
:1049D0009091D7078091D6079817C8F285E8D8CF6D
:1049E000E091D70781E08E0F8093D7078091BB00BD
:1049F000F0E0EA54F84F80838091D90781115CCFB1
:104A000081E08093B40784EA8093BC001092DA07B7
:104A100024CF85EC8093BC001092DA078091630666
:104A2000803230F4E0916306F0E0ED5BF94F1082E4
:104A30006091630670E0E0914106F091420683E4E4
:104A400096E019951092630608CF1092D80734CFDC
:104A50004F925F926F927F92AF92BF92CF92DF920E
:104A6000EF92FF920F931F93CF93DF9300D01F928B
:104A7000CDB7DEB72B013C0129833A834B835C839E
:104A8000A6019501C801B701640D751D861D971D0E
:104A9000211531054105510511F00E9489CD29816B
:104AA0003A814B815C816217730784079507D0F4C4
:104AB000241535054605570530F521E0822F0F9066
:104AC0000F900F900F90DF91CF911F910F91FF905A
:104AD000EF90DF90CF90BF90AF907F906F905F90FE
:104AE0004F900895461657066806790650F421E05F
:104AF00089819A81AB81BC8184159505A605B7058E
:104B0000E8F220E0DBCF21E046165706680679067A
:104B1000A8F2F7CF8F929F92AF92BF92CF92DF927F
:104B2000EF92FF920F931F93CF93DF937C014A0183
:104B30005901C0911A06D0911B06062F660F110B62
:104B4000209709F45CC088858770863009F055C0CD
:104B500064EB73E0CE010E9427936C0182E088161B
:104B6000910449F069EB73E0E3E08E16910429F0BB
:104B7000D0E0C0E006C06DEB73E0CE010E94279349
:104B8000EC01C114D104D9F1F6018085877084301D
:104B9000B1F561857285A801C7010E94A3D2A80161
:104BA00062EC73E0C7010E9485D2209779F1888575
:104BB0008770843059F569857A85A801C7010E94FC
:104BC00085D2A80162EC73E0C7010E9485D2A114CE
:104BD000B10429F0A801B501C7010E9485D2C7011F
:104BE000DF91CF911F910F91FF90EF90DF90CF90C9
:104BF000BF90AF909F908F900895D0E0C0E0A80143
:104C00006BED76E1C7010E9481C6C9CFF2E08F1635
:104C1000910481F083E08816910429F06091880660
:104C200070918906CACFA80165ED76E1C7010E949F
:104C300063C6C7CFA80162ED76E1F8CFCF92DF92CD
:104C4000EF92FF920F931F93CF93DF93CDB7DEB711
:104C5000C154D1090FB6F894DEBF0FBECDBF6C01B1
:104C6000AB0130E020E060E4CE0101967C010E94BF
:104C70008A25F70101900020E9F731978F010E197D
:104C80001F09A801B701C6010E9495D2892B11F016
:104C900010E000E0C801CF5BDF4F0FB6F894DEBF35
:104CA0000FBECDBFDF91CF911F910F91FF90EF907D
:104CB000DF90CF900895CF92DF92EF92FF920F9303
:104CC0001F93CF93DF93CDB7DEB7C054D1090FB692
:104CD000F894DEBF0FBECDBF8091970690919806E5
:104CE000059709F449C06115710509F445C06901CA
:104CF0007A018B0140E450E0CE0101960E94A3D2DC
:104D00006FE270E0CE0101960E946AD2892B41F4D5
:104D1000980143E050E060E4CE0101960E948A25AC
:104D20004FE350E0B601CE0101960E9485D20E9469
:104D30004593882309F180919706909198060697EC
:104D4000D9F480910408811117C0B701CE010196F2
:104D50000E948CA381E090E0C05CDF4F0FB6F89416
:104D6000DEBF0FBECDBFDF91CF911F910F91FF909E
:104D7000EF90DF90CF90089590E080E0EDCFCF935B
:104D8000DF931F921F92CDB7DEB78091680A909192
:104D9000690A009711F484E79AE0BE016F5F7F4FC4
:104DA000681B790B072E000C880B990B0F900F9046
:104DB000DF91CF9108954F925F926F927F928F9281
:104DC0009F92AF92BF92DF92EF92FF920F931F9349
:104DD000CF93DF93CDB7DEB760970FB6F894DEBF01
:104DE0000FBECDBFFC0119861A861B861C869A85CC
:104DF0009F7090669A87A081B181109709F4F7C0DF
:104E00008C91882309F4F3C000811181D8019C9111
:104E1000992309F443C09D3209F4EDC090539A30B0
:104E200028F00F5F1F4F11830083EECFC801D12CF4
:104E3000DC017D01E81AF90A2D91022E000C330BDA
:104E4000205331092A303105A0F35F016EE270E092
:104E5000C8010E946AD2FC01009709F448C0DC0135
:104E60004D018E1A9F0A11968C911197082E000CF5
:104E7000990BC09711960A9798F38181282F082ED5
:104E8000000C330B205331092A30310518F48033DC
:104E90000CF06EC020E030E0A90108C0D12CF12C4C
:104EA000E12CD3CF29E030E040E050E0AAE0B0E0D0
:104EB0000E94CACD2B013C012281822F022E000CC0
:104EC000990BC0978A30910570F420330CF458C0C8
:104ED0002A330CF059C0092E000CAA0BBB0B480E4C
:104EE000591E6A1E7B1E8114910409F052C0C8012C
:104EF0000E94FCC52A852F70206A2A872B013C015D
:104F00006CE270E0D5018D919C910E946AD200976D
:104F100009F068C0F501118210824D865E866F86A9
:104F2000788A88E0FE013996DE01119601900D9293
:104F30008A95E1F729813A814B815C816D817E817F
:104F40008F81988560960FB6F894DEBF0FBECDBFF7
:104F5000DF91CF911F910F91FF90EF90DF90BF9065
:104F6000AF909F908F907F906F905F904F9008953B
:104F70008A330CF097CF032E000C440B550B96CFC1
:104F800080E090E0DC01ABCF89E090E0A0E0B0E011
:104F9000A6CFC801B3E08B169104DCF4E8E0EE166E
:104FA000F104BCF40E94FCC59B01AC01A4E6B0E096
:104FB0000E94CACDDD2041F07094609450944094DA
:104FC000411C511C611C711C460E571E681E791E27
:104FD00097CF0E94DAC52B013C018A858F708067CC
:104FE0008A878ECF0196D5018D939C9396CF412CC5
:104FF000512C320192CFC8010196DD24D39418CFF1
:10500000CF92DF92EF92FF920F931F93CF93DF9394
:10501000EC01A881B981109781F18C91882369F105
:1050200008811981F8019081992351F09D3241F056
:1050300090539A3028F00F5F1F4F19830883F0CFE9
:10504000C8010E94FCC56B017C016CE270E0C801E4
:105050000E946AD2009769F419821882C701B601CA
:10506000DF91CF911F910F91FF90EF90DF90CF9044
:105070000895019699838883F1CFC12CD12C7601B4
:10508000EDCF4F925F926F927F928F929F92AF92ED
:10509000BF92CF92DF92EF92FF920F931F93CF9325
:1050A000DF93CDB7DEB761970FB6F894DEBF0FBEC2
:1050B000CDBF0E94BEA29B01AC016091C30570915F
:1050C000C4058091C5059091C605A12CB12C650140
:1050D00018E8E12E13E1F12E00E010E00E942825EF
:1050E000882319F1E0908606F0908706D701129682
:1050F0008C91823089F566EA76E187E799E00E9433
:105100000C8287E799E00E94158180918606909134
:1051100087060E940A220E94BEA26093C305709374
:10512000C4058093C5059093C60561960FB6F894A3
:10513000DEBF0FBECDBFDF91CF911F910F91FF90CA
:10514000EF90DF90CF90BF90AF909F908F907F9027
:105150006F905F904F9008958091C1059091C20526
:10516000892B09F0DDC083E190E00E9411C48C011D
:105170008DEF96E7F801928B818BF682E58214829F
:10518000108289E0818381E0828383831093C2054A
:105190000093C1050E94BEA26B017C01F0E1CF0E1D
:1051A000F7E2DF1EE11CF11CD8011596ED91FC9190
:1051B00016978FEF838714861382148215821682C6
:1051C000178210861186128614961C929924939445
:1051D000BE01665F7F4FF801858196810E9478222B
:1051E00018160CF071C00E94BEA26C157D058E05CC
:1051F0009F0508F069C067E0CE010A960E947B1106
:1052000099898913E5CFD8018C91811138C0159601
:105210008D919C910E940A22BE01665F7F4FF8012A
:10522000858196810E941A2340E064EBD80115968F
:105230008D919C910E945722F801A580B680C501EE
:105240000E949621C5010E94871167E889E398E0D2
:105250000E94121260E889E398E00E9412120E94F4
:1052600076A0C5010E949621B82ED80115968D9181
:105270009C910E940A22B5FC02C0F8019082AE0106
:105280004F5F5F4FBE01665F7F4FC8010E943923A9
:10529000D8011196BC908A85803109F48CC2BE0178
:1052A000665F7F4FC8010E94A2238B1558F5F80155
:1052B0008181D80111968C93119714968C91149733
:1052C0008F5F14968C9384CF10E000E08091C1052D
:1052D0009091C2052091BF053091C00502171307B8
:1052E000ECF49801B3E0220F331FBA95E1F7609117
:1052F000BD057091BE05620F731F0E94ACA00F5FC9
:105300001F4FE4CF8A85803111F48CE0D2CFBE01EB
:10531000665F7F4FC8010E94A223CBCFFC0112829F
:105320008091BB059091BC052091BF053091C005CF
:10533000821793070CF4D5C00E94BEA22B013C013A
:10534000E0918606F0918706309759F08FEF8387BA
:105350001486138214821582168217821086118693
:1053600012864091BF055091C005E091B705F091BC
:10537000B80590E080E0841795070CF48EC088246F
:105380008394912C8091860690918706009709F46A
:105390008DC02091BF053091C005F3E0220F331F6F
:1053A000FA95E1F76091BD057091BE05620F731F1C
:1053B0000E94782218160CF079C08091BF05909158
:1053C000C00541970CF072C00E94BEA29B01AC01C7
:1053D000A12CB12C650118E8E12E13E1F12E00E0BB
:1053E00010E0C301B2010E94282581115FC0C09066
:1053F000BD05D090BE05A090BF05B090C005850149
:1054000073E0000F111F7A95E1F70C0D1D1D67E089
:10541000C8010E947B11D80117969C91F12CE12CB8
:105420008913B0CFEA14FB040CF057C148E050E0F8
:10543000B801C6010E9424D2B8E0CB0ED11C892B42
:1054400009F04BC0EE0CFF1CE091B705F091B805D8
:10545000EE0DFF1D8081918181609183808360E9E1
:1054600076E187E799E00E940C828091BF059091D8
:10547000C00563E0880F991F6A95E1F72091BD058B
:105480003091BE05820F931F0E94659B69E876E10B
:1054900087E799E00E94308275CF21913191DF0139
:1054A00012972E7F2D933C93019665CF67E976E1A5
:1054B00087E799E00E940C826091BF057091C0055A
:1054C00087E799E00E94CE9787E799E00E941581CF
:1054D0001092BC051092BB051ECEEFEFEE1AFE0A2D
:1054E000A1CF0091BD051091BE059C0143E0220FA4
:1054F000331F4A95E1F7020F131FD8012C91283270
:1055000009F0DBC0AE014F5F5F4FB8018091C1056C
:105510009091C2050E948E23811105C020E030E0E9
:105520004EEF52EC3EC06A8170E0762F6627770F0F
:10553000770F770F2981B8E02B9F90011124262B3C
:10554000372BF80180818031D1F4688570E08F813C
:10555000AB01481B5109CA019695982F882797954A
:1055600087950E9400CECB014097B90113E0660FEA
:10557000771F1A95E1F760789C01260F371F2138B5
:1055800054EE35075CF2B901330F880B990B0E947A
:1055900046CC20E030E040E05CE30E94A5CC9B01DB
:1055A000AC01E091B905F091BA058091BB059091ED
:1055B000BC05BC01A3E0660F771FAA95E1F7A09197
:1055C000BD05B091BE056A0F7B1F309709F0199594
:1055D0000091C1051091C205E090BB05F090BC059B
:1055E00073E0EE0CFF1C7A95E1F78091BD05909178
:1055F000BE05E80EF91ED7018C91803109F463C015
:10560000B701C8010E94A223D82E882309F451C0F3
:10561000F801858196810E940A22882309F449C0F5
:10562000B701D80115968D919C910E941A23F8011B
:10563000408164E4858196810E945722D8011296A8
:105640008C918823B1F1E7EFED0D4EEE842E42E010
:10565000942EE33038F4F0E0EE0FFF1FEF56FD4FCD
:1056600080809180E114F10489F1F801838188231D
:1056700069F1808181112AC00E94BEA22B013C01E8
:10568000092C000CAA08BB08AE014F5F5F4FB701A1
:10569000C8010E943923898181110BC00E94BEA2DA
:1056A000681979098A099B096415750586059705A6
:1056B00058F38091BB059091BC0501969093BC0571
:1056C0008093BB0528CD6CE0D62EA2CFB401990CF7
:1056D000880B990B0E9479A0ECCF8091C105909125
:1056E000C205892B09F44ECE88E0815008F44ACED9
:1056F000F801E80FF11D90819923B9F3AA0CBB1CA6
:105700008091B7059091B805A80EB91ED5018D926C
:105710009C9264E876E187E799E00E940C826091B0
:10572000BF057091C00587E799E00E94CE976DE7AD
:1057300076E187E799E00E940C828091BF05909105
:10574000C00523E0880F991F2A95E1F72091BD0538
:105750003091BE05820F931F0E94659B87E799E0F9
:105760000E9415818091BF059091C00533E0880F9C
:10577000991F3A95E1F76091BD057091BE05680FDC
:10578000791FFB018081883261F48091C10590917D
:10579000C2050E94ACA080918606909187060E9467
:1057A0004B228091BF059091C00501969093C00552
:1057B0008093BF05E7CDFCE0FB1508F478CDA5CDBF
:1057C00060EB74E186EC98E00E940C826DE974E174
:1057D00086EC98E00E940C826FE874E186EC98E019
:1057E0000E940C8267E874E186EC98E00E940C82CB
:1057F00086EC98E00E94158167E774E186EC98E0FA
:105800000E940C826BE674E186EC98E00E940C82A8
:105810006EE574E186EC98E00E940C8269E474E124
:1058200086EC98E00E940C826AE374E186EC98E0D2
:105830000E940C8262E374E186EC98E00E940C8284
:1058400067E274E186EC98E00E940C826AE174E100
:1058500086EC98E00E940C8260E174E186EC98E0AE
:105860000E940C8261E074E186EC98E00E940C8258
:1058700069EF73E186EC98E00E940C826DEE73E1B3
:1058800086EC98E00E940C8263ED73E186EC98E070
:105890000E940C8264EB73E186EC98E00E940C821B
:1058A0006FE973E186EC98E00E940C8262E973E193
:1058B00086EC98E00E940C8264E873E186EC98E044
:1058C0000E940C8268E773E186EC98E00E940C82EB
:1058D00060E773E186EC98E00E940C8265E673E174
:1058E00086EC98E00E940C8268E573E186EC98E013
:1058F0000E940C8260E573E186EC98E00E940C82C5
:1059000065E473E186EC98E00E940C8266E373E143
:1059100086EC98E00E940C826DE273E186EC98E0E0
:105920000E940C826FE173E186EC98E00E940C8289
:1059300061E173E186EC98E00E940C8286EC98E0CD
:105940000C941581009789F0FC0120852770253083
:1059500061F40E949F93009741F0FC01208527701D
:10596000243019F481859285089590E080E00895AF
:10597000CF92DF92EF92FF920F931F93CF93DF931B
:1059800000D000D0CDB7DEB78091190681119AC042
:10599000809197069091980602970CF493C080919D
:1059A000B0059091B105009709F48CC066EC73E0E6
:1059B0000E9427938C01009709F484C00E94D69717
:1059C000E82EF12CE114F10409F47CC070E060E0F1
:1059D000C8010E94A22C6C01EA94EF2809F481C04E
:1059E00061E0C8010E949F93FC0101851285CE01F0
:1059F00001960E94E89CCE0101960E94069D61EBF3
:105A00007CE086EC98E00E940C82B60186EC98E07F
:105A10000E94A6816DEC73E086EC98E00E94A6815E
:105A2000B80186EC98E00E94CE976DEC73E086ECAE
:105A300098E00E94A68163EA77E086EC98E00E94F5
:105A4000A68186EC98E00E94158162E072E085E90B
:105A500099E00E940315D0928B09C0928A09109395
:105A60008D0900938C0983EA97E0892BE9F584EC92
:105A700093E090938F0980938E0980918A0690918C
:105A80008B06009741F070E060E00E94A22C90939A
:105A900089068093880680918806909189060097F0
:105AA00031F190939109809390091092930910928B
:105AB000920981E08093190668E97CE086EC98E021
:105AC0000E940C8226960FB6F894DEBF0FBECDBFA3
:105AD000DF91CF911F910F91FF90EF90DF90CF90CA
:105AE000089502E012E083CF83EA97E0C2CF8AEA0A
:105AF00092E0892B19F484EC93E0D3CF8AEA92E008
:105B0000D0CF2F923F924F925F926F927F928F925F
:105B10009F92AF92BF92CF92DF92EF92FF920F933C
:105B2000CF93DF9300D01F92CDB7DEB77C017A838D
:105B300069835C834B83DB011C92FC0160816623DB
:105B400009F44EC030FF4CC0F9E06F9FB001112442
:105B50006352704ECD010E9481C6D70111968C917F
:105B6000807F41F04B815C816FEC73E089819A8189
:105B70000E9485D2E981FA8101900020E9F73197EE
:105B800029813A81E21BF30B19012E0E3F1E4B8136
:105B90005C814E1B5F0B415051095C834B83D701E5
:105BA0001196EC9111978E2F807F09F4F7C0E29542
:105BB000EF70E150EC3008F0F1C0F0E08827EC51D4
:105BC000F24D8F4F0C9414CEF32D962E032F622F8F
:105BD0007D2F412E132F132F132F2F2E172E992F7A
:105BE00029803A80DCCFF7018481282F30E050E013
:105BF00040E0002359F030E0A4E6B0E00E94DDCDA3
:105C00002FEF30E040E050E00E94ABCD5F934F9328
:105C10003F932F9381ED93E09F938F93FC81FF93AC
:105C20002B812F933F922F920E94BDD2B2C0179624
:105C30008C9117978F9316968C9116978F93159634
:105C40008C9115978F9314968C918F9384ED93E09C
:105C50009F938F93BC81BF93EB81EF93E3CF179614
:105C60008C9117978F9316968C9116978F93159604
:105C70008C9115978F9314968C918F9388ED93E068
:105C8000E7CF1496CD90DD90ED90FC901797F7FE3E
:105C900034C084E6882E912CA12CB12CC701B6010A
:105CA000A50194010E94ABCD9B01AC0188279927E7
:105CB000DC01821B930BA40BB50BBF93AF939F9397
:105CC0008F9366277727CB016C197D098E099F0971
:105CD000A50194010E94ABCD5F934F933F932F9307
:105CE0008CED93E09F938F933C813F934B814F9337
:105CF0003F922F920E94BDD24CC0C701B60124E64C
:105D000030E040E050E00E94ABCD9F938F937F93B3
:105D10006F935F934F933F932F938DED93E09F93FA
:105D20008F939C819F93AB81AF93E2CFC7010E9479
:105D30000913BC01D7011696CC9016971796DC90E4
:105D40001797D0FADD24D0F814969C9114971596E5
:105D5000FC90EB80BC80292F30E050E040E077FDE4
:105D600035C0011135C07F936F931F921F921F9210
:105D70009F931F92FF92DF92CF9286EE93E09F93C4
:105D80008F93FC81FF932B812F933F922F920E9440
:105D9000BDD20FB6F894DEBF0FBECDBF89819A8108
:105DA0000F900F900F900F90DF91CF910F91FF9078
:105DB000EF90DF90CF90BF90AF909F908F907F90AB
:105DC0006F905F904F903F902F900895002361F067
:105DD000292F30E0A4E6B0E00E94DDCD2FEF30E0C7
:105DE00040E050E00E94ABCD5F934F933F932F93E1
:105DF0001F92FF92DF92CF9289EE93E09F938F9351
:105E0000BF92EF9275CF15968C9115971F928F9335
:105E100016969C91169717968C9181708F939F93ED
:105E20008CEE93E015CF14968D909D90AD90BC9024
:105E3000179720E030E0A901C501B4010E943FCCD2
:105E40002401350187FF04C077FA709477F87094C5
:105E5000C301B2010E9411CF6B01072E000C880B09
:105E6000990B0E9446CC9B01AC01C301B2010E9478
:105E700032CE20E030E04AE754E40E94A5CC0E94F4
:105E80009CCF0E9411CF062F772E20E030E0A90191
:105E9000C501B4010E943FCC87FF07C07F920F93DA
:105EA000DF92CF9282EF93E0D3CE7F920F93DF9277
:105EB000CF9283EF93E09F938F933C813F934B81ED
:105EC0004F93B0CE14968C9114971F928F93159682
:105ED0008C9115971F928F9316968C911F928F938A
:105EE00089EE93E09F938F93BC81BF93EB81EF93F7
:105EF0003F922F920E94BDD24CCF17968C9117974C
:105F00001F928F9314968C9114971F928F931596CE
:105F10008C9115971F928F9316968C911F928F9349
:105F200086EE93E09F938F93BC81BF93EB81EF93B9
:105F3000DFCE14966D917C914B815C81C1010E94F2
:105F4000A3D22CCFEF92FF920F93CF93DF93CDB7D5
:105F5000DEB7A0970FB6F894DEBF0FBECDBF7C01B1
:105F600000E020E033E040E250E0BE016F5F7F4F91
:105F70000E94812DBE016F5F7F4F87E799E00E94ED
:105F8000A68163E87BE087E799E00E940C82F70135
:105F9000618162956F7087E799E00E94C7976CE70F
:105FA0007BE087E799E00E940C82F70161816F70C6
:105FB00087E799E00E94C79787E799E00E941581DB
:105FC000A0960FB6F894DEBF0FBECDBFDF91CF9184
:105FD0000F91FF90EF900895AF92BF92CF92EF9202
:105FE000FF920F931F93CF93DF9300D000D01F92A7
:105FF0001F92CDB7DEB75C0109831A832B833C83E4
:106000004D835E836F83788762E776E187E799E067
:106010000E940C82CE0101960E94A22FE114F1048D
:1060200039F06BE676E1C7010E944AC6009721F17C
:10603000F5010281138101151105E1F089818111BA
:1060400059C08A818F70813009F45CC038F1823088
:1060500019F1082F10E06EE476E187E799E00E94DD
:106060000C82B80187E799E00E94CE9787E799E014
:106070000E94158190E080E028960FB6F894DEBF6C
:106080000FBECDBFDF91CF911F910F91FF90EF9089
:10609000CF90BF90AF900895CC20B9F0CE0101967B
:1060A0000E94AE93892B09F444C0C8010E94A01835
:1060B000672B682B692BD9F480E00E943015AB0167
:1060C000BC01C8010E943C1B12C0C8010E94EB1811
:1060D0008E3019F048F4813051F4CE0101960E94BF
:1060E000AE93892B21F0E1CF83518330B0F381E06F
:1060F00090E0C2CF8031C0F48E30B8F68130A9F282
:106100008230B9F06EE576E187E799E00E940C8273
:10611000698187E799E00E94C79787E799E00E9425
:10612000158101E010E097CF8351833008F4BDCF93
:10613000E9CF40E050E0BA01C8010E943C1B60E09A
:10614000C5010E94F818D3CFCF92DF92EF92FF9251
:106150000F931F93CF93DF936115710509F459C015
:106160006A017B018C01CB010E942B13D82F88235D
:1061700079F1D70114968D919C910097F1F1FC0172
:10618000C0852C2F27703EEF320F323010F02111D6
:1061900029C0C695C695C695D0FE59C0C7010E94B4
:1061A000EB18F8018083CC2351F1C295C07F818127
:1061B0008F70C82BC183D7011496ED91FC91818516
:1061C0009285A385B485F80184839583A683B783DC
:1061D0008D2FDF91CF911F910F91FF90EF90DF9066
:1061E000CF900895253049F460E00E949F93009776
:1061F00021F0DC011896CC91CCCFC0E0CDCFD701F7
:106200001496ED91FC9180858770823021F0833067
:1062100081F0D0E0DDCF4185528563857485F8013A
:1062200081818F70806A81834483558366837783FD
:10623000CFCF4185528563857485F80181818F7048
:10624000806781834483558366837783C1CFCC2362
:10625000B1F2C295C07FF801AACF0F931F93CF93DD
:10626000DF9300D000D01F921F92CDB7DEB7198206
:106270001A821B821C821D821E821F8218862A811E
:106280002F702A83FC0102811381C8010E94EB1840
:10629000813041F020F0823011F0853081F490E0BF
:1062A00080E002C081E090E028960FB6F894DEBF4F
:1062B0000FBECDBFDF91CF911F910F91089540E0A8
:1062C00052E0B801CE0101960E94A430CE010196A1
:1062D0000E94AE93E9CFCF93DF9300D000D01F92FE
:1062E0001F92CDB7DEB7FC01862F8F706181607F72
:1062F000682B618388E0DE01119601900D928A95EA
:10630000E1F729813A814B815C816D817E818F81AA
:10631000988528960FB6F894DEBF0FBECDBFDF91EB
:10632000CF910895CF93DF9300D000D01F921F929A
:10633000CDB7DEB7FC01608398E0DE0111960190D5
:106340000D929A95E1F729813A814B815C816D81AB
:106350007E818F81988528960FB6F894DEBF0FBE98
:10636000CDBFDF91CF910895DC011196EC9111978B
:10637000E295EF70E150EB3008F037C0F0E088278D
:10638000EB53FE4C8F4F0C9414CED731D731F531EF
:10639000D031D031E631DD31DD31DD31D031D031B8
:1063A00014966D917D918D919C91179708951496F7
:1063B0006C9170E090E080E0089514966D917D916D
:1063C0008D919C9117970E9411CF089514966D910D
:1063D0007D918D919C91179724E630E040E050E04C
:1063E0000E94ABCDCA01B901089560E070E0CB0115
:1063F00008958F929F92AF92BF92CF92DF92EF92C9
:106400000F931F93CF93DF9300D000D01F921F9262
:10641000CDB7DEB709831A832B833C834D835E831C
:106420006F837887FC012081318121153105A1F42A
:1064300090E080E028960FB6F894DEBF0FBECDBF87
:10644000DF91CF911F910F91EF90DF90CF90BF9090
:10645000AF909F908F9008958C01C9010E94D697AC
:10646000C82ED12CF6E0CF16D10494F40E941F86DA
:10647000009721F0FC012085287F2087BC01F801CE
:10648000808191810E94A697FFEFCF1ADF0AEACFA1
:1064900065E0F801808191810E949F938C01892B96
:1064A00039F28981803120F6CE0101960E94B43103
:1064B000161617061806190624F4F801808585704B
:1064C00089F0F8018085877080876DEF76E087E737
:1064D00099E00E940C8287E799E00E94158181E093
:1064E00090E0A8CF0E94BEA24B015C01CE010196B4
:1064F0000E94B431860E971EA81EB91EF80181862F
:106500009286A386B4868085887F82608087898111
:106510008F7090E0E11090E1892B880F880F880F31
:10652000F80190859770892B808762EF76E087E786
:1065300099E00E940C82CE0101960E94B431AB0119
:10654000BC012AE030E087E799E00E9420816CEEF0
:1065500076E087E799E00E940C82F8014185528538
:10656000638574852AE030E087E799E00E94208106
:10657000B2CFCF92DF92EF920F931F93CF93DF931F
:10658000CDB7DEB7C856D1090FB6F894DEBF0FBE3F
:10659000CDBF6C01A2960FAFA297A3961FAFA39792
:1065A000A4962FAFA497A5963FAFA597A6964FAFF9
:1065B000A697A7965FAFA797A8966FAFA897A9963B
:1065C0007FAFA99798E0FE01EF59FF4FDE01A75A70
:1065D000BF4F01900D929A95E1F7A296EFADA29769
:1065E000E150ED3008F07EC0F0E08827E550FD4C2A
:1065F0008F4F0C9414CE603362336E3370336C3330
:1066000008335E3372337233643366336A3368330C
:1066100067E0CE01875A9F4F0E94923168ED76E085
:1066200087E799E00E940C826A966FAD6A9787E7C8
:1066300099E00E94C7976DEC76E087E799E00E94A9
:106640000C82CE01875A9F4F0E94B431AB01BC012E
:106650002AE030E087E799E00E94208187E799E00F
:106660000E9415816A960FAD6A976B961FAD6B9766
:106670006C962FAD6C976D963FAD6D976E964FAD46
:106680006E976F965FAD6F97A0966FADA097A1962E
:106690007FADA197C6010E94F93181E090E0C85911
:1066A000DF4F0FB6F894DEBF0FBECDBFDF91CF91A5
:1066B0001F910F91EF90DF90CF90089566E0A9CFE2
:1066C00062E0A7CF61E0A5CF6BE0A3CF6AE0A1CFE6
:1066D0006CE09FCF6DE09DCF63E09BCF65E099CFED
:1066E00064E097CF90E080E0DACFCF93DF93EC01C6
:1066F0006115710539F48F8181708F8381E0DF919D
:10670000CF9108958981982F92959F7029F180E00B
:106710009430A8F79B01770F440B550B2959310989
:1067200041095109A4E6B0E00E94CACD2BE531E051
:1067300040E050E00E94ABCD37FF02C030E020E0E7
:106740002536310514F024E630E02F5F220F8F81CB
:106750008170282B2F83D2CF8F7080628983DACF0C
:106760002F923F924F925F926F927F928F929F9261
:10677000AF92BF92CF92DF92EF92FF920F931F934F
:10678000CF93DF93CDB7DEB76A970FB6F894DEBF2D
:106790000FBECDBF1C0109871A872B873C874D8709
:1067A0005E876F87788B22E1E216F10408F035C02E
:1067B000F701EC54FD4F30813D8BCE0109960E94CC
:1067C000091397FD04C0BC01C1010E9475339A856D
:1067D000892F8F70D1011196EC911197E07FE82BF2
:1067E0001196EC93119789858C93E295EF70EC30BC
:1067F00008F063C0F0E08827EF5FFB4C8F4F0C94EC
:1068000014CEF0352A342A348F350F3424365935D6
:10681000983598359835593559351D8ACECF10E0C1
:1068200092959F709D3008F011C4E92FF0E0882701
:10683000E35EFB4C8F4F0C9414CE5D345D367D3699
:106840005D36263626365D365D36263826385D3688
:106850005D36333592959F709D3008F014C1E92F55
:10686000F0E08827E95CFB4C8F4F0C9414CE5D342C
:1068700011350435C73447344434E83413354335CF
:106880004335D234D23433358889F10187838F85FB
:10689000D10116968C9316978E8515968C93159725
:1068A0008D8514968C9314979295907F11968C9168
:1068B00011978F70982B11969C93FD89FF2309F4F3
:1068C00063C0D10111968C9182958F702F2F30E08B
:1068D0008217130609F458C066ED7AE087E799E05D
:1068E0000E940C82F101618162956F7087E799E0E7
:1068F0000E94C79763ED7AE087E799E00E940C82D7
:106900006D8987E799E00E94C79761ED7AE087E794
:1069100099E00E940C82D1010C9119821A821B828B
:106920001C821D821E821F8218868D898295807F1F
:106930009A819F70892B8A830983EE24EA94FE2C26
:1069400011961C91119712962C91129713963C91C7
:10695000139714964C91149715965C91159716966B
:106960006C91169717967C91CE0101960E94B033D8
:10697000F10120833183428353836483758386834B
:106980009783C1010E94A22F88E0F1016FC18F851A
:106990009889F1018683878190FB80F987838E85B2
:1069A00085838BCF8D859E85AF85B889B7FD0EC059
:1069B0008F3F9105A105B10529F024F08FEF90E0FC
:1069C000A0E0B0E0D10114968C9377CF80E0FACFAD
:1069D0006D857E858F85988920E06D39BFEF7B07B7
:1069E0008B079B076CF02FEF6115E4E67E078105AE
:1069F000910534F424E630E040E050E00E94ABCD55
:106A0000D10114962C9359CF8F859889F1018683F3
:106A1000878190FB80F987838E8585838D8584832C
:106A20004CCF8D85CFCFCD84DE84EF84F88820E0F5
:106A300030E0A901C701B6010E943FCC60E087FDAC
:106A40000FC020E030E04FE753E4C701B6010E94D9
:106A500047CF6FEF181624F0C701B6010E9418CF78
:106A6000F10164832ACFD10111968C9111978F7017
:106A7000806C11968C9311978D859E8515969C93AD
:106A80008E9314971ACF63E67BE087E799E00E9424
:106A90000C826A8562956F7087E799E00E94C797BC
:106AA00060E67BE087E799E00E940C82F10161815A
:106AB000C0C092959F70933091F09C30A1F24D85AB
:106AC0005E856F857889F10144835583668377837A
:106AD0009295907F81818F70982B9183EECEC1012A
:106AE0000E94AE93D10114968C9314978F85988948
:106AF00016968C93169717968C91179790FB80F9A2
:106B000017968C9317978E8515968C9315971196DB
:106B10008C9111978F70806211968C93CECECE019E
:106B200009960E94AE93D10114968C931497EFCFDF
:106B300092959F709D3008F066C0E92FF0E088279D
:106B4000EB55FA4C8F4F0C9414CE5D34C035EF35B5
:106B50006F35EF35EF35B235DF35DF35DF35CE3523
:106B6000DA3533358D859E85AF85B889F10184830B
:106B70009583A683B78381818F70806681839DCE44
:106B80006D8570E090E080E00E9444CCD1011496C5
:106B90006D937D938D939C9317978FCE6D857E8596
:106BA0008F8598890E9446CCF10164837583868322
:106BB000978383CE6D857E858F859889E5CF929565
:106BC000907FF10181818F70982B91838D859E85B7
:106BD000AF85B88984839583A683B7836ECE92955B
:106BE000907FD10111968C9111978F70982B1196EF
:106BF0009C938D859E85AF85B889F10184839583AB
:106C0000A683B7835ACE6EE47BE087E799E00E94C3
:106C10000C826A8562956F7087E799E00E94C7973A
:106C20006BE47BE087E799E00E940C82D10111962A
:106C30006C9162956F7087E799E00E94C79787E72C
:106C400099E00E94158139CE11E0EACD4D855E852F
:106C50006F857889F10144835583668377839295A4
:106C6000907F81818F70982B918388E0DE0111964F
:106C700001900D928A95E1F729813A814B815C81DF
:106C80006D817E818F8198856A960FB6F894DEBFFC
:106C90000FBECDBFDF91CF911F910F91FF90EF906D
:106CA000DF90CF90BF90AF909F908F907F906F902C
:106CB0005F904F903F902F900895963009F4C1C097
:106CC00048F46D85913071F06FEF70E0933051F0C2
:106CD00060E008C0973009F4C0C09A506D857E8589
:106CE0009230B0F784E68F8788898E7F888B1E86E6
:106CF0008A858F7080628A876D872E8530E0AFEF3E
:106D0000B0E00E94DDCDC12CD12C7601CA94611572
:106D1000F4E67F078105910544F424E630E040E085
:106D200050E00E94ABCD69017A01112309F475C0CE
:106D3000DA8AC98A2D852E8B022F10E088898695E4
:106D4000A82FA150BB0BB88FAF8B119609F0A4C030
:106D50009601203831050CF087C08FE790E08C1940
:106D60009D09809FD001819FB00D909FB00D11248F
:106D70002FEF30E00E942BCE21E83EE740E050E0CC
:106D80000E94ABCDD10117962C93ABE9B0E0A701DF
:106D900096010E94CACD3FE7432E512C612C712CE5
:106DA000A30192010E94ABCD2C593F4F4F4F5F4F33
:106DB0005901AEEFB1E0A70196010E94CACDA3012F
:106DC00092010E94ABCDD8010E94CACD2FEF30E0D6
:106DD00040E050E00E94ABCD89012F3F310519F012
:106DE00014F00FEF10E06EE37BE087E799E00E947C
:106DF0000C82B50187E799E00E94CE9760E37BE0C3
:106E000087E799E00E940C82B80187E799E00E9429
:106E1000CE9787E799E00E9415816EEF7AE087E7C9
:106E200099E00E940C8287E799E00E94158167EF44
:106E30007AE087E799E00E940C82C1010E94A22FAC
:106E40003CCD6D857E858F85988924E630E040E0D5
:106E500050E00E94ABCDB90145CF6D857E858F8511
:106E600098890E9411CF3ECFA701205831094109CE
:106E70005109ABE9B0E00E94CACD2FE730E040E015
:106E800050E00E94ABCD2C593F4F4F4F5F4F5901FF
:106E9000D10117961C92A7CF2F89388DAAEBBFEF8F
:106EA0000E9423CE24E6822E912CA12CB12CA50188
:106EB00094010E94ABCD29013A01B4E64B0E511C5E
:106EC000611C711C26E430E0AF89B88D0E942BCE86
:106ED000A50194010E94ABCD49015A01EEE18E0E4D
:106EE000911CA11CB11C29893A89203831050CF06C
:106EF00094C08FE790E0821B930B809FD001819F0D
:106F0000B00D909FB00D1124A50194010E94D5CD24
:106F10009B01AC01AFEFB0E00E94CACD24E63AE697
:106F200040E050E00E94ABCDD10117962C93A70111
:106F30009601240D351D461D571DAEEFB1E00E9490
:106F4000CACD23EE30E040E050E00E94ABCD298B6B
:106F50003A8B4B8B5C8BE989FA89FA8FE98FAFEF1B
:106F6000B0E0A70196010E94CACD2FE730E040E0D3
:106F700050E00E94ABCD7901FE89AF2FB0E02989A6
:106F80003A894B895C890E94CACD2FEF30E040E0FE
:106F900050E00E94ABCD89012F3F310519F014F06C
:106FA0000FEF10E06AE27BE087E799E00E940C8235
:106FB0002AE030E0B301A20187E799E00E94208136
:106FC00064E27BE087E799E00E940C822AE030E0EF
:106FD000B501A40187E799E00E9420816CE17BE084
:106FE00087E799E00E940C82B70187E799E00E9449
:106FF000CE9764E17BE087E799E00E940C82B801BC
:1070000087E799E00E94CE976BE07BE087E799E005
:107010000E940C82698D7A8DF8CEA70196012058C6
:10702000310941095109ABE9B0E00E94CACD2FE70F
:1070300030E040E050E00E94ABCD2C593F4F4F4F25
:107040005F4F7901D10117961C92ACCF65EE7AE0C3
:1070500087E799E00E940C826A8562956F7087E7E6
:1070600099E00E94C79762EE7AE01CCDFC01918105
:10707000892F82958F7021F0823029F080E0089569
:107080009F70906291839B0177FF02C030E020E007
:107090002E3681E0380714F02DE631E02683878113
:1070A00030FB80F9878381E008950F931F93CF937E
:1070B000DF938C01FC01C081D1816FE270E0CE01D1
:1070C0000E94B2D20097D9F0FC011192CF010E9428
:1070D0003F17EC0161EC76E087E799E00E940C82B3
:1070E000BE0187E799E00E94CE9787E799E00E946A
:1070F0001581CE01DF91CF911F910F910895CE019F
:107100000E943F17EC01892BA1F3F8011182108234
:10711000F0CF8F929F92AF92BF92CF92DF92EF9279
:10712000FF920F931F93CF93DF93CDB7DEB767978F
:107130000FB6F894DEBF0FBECDBF8C017B014C01B2
:107140008BE0880E911C9F8A8E8AF8011286118628
:107150001386148E138E672B09F463C0A0909906D2
:10716000B0909A06A114B10409F45BC06FE270E01C
:10717000C7010E946AD26C01892B09F44AC0F70149
:10718000DE01119690E080E0BD012191222341F0C3
:107190002F3231F08431910519F02D930196F5CFFE
:1071A000860F971FFC011082C5010E942793F801EA
:1071B00091838083B6016F5F7F4F4FE050E0C40141
:1071C0000E94A3D2CE0146960E945538F801948FB2
:1071D000838F8E899F89892B09F41386C8010E94A9
:1071E0002B13882319F0C8010E949C1B67960FB6C9
:1071F000F894DEBF0FBECDBFDF91CF911F910F91ED
:10720000FF90EF90DF90CF90BF90AF909F908F90C6
:107210000895B701C5010E942793F80191838083E7
:10722000DDCFF80111821082D9CF8F929F92AF9259
:10723000BF92CF92DF92EF92FF920F931F93CF9363
:10724000DF93CDB7DEB7CD55D1090FB6F894DEBFC9
:107250000FBECDBF8C016B016115710519F0411591
:107260005105D1F46FE87CE087E799E00E940C8239
:1072700066E87CE087E799E00E940C82B80187E726
:1072800099E00E94A68164E87CE087E799E00E948B
:107290000C8287E799E030C0460F571FDA011C9235
:1072A0000E94BF264B0162E87CE087E799E00E94DC
:1072B0000C82B40187E799E00E94CE976FE77CE0EB
:1072C00087E799E00E940C82B80187E799E00E9465
:1072D000A6816CE77CE087E799E00E940C82BAE324
:1072E0008B16B1E09B06F4F46FE67CE080ED98E04D
:1072F0000E940C8280ED98E00E941581C35ADF4FF6
:107300000FB6F894DEBF0FBECDBFDF91CF911F91B6
:107310000F91FF90EF90DF90CF90BF90AF909F9034
:107320008F9008956DE67CE087E799E00E940C82DB
:10733000B60187E799E00E94A6816BE67CE087E7CB
:1073400099E00E940C8287E799E00E9415811A82D9
:107350001982FE0133968EE3DF011D928A95E9F7CB
:107360008091970690919806059791F563E070E0FB
:10737000C8010E941E267C01892BE9F5E0914B088B
:10738000F0914C08808180FFB9CF61E070E0C801C6
:107390000E941E26892B09F4B1CF64E270E0C80177
:1073A0000E94B2D2892B09F0A9CF63E57CE087E780
:1073B00099E00E940C82B80187E799E00E94A681BB
:1073C00087E799E00E941581C8010E942A9E96CF06
:1073D00061E070E0C8010E941E267C01892B21F526
:1073E00062E070E0C8010E941E267C0168E47CE037
:1073F000892B09F44ACFE00EF11E6FE37CE0C70150
:107400000E944AC6892BC1F4F60101900020E9F7D9
:107410003197EC19FD09329778F0C8010E942A9E35
:10742000C6010E94E6826ACF4FE350E0B801CE0168
:1074300001960E94A3D2DFCF64E270E0C8010E94EF
:10744000B2D2892B09F05ACFB701CE018F5B9F4F83
:107450000E948938CE018F5B9F4F0E942B13882397
:1074600039F1B601CE018F5B9F4F0E949B98181691
:107470001906F4F489818823D9F0809197069091B8
:1074800098060597A9F067E27CE087E799E00E94FB
:107490000C82BE016F5F7F4F87E799E00E94A68153
:1074A00087E799E00E941581CE0101960E942A9EED
:1074B000CE018F5B9F4F0E94611320CFCF92DF924E
:1074C000EF92FF926A017B0163E0FC018081918170
:1074D0000E949F93FC01892BA9F08085857091F40F
:1074E000C094D094E094F094CC24CA948185928581
:1074F000A385B4858C219D21AE21BF2181879287F0
:10750000A387B487FF90EF90DF90CF900895CF923C
:10751000DF92EF92FF926A017B0163E0FC018081C0
:1075200091810E949F93FC01892BA9F09085892F5E
:10753000857089F4987F92609087CC24FF244185E0
:107540005285638574854C295D296E297F29418781
:10755000528763877487FF90EF90DF90CF900895F4
:10756000CF92DF92FF920F931F93CF93DF938C0103
:10757000EB016A01CB010E942B13F82E882309F43A
:1075800095C0D2FE0AC0D8018C918B3009F451C04D
:1075900008F042C08A3009F451C0D0FE09C0F80199
:1075A000608186EF860F843018F0CE010E94BC18EF
:1075B000D1FE73C0D80114964D915D916D917C916F
:1075C000179711968C9182958F70873038F089309B
:1075D00008F443C08A50823008F471C0CE010E9482
:1075E0003713EC81FD81309709F457C0808587708F
:1075F0009EEF980F923010F081114FC0D801119674
:107600008C9182958F70982F990F990F990F808583
:107610008770892B808741C08C30B9F040E050E002
:1076200062E070E08D3009F0B8CFCE010E94873A59
:10763000B4CF40E050E061E070E0F7CF40E050E0D0
:1076400061E070E0CE010E945E3A40E050E062E00E
:1076500070E0CE010E945E3AA0CFEC81FD813097B0
:10766000E1F0808587709EEF980F923010F08111C5
:1076700014C04187528763877487EC81FD818085C0
:10768000887F83608087EC81FD818085982F987F3B
:1076900087708863903309F4BDCF65E77BE087E7A7
:1076A00099E00E940C82C8010E94A22F8F2DDF91C9
:1076B000CF911F910F91FF90DF90CF900895CE0151
:1076C0000E943713EACFCF92DF92EF92FF926A01C6
:1076D0007B0163E0FC01808191810E949F93009770
:1076E00091F0FC0120852770223069F46185728554
:1076F000838594856C217D218E219F21FF90EF90C1
:10770000DF90CF90089560E070E0CB01F7CFCF928B
:10771000DF92EF92FF920F931F93CF93DF9300D0EE
:1077200000D01F921F92CDB7DEB76C017B0160FFC6
:1077300003C0E894E0F8F4F8F4FC0DC00E94BF2602
:10774000663971058105910530F080919706909119
:107750009806059709F5A70144275770052E000CD8
:10776000660B770BC6010E94873A61EF79E087E7E5
:1077700099E00E940C828FEF9FEF28960FB6F89445
:10778000DEBF0FBECDBFDF91CF911F910F91FF9054
:10779000EF90DF90CF90089519821A821B821C828D
:1077A0001D821E821F8218868A818F708A8340E024
:1077B00053E0B601CE0101960E94A43040E057E0AC
:1077C00060E070E0C6010E94633BE62AF72A098167
:1077D0001A812B813C814D815E816F817885C60144
:1077E0000E94A7A3CACF2F923F924F925F926F92AF
:1077F0007F928F929F92AF92BF92CF92DF92EF9241
:10780000FF920F931F93CF93DF93CDB7DEB7C15C89
:10781000D1090FB6F894DEBF0FBECDBF1C01C7550E
:10782000DF4F0883C95AD040C655DF4F1883CA5A64
:10783000D040C555DF4F2883CB5AD040C455DF4FC9
:107840003883CC5AD040C355DF4F4883CD5AD040FF
:10785000C255DF4F5883CE5AD040C155DF4F6883A1
:10786000CF5AD040C055DF4F7883C05BD040CF5453
:10787000DF4FF982E882C15BD040C954DF4FC88234
:10788000C75BD040C754DF4FA882C95BD0400E947D
:10789000BF266B01C454DF4F79836883CC5BD04033
:1078A000683C7105A4F461E679E080ED98E00E94FF
:1078B0000C82B60180ED98E00E94CE9780ED98E0B2
:1078C0000E94158166246A94762C0C9400470E94CD
:1078D000BEA2C254DF4F688379838A839B83CE5BC9
:1078E000D040C655DF4F8881CA5AD0408F70282FAC
:1078F00030E0CD54DF4F39832883C35BD040809183
:10790000970690919806C654DF4F99838883CA5B87
:10791000D040CF54DF4FE881F981C15BD040309730
:1079200021F0808181110C94B24DD1011B968C9174
:10793000882341F0C1010B96CF54DF4F9983888390
:10794000C15BD040CD54DF4FE881F981C35BD040AB
:10795000EF2B11F00C940E4ECF54DF4FE881F981DC
:10796000C15BD040309711F00C94BB4DD1015B96B8
:107970000D90BC91A02DCD54DF4FB983A883C35B7C
:10798000D040AB2B11F40C940E4EC655DF4F8881BE
:10799000CA5AD0408F7011F00C940E4ECD54DF4F68
:1079A0006881C35BD040CE0187559F4F0E946B31E9
:1079B000C756DF4F2883C959D040C656DF4F38839A
:1079C000CA59D040C556DF4F4883CB59D040C45622
:1079D000DF4F5883CC59D040C356DF4F6883CD5911
:1079E000D040C256DF4F7883CE59D040C156DF4FCA
:1079F0008883CF59D040C056DF4F9883C05AD040BB
:107A00000C940E4ED1018D919C91892B09F45ACF83
:107A1000CD54DF4F08811981C35BD040043011057C
:107A200099F5C754DF4FE880C95BD040C755DF4F99
:107A30000881C95AD040C655DF4F1881CA5AD04074
:107A4000C555DF4F2881CB5AD040C455DF4F388110
:107A5000CC5AD040C355DF4F4881CD5AD040C25593
:107A6000DF4F5881CE5AD040C155DF4F6881CF5A81
:107A7000D040C055DF4F7881C05BD040C1010E942B
:107A8000F9313C010C940047C755DF4F1881C95AA2
:107A9000D040143009F4DAC248F4112309F435C097
:107AA000912C812C66246A94762C54C388EF810F24
:107AB0008230B0F788E0FE01E755FF4FDE011196F6
:107AC00001900D928A95E1F7C655DF4FE881CA5AB9
:107AD000D0408E2F807F09F46DC3E295EF70E150A6
:107AE000EB3008F067C3F0E08827E658F24C8F4F80
:107AF0000C9414CEC840C840DA40B940B9402F4178
:107B00001E411E411E41B940B94019821A821B8292
:107B10001C821D821E821F8218868A818F708A8332
:107B2000C655DF4F8881CA5AD040807F09F4B8CF4C
:107B3000CD54DF4F28813981C35BD0402A303105D5
:107B400009F43CC254F42115310569F122303105A4
:107B500009F4DEC0912C812C28C2CD54DF4F8881DE
:107B60009981C35BD0408B30910509F4CFC10C974C
:107B700089F7B101CE0101960E940898CE01875580
:107B80009F4F0E940913BC01CE0101960E947533DC
:107B900088E0FE013196DE01A755BF4F01900D929E
:107BA0008A95E1F7FFC1EF2B59F06EE179E087E7A5
:107BB00099E00E940C8287E799E00E941581CACF64
:107BC000C1010E940F578C0161E070E01816190680
:107BD00014F070E060E087E799E00E94CE976FECC8
:107BE00073E087E799E00E94A681CE0187559F4FF9
:107BF0000E94B431AB01BC012AE030E087E799E094
:107C00000E94208187E799E00E941581CE01875567
:107C10009F4F1016110614F00C94A04D0E94B43121
:107C2000672B682B692B09F068C162E0CE0187558C
:107C30009F4F0E949231CF56DF4F2883C159D040C9
:107C4000CE56DF4F3883C259D040CD56DF4F4883E0
:107C5000C359D040CC56DF4F5883C459D040CB567F
:107C6000DF4F6883C559D040CA56DF4F7883C65965
:107C7000D040C956DF4F8883C759D040C856DF4F20
:107C80009883C859D04088248394982C91E0C85494
:107C9000DF4F9883C85BD040DD24D39442C061E0BD
:107CA000CE0187559F4F0E949231C757DF4F2883DF
:107CB000C958D040C657DF4F3883CA58D040C5573F
:107CC000DF4F4883CB58D040C457DF4F5883CC5840
:107CD000D040C357DF4F6883CD58D040C257DF4FE5
:107CE0007883CE58D040C157DF4F8883CF58D040DB
:107CF000C057DF4F9883C059D04088248394982C74
:107D0000A1E0C854DF4FA883C85BD040D12C09C084
:107D1000912C812CC854DF4F1882C85BD040DD24E1
:107D2000DA94B101CE0101960E9408988A81982FB9
:107D300092959F70945F9F70923060F4C655DF4FAC
:107D40009881CA5AD04092959F70923019F48F70E2
:107D500080628A83F1019085973071F4C655DF4FB8
:107D60008881CA5AD040807E803211F0803421F45C
:107D70008A818F7080628A83F101A185B285892F03
:107D800090E0109741F0ED91FC911197048CF58DE6
:107D9000E02DCD0119957C01C755DF4F0881C95AE7
:107DA000D040C655DF4F1881CA5AD040C555DF4F65
:107DB0002881CB5AD040C455DF4F3881CC5AD040AF
:107DC000C355DF4F4881CD5AD040C255DF4F58814F
:107DD000CE5AD040C155DF4F6881CF5AD040C055F0
:107DE000DF4F7881C05BD040CE0101960E94B03356
:107DF000CF57DF4F2883C158D040CE57DF4F38834D
:107E0000C258D040CD57DF4F4883C358D040CC57DD
:107E1000DF4F5883C458D040CB57DF4F6883C558D5
:107E2000D040CA57DF4F7883C658D040C957DF4F7C
:107E30008883C758D040C857DF4F9883C858D04070
:107E4000CE0101960E94A22FC854DF4FF881C85B73
:107E5000D040FF2351F1C655DF4F8881CA5AD04028
:107E600082958F709FE0980F9F70923020F08A5F0C
:107E70008F708230D0F48A8182958F7081508230E9
:107E8000A0F42D8130E0AFEFB0E00E94DDCD2FEF08
:107E9000611504E670078105910534F424E630E0AD
:107EA00040E050E00E94ABCD2D8388E0FE0131968A
:107EB000DE01A755BF4F01900D928A95E1F712E1BF
:107EC000912AC12C66246A94762CD10118968C9143
:107ED0001897873009F0E1C6C454DF4FE881F98173
:107EE000CC5BD040EE35F1400CF008C46AED78E090
:107EF00080ED98E00E940C82E1CC912C812CB1E0C5
:107F0000C854DF4FB883C85BD040C6CEB101CE01A4
:107F100001960E940898C255DF4F8881CE5AD04002
:107F20009A8192959F7039F0923049F0912C812C72
:107F3000CC24C3943BC09A819F7090629A8390E056
:107F40008536910514F084E690E08E8388E0FE018A
:107F50003196DE01A755BF4F01900D928A95E1F74A
:107F600062E0CE0187559F4F0E946B31EA962FAF9A
:107F7000EA97EB963FAFEB97EC964FAFEC97ED9609
:107F80005FAFED97EE966FAFEE97EF967FAFEF97FF
:107F9000C158DF4F8883CF57D040C058DF4F9883F8
:107FA000C058D040812C42E1942EC12CC854DF4FE0
:107FB0001882C85BD040DD24DA9484CFB101CE01B1
:107FC00001960E940898C155DF4F6881CF5AD04072
:107FD000C055DF4F7881C05BD0407170CE010196F3
:107FE0000E943638C854DF4F8883C85BD040912C3C
:107FF000812CCC24C3948823F1F288E0FE013196D1
:10800000DE01A755BF4F01900D928A95E1F762E01E
:10801000CE0187559F4F0E946B31E2962FAFE297BA
:10802000E3963FAFE397E4964FAFE497E5965FAFF3
:10803000E597E6966FAFE697E7967FAFE797E89606
:108040008FAFE897E9969FAFE997ACCFCD54DF4F5C
:1080500028813981C35BD0402930310509F461C0E2
:10806000C1010E940F571816190674F562E0CE017F
:1080700087559F4F0E949231AA962FAFAA97AB9631
:108080003FAFAB97AC964FAFAC97AD965FAFAD97A8
:10809000AE966FAFAE97AF967FAFAF97E0968FAFCC
:1080A000E097E1969FAFE19788248394982C66240B
:1080B0006A94762CC12C31E0C854DF4F3883C85BFA
:1080C000D040DD24D39401CF61E0CE0187559F4F8E
:1080D0000E949231A2962FAFA297A3963FAFA3978B
:1080E000A4964FAFA497A5965FAFA597A6966FAF3E
:1080F000A697A7967FAFA797A8968FAFA897A996A0
:108100009FAFA99788248394982C66246A94762C30
:10811000C12C81E0C854DF4F8883C85BD040D12C8C
:10812000D4CE40E050E061E070E0C1010E94633BCA
:10813000672B682B692BA9F040E050E061E070E00C
:10814000C1010E945E3A88248394B4E09B2E662489
:108150006394712CC12CC854DF4F1882C85BD04087
:1081600055C140E050E061E070E0C1010E94873AF3
:10817000EACFC355DF4F288139814A815B81CD5ACF
:10818000D040A4E6B0E00E94CACD6B017C010DC0D6
:10819000C355DF4FC880CD5AD04094E6C99E6001D8
:1081A00011240D2C000CEE08FF08C114D104E104C9
:1081B000F10429F4A5E0CA2ED12CE12CF12C1930C0
:1081C00041F4F094E094D094C094C11CD11CE11C03
:1081D000F11CB101CE0187559F4F0E94089860E0C5
:1081E000CE0187559F4F0E9492316A962FAF6A97B2
:1081F0006B963FAF6B976C964FAF6C976D965FAF7A
:108200006D976E966FAF6E976F967FAF6F97A096D4
:108210008FAFA097A1969FAFA197CD54DF4FA881B4
:10822000B981C35BD040A230B10509F474C004F534
:10823000AB2B09F4AEC0912C812C33C220E030E08E
:1082400048EC52E4C355DF4F688179818A819B8174
:10825000CD5AD0400E94A5CC0E9411CF96CFC355D5
:10826000DF4FC880D980EA80FB80CD5AD0409DCFB7
:10827000CD54DF4FE881F981C35BD040EA30F1058E
:1082800009F4B2C13B97B9F6C655DF4F8881CA5A87
:10829000D04082958F70823009F023C2C701B601A9
:1082A00024E630E040E050E00E94ABCDC255DF4F05
:1082B0008881CE5AD04090E0280F391F37FF02C086
:1082C00030E020E02536310514F024E630E0C255D8
:1082D000DF4F2883CE5AD04062E0CE0187559F4FB2
:1082E0000E946B312A962FAF2A972B963FAF2B9780
:1082F0002C964FAF2C972D965FAF2D972E966FAF84
:108300002E972F967FAF2F9760968FAF60976196CD
:108310009FAF6197C3C1C854DF4F1882C85BD0407C
:10832000D10119968D919C911A97009709F038C048
:1083300018968C9190E0E0E58E2E912CA12CB12C1A
:108340008530910549F0812C912C5401449721F0FE
:10835000812C912C54018A94C655DF4FE881CA5A6A
:10836000D040E295EF70E150EB3008F02EC1F0E024
:108370008827E254FE4B8F4F0C9414CED841D8413D
:10838000E542E542E542B24278427842784209420B
:108390000942F1E0C854DF4FF883C85BD040C0CF3A
:1083A000DC01ED91FC91048CF58DE02D1995C3CF86
:1083B000C355DF4F1881CD5AD040C701B60124E61E
:1083C00030E040E050E00E94ABCDDA01C901810FFE
:1083D000911DA11DB11DB7FF03C080E090E0DC013D
:1083E0008F3F9105A105B10529F024F08FEF90E0B2
:1083F000A0E0B0E0C355DF4F8883CD5AD040812C38
:1084000072E1972EC12C66246A94762CDD24DA94CE
:108410005CCDC355DF4F488059806A807B80CD5A40
:10842000D040B4E6CB16D104E104F104DCF5A4E6B7
:10843000B0E0A30192010E94CACDC60ED71EE81E6D
:10844000F91E81149104A104B104B9F0A5019401AD
:108450000E94CACD362F272FB701A60177FF03C090
:1084600040E050E0BA01C32ED22E7C014C155D05D0
:108470006E057F0514F46A017B01C355DF4FC88286
:10848000D982EA82FB82CD5AD040C655DF4F88811F
:10849000CA5AD0408F708066C655DF4F8883CA5A4B
:1084A000D040ADCFC701B60124E630E040E050E057
:1084B0000E94ABCD420E531E641E751E81149104A2
:1084C000A104B10461F077FE03C0412C512C3201AC
:1084D00084149504A604B70414F424013501C3558B
:1084E000DF4F488259826A827B82CD5AD04087CF43
:1084F000C355DF4F688179818A819B81CD5AD040F5
:108500000E9411CF2B013C01C701B60124E630E0E7
:1085100040E050E00E94ABCDCA01B901640D751D69
:10852000861D971D81149104A104B10481F02B01D3
:108530003C0177FE03C0412C512C3201C301B20132
:1085400086169706A806B90614F4C501B4010E9460
:1085500046CCC355DF4F688379838A839B83CD5A8A
:10856000D0404DCFC355DF4F88819981AA81BB810F
:10857000CD5AD040C80ED91EEA1EFB1E81149104AC
:10858000A104B104C9F0A4E6B0E0A50194010E94E1
:10859000CACD362F272FB701A60177FF03C040E0D1
:1085A00050E0BA01C32ED22E7C014C155D056E053C
:1085B0007F0514F46A017B01C355DF4FC882D9825D
:1085C000EA82FB82CD5AD0401ACF88E0FE01319674
:1085D000DE01A755BF4F01900D928A95E1F7912CCE
:1085E000812CCC24C3940FCFC655DF4F8881CA5A43
:1085F000D04082958F70823009F055C0C701B60116
:1086000024E630E040E050E00E94ABCDC155DF4FA2
:108610008881CF5AD040C055DF4F6881C05BD040C1
:10862000962F9170280F391F2E36E1E03E072CF46B
:1086300037FF05C02DE631E002C030E020E0C15533
:10864000DF4F2883CF5AD040C055DF4F8881C05BB1
:10865000D04030FB80F9C055DF4F8883C05BD040ED
:1086600062E0CE0187559F4F0E946B3162962FAF1B
:10867000629763963FAF639764964FAF6497659632
:108680005FAF659766966FAF669767967FAF6797A0
:1086900068968FAF689769969FAF6997812C62E162
:1086A000962EC12C18C088E0FE013196DE01A75538
:1086B000BF4F01900D928A95E1F762E179E080ED7C
:1086C00098E00E940C8280ED98E00E941581912C28
:1086D000812CCC24C394C854DF4F1882C85BD0408F
:1086E00092CE88E0FE013196DE01A755BF4F019082
:1086F0000D928A95E1F766E079E0E1CFC954DF4F4A
:108700001881C75BD040112361F11296ED91FC9165
:1087100080858770853029F5C654DF4FE881F9815F
:10872000CA5BD0403597E9F0C1010E940F57DD24A4
:10873000D394181619060CF0D12CCF54DF4F488172
:108740005981C15BD040C754DF4F2881C95BD040FD
:10875000BE0167557F4FD10112968D919C910E9469
:108760004856C755DF4F8881C95AD040853009F433
:1087700012C228F4833009F477C0C401FCC08630EB
:1087800009F40CC18730C9F7C1010E94EB18182FFA
:10879000863009F0F2C0CD54DF4F08811981C35BE8
:1087A000D0400130110509F03EC0C655DF4F888129
:1087B000CA5AD040807FB9F1D11005C0C1010E94D2
:1087C0008B18892B81F1C754DF4FE880C95BD040FB
:1087D000C755DF4F0881C95AD040C655DF4F1881B1
:1087E000CA5AD040C555DF4F2881CB5AD040C45516
:1087F000DF4F3881CC5AD040C355DF4F4881CD5A26
:10880000D040C255DF4F5881CE5AD040C155DF4FBE
:108810006881CF5AD040C055DF4F7881C05BD040CF
:10882000C1010E94B9326EEA78E087E799E00E94C0
:108830000C8266E070E087E799E00E94CE9787E7B8
:1088400099E00E94158162E0CE0187559F4F0E94FA
:10885000923129AF3AAF4BAF5CAF6DAF7EAF8FAF08
:1088600021969FAF219784C0C1010E94EB188530EB
:1088700021F093E0692E712CC3C2CD54DF4FE88103
:10888000F981C35BD040319709F03EC0C655DF4F38
:108890008881CA5AD040807FB9F1DD2029F0C1011A
:1088A0000E948B18892B81F1C754DF4FE880C95B88
:1088B000D040C755DF4F0881C95AD040C655DF4F59
:1088C0001881CA5AD040C555DF4F2881CB5AD040B5
:1088D000C455DF4F3881CC5AD040C355DF4F488153
:1088E000CD5AD040C255DF4F5881CE5AD040C155E5
:1088F000DF4F6881CF5AD040C055DF4F7881C05BD1
:10890000D040C1010E94B93265EC78E087E799E078
:108910000E940C8265E070E087E799E00E94CE97A4
:1089200087E799E00E941581B101CE0187559F4FDD
:108930000E94089861E0CE0187559F4F0E949231B6
:1089400022962FAF229723963FAF239724964FAFBF
:10895000249725965FAF259726966FAF2697279683
:108960007FAF279728968FAF289729969FAF299793
:10897000C40181609160B12C8DC060E978E087E727
:1089800099E00E940C82612F70E087E799E00E94D5
:10899000CE9787E799E00E9415816BCF40E050E0C9
:1089A00061E070E0C1010E94633B672B682B692B7B
:1089B00009F0EEC01FEFD11209C0C1010E940F578C
:1089C000DD24D394181619060CF0D12CCD54DF4FAA
:1089D00028813981C35BD0402130310509F03FC087
:1089E000C655DF4F8881CA5AD040807FC1F1DD2053
:1089F00031F0C1010E948B18892B09F4C2C0C75401
:108A0000DF4FE880C95BD040C755DF4F0881C95AA6
:108A1000D040C655DF4F1881CA5AD040C555DF4FE8
:108A20002881CB5AD040C455DF4F3881CC5AD04032
:108A3000C355DF4F4881CD5AD040C255DF4F5881D2
:108A4000CE5AD040C155DF4F6881CF5AD040C05573
:108A5000DF4F7881C05BD040C1010E94B932D11094
:108A600090C0B101CE0187559F4F0E94089861E0E8
:108A7000CE0187559F4F0E94923129AB3AAB4BAB49
:108A80005CAB6DAB7EAB8FAB98AFC4018160916086
:108A900036E0B32E4C01689480F8C655DF4F28812C
:108AA000CA5AD040322F3F70323058F4C755DF4F8A
:108AB0003881C95AD040332321F04C01689480F8A2
:108AC00090F8207F09F4D4C0689491F8C854DF4F1F
:108AD0009881C85BD040C954DF4F9883C75BD040B2
:108AE00066246394712CC1100C945C4ED1011996CC
:108AF0008D919C91009709F071C640E050E062E0D2
:108B000070E0C1010E94633B672B682B692B09F45D
:108B100097C662E377E080ED98E00E940C8280EDDA
:108B200098E00E94158192FE02C00C948A4D67E184
:108B300077E087E799E00E940C82B30187E799E02C
:108B40000E94CE9760E177E087E799E00E940C826F
:108B50000E94BEA2AB01BC01C254DF4F0881198143
:108B60002A813B81CE5BD040401B510B620B730BC3
:108B700087E799E00E94C49787E799E00E941581F2
:108B80003FC166E778E087E799E00E940C8271CEEA
:108B900061E678E0F8CF3FEFD31209C0C1010E942F
:108BA0000F57DD24D394181619060CF0D12CCD5490
:108BB000DF4F88819981C35BD040019709F03FC0A6
:108BC000C655DF4F8881CA5AD040807FC1F1D1108D
:108BD00006C0C1010E948B18892B09F446C0C754F6
:108BE000DF4FE880C95BD040C755DF4F0881C95AC5
:108BF000D040C655DF4F1881CA5AD040C555DF4F07
:108C00002881CB5AD040C455DF4F3881CC5AD04050
:108C1000C355DF4F4881CD5AD040C255DF4F5881F0
:108C2000CE5AD040C155DF4F6881CF5AD040C05591
:108C3000DF4F7881C05BD040C1010E94B932DD2096
:108C4000A1F062E0CE0187559F4F0E94923129A783
:108C50003AA74BA75CA76DA77EA78FA798ABC401C7
:108C60008160916025E0B22E15CF64E478E08BCF6F
:108C700040E052E0B101CE0187559F4F0E94A430E1
:108C8000811122CFC854DF4FA881C85BD040C9549E
:108C9000DF4FA883C75BD04023CFBFEFDB12CBC031
:108CA000C1010E940F57DD24D394181619060CF445
:108CB000C5C0D12C66E378E087E799E00E940C827A
:108CC0004D2C0D2C000C5508B20187E799E00E944D
:108CD000CE976FE278E087E799E00E940C82C85453
:108CE000DF4FF881C85BD0406F2F70E087E799E0D5
:108CF0000E94CE9787E799E00E941581CF54DF4FFD
:108D0000E880F980C15BD040E114F10409F4A3C00C
:108D100065E971E2C7010E944AC601E010E0892BB3
:108D200009F44BC061E971E2C7010E944AC602E042
:108D300010E0892B09F441C06BE077E0C7010E9485
:108D40004AC605E010E0892BC1F167E077E0C70172
:108D50000E944AC606E010E0892B79F166E571E2CF
:108D6000C7010E944AC603E110E0892B31F161E599
:108D700071E2C7010E944AC604E110E0892BE9F0C4
:108D80006BE571E2C7010E944AC60EE010E0892B34
:108D9000A1F064E471E2C7010E944AC60FE010E04E
:108DA000892B59F06DE471E2C7010E944AC610E0B8
:108DB00000E0892B11F405E110E0C1010E94EB18DD
:108DC000A82EB12CA114B10409F45201011511050A
:108DD00009F466C0A016B106C1F163E178E087E747
:108DE00099E00E940C82B50187E799E00E94CE9736
:108DF00087E799E00E9415811DEF612E77247A9410
:108E0000C301CF53DF4F0FB6F894DEBF0FBECDBF07
:108E1000DF91CF911F910F91FF90EF90DF90CF9056
:108E2000BF90AF909F908F907F906F905F904F908A
:108E30003F902F900895DD2009F43CCFE1E0C85425
:108E4000DF4FE883C85BD04035CFCF54DF4F198266
:108E50001882C15BD040C755DF4FE881C95AD04066
:108E6000E63108F07AC4F0E08827E65CF84B8F4FD3
:108E70000C9414CEBB4B0E4AAE499247BB4B3F49B4
:108E8000B3482A48BB4BBB4BA74ACA4A204B514B5D
:108E9000814A814AAD4BAD4BAD4B814A814A814AF3
:108EA000D10119968D919C91009709F4D4CFDC01E2
:108EB000ED91FC910488F589E02DC754DF4FA8801F
:108EC000C95BD040C854DF4FC880C85BD040C7558D
:108ED000DF4F0881C95AD040C655DF4F1881CA5AA2
:108EE000D040C555DF4F2881CB5AD040C455DF4F05
:108EF0003881CC5AD040C355DF4F4881CD5AD0403D
:108F0000C255DF4F5881CE5AD040C155DF4F6881DE
:108F1000CF5AD040C055DF4F7881C05BD040199503
:108F20000C94413DC1010E94EB18853009F0A1CCA1
:108F3000CD54DF4FE881F981C35BD040319709F010
:108F400046C0C954DF4FF881C75BD040FF2309F406
:108F50003EC0C655DF4F8881CA5AD040807FB9F1E4
:108F6000D11005C0C1010E948B18892B81F1C75413
:108F7000DF4FE880C95BD040C755DF4F0881C95A31
:108F8000D040C655DF4F1881CA5AD040C555DF4F73
:108F90002881CB5AD040C455DF4F3881CC5AD040BD
:108FA000C355DF4F4881CD5AD040C255DF4F58815D
:108FB000CE5AD040C155DF4F6881CF5AD040C055FE
:108FC000DF4F7881C05BD040C1010E94B9326EEFA3
:108FD00077E087E799E00E940C8265E070E087E720
:108FE00099E00E94CE9787E799E00E941581B10130
:108FF000CE0187559F4F0E940898D10118968C91F9
:109000008530C9F46EE0CE0187559F4F0E949231A2
:1090100029A33AA34BA35CA36DA37EA38FA398A718
:10902000689480F890F8B12CB1E0C954DF4FB88350
:10903000C75BD04058CD61E0CE0187559F4F0E945D
:109040009231298F3A8F4B8F5C8F6D8F7E8F8F8FF0
:1090500098A3E6CFC1010E94EB18182F863009F0C3
:109060007FC0CD54DF4FE881F981C35BD040319799
:1090700009F046C0C954DF4FF881C75BD040FF23D9
:1090800009F43EC0C655DF4F8881CA5AD040807F60
:10909000B9F1D11005C0C1010E948B18892B81F153
:1090A000C754DF4FE880C95BD040C755DF4F088108
:1090B000C95AD040C655DF4F1881CA5AD040C5554D
:1090C000DF4F2881CB5AD040C455DF4F3881CC5A6E
:1090D000D040C355DF4F4881CD5AD040C255DF4FF5
:1090E0005881CE5AD040C155DF4F6881CF5AD04009
:1090F000C055DF4F7881C05BD040C1010E94B932BA
:1091000067EE77E087E799E00E940C8266E070E006
:1091100087E799E00E94CE9787E799E00E94158142
:1091200062E0CE0187559F4F0E949231298B3A8B86
:109130004B8B5C8B6D8B7E8B8F8B988F40E050E0E0
:1091400068E070E0C1010E945E3A689480F890F88F
:10915000B12C01E0C954DF4F0883C75BD040C3CCBA
:1091600069EC77E00CCC40E050E061E070E0C101D8
:109170000E94633B672B682B692B09F07DC0CD549F
:10918000DF4F28813981C35BD0402130310509F0A0
:1091900047C0C954DF4F3881C75BD040332309F43F
:1091A0003FC0C655DF4F8881CA5AD040807FC1F189
:1091B000DD2031F0C1010E948B18892B09F459C0C0
:1091C000C754DF4FE880C95BD040C755DF4F0881E7
:1091D000C95AD040C655DF4F1881CA5AD040C5552C
:1091E000DF4F2881CB5AD040C455DF4F3881CC5A4D
:1091F000D040C355DF4F4881CD5AD040C255DF4FD4
:109200005881CE5AD040C155DF4F6881CF5AD040E7
:10921000C055DF4F7881C05BD040C1010E94B93298
:10922000D11027C0B101CE0187559F4F0E940898E9
:1092300061E0CE0187559F4F0E94923129873A877E
:109240004B875C876D877E878F87988B40E050E0E7
:1092500068E070E0C1010E94873A689480F890F855
:10926000B6E0BB2E81E0C954DF4F8883C75BD04096
:109270003ACC6FEA77E087CC6AE977E084CCCD54CA
:10928000DF4FA881B981C35BD040119709F047C077
:10929000C954DF4FB881C75BD040BB2309F43FC03E
:1092A000C655DF4F8881CA5AD040807FC1F1D110A6
:1092B00006C0C1010E948B18892B09F44CC0C75409
:1092C000DF4FE880C95BD040C755DF4F0881C95ADE
:1092D000D040C655DF4F1881CA5AD040C555DF4F20
:1092E0002881CB5AD040C455DF4F3881CC5AD0406A
:1092F000C355DF4F4881CD5AD040C255DF4F58810A
:10930000CE5AD040C155DF4F6881CF5AD040C055AA
:10931000DF4F7881C05BD040C1010E94B932DD20AF
:10932000D1F062E0CE0187559F4F0E949231298390
:109330003A834B835C836D837E838F8398876894A5
:1093400080F890F8A5E0BA2EE1E0C954DF4FE88339
:10935000C75BD040C8CB6DE777E015CCC655DF4F73
:109360001881CA5AD040812F8F70B12C823008F0FA
:1093700027C2C1010E94EB18853009F47ACACD5486
:10938000DF4F28813981C35BD0402130310509F09E
:1093900040C0C954DF4F3881C75BD0403323C9F187
:1093A000107FB9F1D11005C0C1010E948B18892B23
:1093B00081F1C754DF4FE880C95BD040C755DF4F0C
:1093C0000881C95AD040C655DF4F1881CA5AD040CB
:1093D000C555DF4F2881CB5AD040C455DF4F388167
:1093E000CC5AD040C355DF4F4881CD5AD040C255EA
:1093F000DF4F5881CE5AD040C155DF4F6881CF5AD8
:10940000D040C055DF4F7881C05BD040C1010E9481
:10941000B932689480F890F8B12C24CFCD54DF4F46
:10942000A881B981C35BD040119709F046C0C954E7
:10943000DF4FB881C75BD040BB2309F43EC0C6559F
:10944000DF4F8881CA5AD040807FB9F1DD2029F0F2
:10945000C1010E948B18892B81F1C754DF4FE8802E
:10946000C95BD040C755DF4F0881C95AD040C655A7
:10947000DF4F1881CA5AD040C555DF4F2881CB5ADB
:10948000D040C455DF4F3881CC5AD040C355DF4F50
:109490004881CD5AD040C255DF4F5881CE5AD04076
:1094A000C155DF4F6881CF5AD040C055DF4F78811A
:1094B000C05BD040C1010E94B932C655DF4F8881E0
:1094C000CA5AD0408F70B12C823008F080C1C75585
:1094D000DF4FB880C95AD040BB2009F4C3CEDD208D
:1094E00081F064E677E087E799E00E940C8261E012
:1094F000C1010E94BC1860E071E1C1010E94873B7C
:10950000B8C9C655DF4F8881CA5AD040982F9F707E
:10951000923008F03BC1C755DF4FB880C95AD040E0
:10952000BB2009F43BC1807F31F4B101CE018755E6
:109530009F4F0E940898689480F8E3E09E2AB12C1F
:10954000F1E0C954DF4FF883C75BD040CCCA6894C0
:1095500092F8C954DF4F0881C75BD040002309F45B
:1095600062CDC655DF4F8881CA5AD040807F81F0D6
:1095700040E050E061E070E0C1010E94633B672B76
:10958000682B692B61F5C1010E948B18892B39F575
:10959000B12CA9CA689492F8CD54DF4F2881398143
:1095A000C35BD0402130310509F0E0C0C954DF4F22
:1095B0003881C75BD040332311F2C655DF4F888115
:1095C000CA5AD040807F21F340E050E061E070E073
:1095D000C1010E94633B672B682B692BA1F6C7541E
:1095E000DF4FE880C95BD040C755DF4F0881C95ABB
:1095F000D040C655DF4F1881CA5AD040C555DF4FFD
:109600002881CB5AD040C455DF4F3881CC5AD04046
:10961000C355DF4F4881CD5AD040C255DF4F5881E6
:10962000CE5AD040C155DF4F6881CF5AD040C05587
:10963000DF4F7881C05BD040C1010E94B932A8CF12
:10964000CD54DF4F88819981C35BD040B12C812CF0
:10965000F4E09F2E019709F07CCDC954DF4F98812B
:10966000C75BD040992309F4A0C0C655DF4F88815D
:10967000CA5AD040807F81F040E050E062E070E064
:10968000C1010E94633B672B682B692BA9F5C101BF
:109690000E948B18892B81F5B12C812C54E0952EDA
:1096A00022CACD54DF4FA881B981C35BD040B12C11
:1096B000812C74E0972E119709F082C0C954DF4FB6
:1096C000B881C75BD040B12C812C64E0962EBB23BF
:1096D00009F47DC0C655DF4F8881CA5AD040807FCB
:1096E000D9F240E050E062E070E0C1010E94633BCB
:1096F000672B682B692B59F6C754DF4FE880C95B8D
:10970000D040C755DF4F0881C95AD040C655DF4FFA
:109710001881CA5AD040C555DF4F2881CB5AD04056
:10972000C455DF4F3881CC5AD040C355DF4F4881F4
:10973000CD5AD040C255DF4F5881CE5AD040C15586
:10974000DF4F6881CF5AD040C055DF4F7881C05B72
:10975000D040C1010E94B9329FCFC655DF4F8881EA
:10976000CA5AD040807F21F4689490F8B12CECCD97
:10977000F3E09F2AEDCCC854DF4F1881C85BD0407E
:10978000C954DF4F1883C75BD04002CFB12C91E0A2
:10979000C954DF4F9883C75BD040A5C9A1E0C95425
:1097A000DF4FA883C75BD0409EC9B12C812CE4E079
:1097B0009E2E11E0C954DF4F1883C75BD04093C978
:1097C00021E0C954DF4F2883C75BD0408CC931E00A
:1097D000C954DF4F3883C75BD04085C9DC01ED91A8
:1097E000FC91008CF18DE02DC755DF4F0881C95ADF
:1097F000D040C655DF4F1881CA5AD040C555DF4FFB
:109800002881CB5AD040C455DF4F3881CC5AD04044
:10981000C355DF4F4881CD5AD040C255DF4F5881E4
:10982000CE5AD040C155DF4F6881CF5AD040C05585
:10983000DF4F7881C05BD040199581115EC969C93D
:10984000F10181859285892B09F472C081149104FC
:1098500039F0A401B101CE0187559F4F0E94B03A63
:10986000D10119968D919C91CF54DF4FE880F980FA
:10987000C15BD040DC01ED91FC910488F589E02DBD
:10988000C754DF4FA880C95BD040C954DF4FC880A0
:10989000C75BD040C755DF4F0881C95AD040C65575
:1098A000DF4F1881CA5AD040C555DF4F2881CB5AA7
:1098B000D040C455DF4F3881CC5AD040C355DF4F1C
:1098C0004881CD5AD040C255DF4F5881CE5AD04042
:1098D000C155DF4F6881CF5AD040C055DF4F7881E6
:1098E000C05BD04019953C01F10181859285DC0176
:1098F000ED91FC91048CF58DE02D1995059711F4EF
:10990000689480F892FCFEC0BB2021F06B2DC10151
:109910000E94BC18C654DF4FE881F981CA5BD04071
:10992000B401359709F403C9C1010E94873BFFC800
:109930008085853009F474C0863031F7C755DF4F14
:10994000D880C95AD040DD2009F46AC0C1010E9404
:10995000E6978C018114910439F0A401B101CE0184
:1099600087559F4F0E94B03A0115110569F2F12CFD
:10997000E12C17FF06C0119501951109EE24E3941F
:10998000F12CC80101978634910508F0BDCFC02E97
:1099900061E0802F0E94089FEFEFED0DE53110F59B
:1099A000F0E08827E952F34B8F4F0C9414CEEC4C27
:1099B000EE4CF24CF24CEE4CEC4CEE4CF24CF24CC9
:1099C000F24CF24CF24CF24CEC4CEC4CF24CF24CB3
:1099D000F24CF24CEC4CEC4CF1E0EF266E2D8C2D61
:1099E0000E94DA9E6DE277E087E799E00E940C82A0
:1099F000B80187E799E00E94CE976BE277E087E7AE
:109A000099E00E940C82B70187E799E00E94CE9707
:109A100087E799E00E941581689480F890F872C0F9
:109A20008114910439F0A401B101CE0187559F4FF3
:109A30000E94B03ACD54DF4F08811981C35BD040FA
:109A40000230110509F462C00330110529F001301C
:109A5000110509F059CFE0CFC1010E94A018892B50
:109A600049F4D101ED91FC91608171818BEF93E01C
:109A70000E948CA6CE0187559F4F0E94C21220E003
:109A800030E048EC52E40E94A5CC0E9411CFCD54A6
:109A9000DF4F688379838A839B83C35BD040CD5437
:109AA000DF4FC880D980C35BD04088E00E9430156A
:109AB0002B013C0167E277E087E799E00E940C8286
:109AC000CD54DF4F68817981C35BD04087E799E04F
:109AD0000E94CE9762E277E087E799E00E940C82CD
:109AE000B301A201662777272AE087E799E00E9461
:109AF000C98087E799E00E941581B201A601C101E2
:109B00000E943C1B66246394712CFECE689480F8FE
:109B100091F8F8CFC654DF4F08811981CA5BD04055
:109B20000530110511F40C94974540E054E0B10163
:109B3000CE0187559F4F0E94B03A60E074E0F4CEAA
:109B40000E94B431672B682B692B11F00C944F3EA7
:109B5000912C812C11E0C854DF4F1883C85BD04092
:109B60000C94863ECD54DF4F28813981C35BD040B1
:109B7000232B09F053C08081882311F40C94B63C48
:109B8000CE018F549F4F0E945538CD54DF4F99839B
:109B90008883C35BD040C655DF4F8881CA5AD04006
:109BA0008F7091F5CD54DF4F6881C35BD040CE01FB
:109BB00087559F4F0E946B31CF55DF4F2883C15A85
:109BC000D040CE55DF4F3883C25AD040CD55DF4FFD
:109BD0004883C35AD040CC55DF4F5883C45AD04035
:109BE000CB55DF4F6883C55AD040CA55DF4F7883C5
:109BF000C65AD040C955DF4F8883C75AD040C85590
:109C0000DF4F9883C85AD040CD54DF4FE881F981A7
:109C1000C35BD040EF2B11F40C94B63C66E579E0C1
:109C200087E799E00E940C82B60187E799E00E94DD
:109C3000CE976FE479E087E799E00E940C82D1012A
:109C4000ED91FC916081718187E799E00E94A68186
:109C500069E479E087E799E00E940C82CF54DF4FF6
:109C600068817981C15BD04087E799E00E94A68135
:109C700067E479E087E799E00E940C82CE0187557E
:109C80009F4F0E94A22FCF54DF4FE881F981C15B23
:109C9000D040309711F40C94023D8081843211F051
:109CA0000C94023D63E379E087E799E00E940C821F
:109CB00087E799E00E9415818CEF682E77247A94CB
:109CC0009FC82F923F924F925F926F927F928F9296
:109CD0009F92AF92BF92CF92DF92EF92FF920F933B
:109CE0001F93CF93DF93CDB7DEB7C955D1090FB618
:109CF000F894DEBF0FBECDBF3C01562E6296EFAE8C
:109D000062976396FFAE639764960FAF649765960C
:109D10001FAF659766962FAF669767963FAF6797B9
:109D200068964FAF689769965FAF69976A96CFAEAE
:109D30006A972D2C4A2C3B2C009709F464C1FC0136
:109D400080858770843009F449C128F4882309F498
:109D50004EC180E02DC0853009F444C08630C9F77B
:109D60006AE074E0C3010E9427934C01009709F454
:109D70006FC0B12CA12CD12CC12C6296EFAC629794
:109D80006396FFAC639764960FAD649765961FADBD
:109D9000659766962FAD669767963FAD679768960D
:109DA0004FAD689769965FAD6997652D0E94614ECA
:109DB000C75ADF4F0FB6F894DEBF0FBECDBFDF919D
:109DC000CF911F910F91FF90EF90DF90CF90BF90B8
:109DD000AF909F908F907F906F905F904F903F904B
:109DE0002F90089580918D068F5F80938D068680D9
:109DF00097808114910431F1A42CB32C6A96CFACD6
:109E00006A97D22C6296EFAC62976396FFAC639729
:109E100064960FAD649765961FAD659766962FADF6
:109E2000669767963FAD679768964FAD6897699656
:109E30005FAD6997652DC4010E94614EF401828077
:109E40009380D7CF80918D06815080938D0681CFEE
:109E50006EE074E0C3010E9427937C0163E174E02B
:109E6000C3010E9427936C01552039F0F1E05F1681
:109E700009F495C010E000E00CC068E174E0C30193
:109E80000E9427934C016DE174E0C3010E94279367
:109E90008C018114910409F443010115110509F4A1
:109EA0008301E114F10421F46A96EFAC6A97F22C75
:109EB000C114D10411F4C42CD32C8114910409F4DD
:109EC0009FC0F40180858770843009F099C0818437
:109ED00092840115110509F49EC0F80180858770F0
:109EE000843009F098C001851285E114F10409F469
:109EF000E0C08114910409F49DC06BE177E187E72C
:109F000099E00E940C82F7016185728587E799E0EC
:109F10000E94A68166E177E187E799E00E940C82C2
:109F2000B40187E799E00E94A68187E799E00E9443
:109F30001581CE018F5A9F4F0E94A22FC114D104C8
:109F400009F0C0C0F70180858770843009F00CC12A
:109F500061857285CE0101960E948938CE010196F5
:109F60000E942B138823B1F00E94BF266B01683C2E
:109F700071050CF073C062EE76E180ED98E00E940E
:109F80000C82B60180ED98E00E94CE9780ED98E0BB
:109F90000E941581CE0101960E946113E5C062E224
:109FA00074E0C3010E9427934C0167E274E0C3018F
:109FB0000E9427938C018114910409F0D7C068E1B5
:109FC00074E0C3010E9427934C010115110509F4A7
:109FD0005ACF892B09F065CF430163CF10E000E031
:109FE000912C812CD12CC12CF12CE12C52CF10E0E2
:109FF00000E0912C812CD12CC12CF12CE12C51CFE3
:10A00000912C812C66CFCA2CDB2C6A96EFAC6A9718
:10A01000F22C912C812C00E020E033E040E150E074
:10A02000BE016F5B7F4FCE018F5A9F4F0E94812DE3
:10A030008C015BCF6CE077E187E799E00E940C82AE
:10A04000F7016185728587E799E00E94A68167E044
:10A0500077E187E799E00E940C826BCF811491042D
:10A0600031F0B401CE0101960E949B9893CFA12CB0
:10A07000CC24C394F12CE12C62960FAD62976396C9
:10A080001FAD639764962FAD649765963FAD659756
:10A0900066964FAD669767965FAD679768966FADAA
:10A0A000689769967FAD6997CE0101960E94F33B50
:10A0B00071CFC114D10409F457C00115110509F479
:10A0C00053C004C00115110509F43CCFF601808589
:10A0D0008770843009F044C060E077E187E799E059
:10A0E0000E940C82F6016185728587E799E00E94E3
:10A0F000A6816BEF76E187E799E00E940C82B801B8
:10A1000087E799E00E94A68187E799E00E94158180
:10A11000F6016185728540E450E0CE0101960E940F
:10A12000A3D20E9445938823D9F08091040881111D
:10A1300017C06FE270E0CE0101960E946AD2892BAF
:10A1400051F4F6012185328543E050E060E4CE0110
:10A1500001960E948A25B801CE0101960E948CA327
:10A16000E114F10409F0EECE81E022CE892B09F052
:10A1700098CE89CE8F929F92AF92BF92CF92DF926C
:10A18000EF92FF920F931F93CF93DF93CDB7DEB77C
:10A19000E0970FB6F894DEBF0FBECDBF84E0E0E1DC
:10A1A000F2E0DE01119601900D928A95E1F7FE0131
:10A1B00035968CE1DF011D928A95E9F7CE01019673
:10A1C000DB01685F7F4FFD900F2D10E0E4E01595F7
:10A1D0000795EA95E1F70C5A1D4FF8011081FC0133
:10A1E0001083EF2DEF70F0E0EC5AFD4F1081FC0171
:10A1F000118302966A177B0731F7198A1A8A8091B0
:10A20000B0059091B105892B09F46CC069017A0100
:10A2100087E799E00E94158164EC7CE087E799E08C
:10A220000E940C8242E0C701B6010E94B99B62EC19
:10A230007CE087E799E00E940C82BE016F5F7F4F50
:10A2400087E799E00E94A68160EC7CE087E799E0CF
:10A250000E940C8287E799E00E941581BE016F5F22
:10A260007F4F80919B0690919C060E9427934C0102
:10A2700020E030E04EEF52ECC701B6010E943FCC27
:10A28000882381F120E030E04AEA52E4C701B601B8
:10A290000E943FCC882331F120E030E0A901C701C2
:10A2A000B6010E943FCC8823E9F019A61AA61BA686
:10A2B0001CA68AA58F7080678AA7CDA6DEA6EFA60A
:10A2C000F8AA63E0CE0189960E946B31B12CA12CD3
:10A2D000D12CC12C79018A019B01AC016FEFC40123
:10A2E0000E94614EE0960FB6F894DEBF0FBECDBF60
:10A2F000DF91CF911F910F91FF90EF90DF90CF9062
:10A30000BF90AF909F908F9008956F927F928F92A1
:10A310009F92AF92BF92CF92DF92EF92FF920F93F4
:10A320001F93CF93DF93CDB7DEB7A0970FB6F89406
:10A33000DEBF0FBECDBF8C01862E7A01DC018D9170
:10A340009C911197892B09F460C01496ED91FC91B2
:10A35000309709F45AC080818071BFEF6B1357C0EA
:10A36000B1F481E0A0960FB6F894DEBF0FBECDBF6A
:10A37000DF91CF911F910F91FF90EF90DF90CF90E1
:10A38000BF90AF909F908F907F906F9008954330D3
:10A39000510539F3818082942FE082226DE776E0C7
:10A3A00087E799E00E940C82D80113966C9187E7A9
:10A3B00099E00E94C7976BE776E087E799E00E94F3
:10A3C0000C82D8011496ED91FC9161816F7087E742
:10A3D00099E00E94C79768E776E087E799E00E94D6
:10A3E0000C82682D87E799E00E94C79787E799E07C
:10A3F0000E941581D8011496ED91FC9181818F7096
:10A40000881207C080818F7E808380E0ABCF81116E
:10A41000FCCF198E1A8E1B8E1C8E1D8E1E8E1F8ECB
:10A4200018A28A8D8F708A8FD8011496ED91FC91B5
:10A4300081818F70881579F1B3E0EB16F10459F141
:10A4400066E776E087E799E00E940C82F801638175
:10A4500087E799E00E94C79764E776E087E799E08D
:10A460000E940C82D8011496ED91FC9161816F706D
:10A4700087E799E00E94C79761E776E087E799E070
:10A480000E940C82682D87E799E00E94C79787E7B2
:10A4900099E00E941581F80120813181FCE0F815D6
:10A4A00008F416C1E82DF0E08827E65AFD4A8F4FE0
:10A4B0000C9414CE6752A45225533C534853255351
:10A4C000FE5225534B535653125359536553D801DB
:10A4D0001496CD90DC90F60181818F70853009F45F
:10A4E000F7C050F48230C1F06AE374E0C9010E9401
:10A4F00027933C01912C4BC08730D1F08A30A1F7D3
:10A5000063E374E0C9010E9427933C01D6019C904B
:10A5100092FA992490F83BC06DE274E0C9010E9460
:10A5200027933C01D6019C9090FA992490F82FC073
:10A530006CE274E0C9010E9427933C01F60190800F
:10A5400091FA992490F823C06FE374E0C9010E9446
:10A5500027933C01D8011496ED91FC91808180FBFA
:10A56000992490F8982F9E7F80FF916090836114CA
:10A57000710469F461E0CE0149960E949231298B01
:10A580003A8B4B8B5C8B6D8B7E8B8F8B988FF8010E
:10A59000A080B1806EE074E0C5010E9427936C0139
:10A5A00063E174E0C5010E9427935C01892B81F46B
:10A5B000C114D10469F460E0CE0149960E94923141
:10A5C00029833A834B835C836D837E838F83988753
:10A5D000D8011496ED91FC916114710409F07CC0CE
:10A5E000898D811179C0B82DBF708B2E8181807FBC
:10A5F000882A818280818F7E8083B3CE64E474E078
:10A60000C9010E9427933C01D8011496ED91FC9159
:10A61000808181FB992490F8982F9D7F81FF926023
:10A620009083B5CF6AE474E0C9010E9427933C018E
:10A63000D8011496ED91FC91808182FB992490F8C9
:10A64000982F9B7F82FF9460EBCF6AE374E0C9018F
:10A650000E9427933C01892B09F04CCF62E0CE0188
:10A6600049960E94923129873A874B875C876D878C
:10A670007E878F87988B3ECF60E574E0C9010E948A
:10A6800027933C01D8011496ED91FC9190804CCF1A
:10A6900065E574E0F3CF6BE574E0C9010E94279390
:10A6A0003C01D8011496ED91FC9149CF61E674E02C
:10A6B000F4CF68E674E0C9010E9427933C01D801F9
:10A6C0001496ED91FC91908023CF6EE674E0F3CF69
:10A6D000912C712C612C5BCF83E0E816F104B9F06A
:10A6E000982D9F70892E8181807F882A8182808128
:10A6F0008F7E8083E98CFA8C0B8D1C8D2D8D3E8D89
:10A700004F8D58A1692DC3010E94614E2ACE8181CF
:10A710008F70881509F425CE829490EF8922882ABB
:10A7200081828081806168CF2F923F924F925F92A9
:10A730006F927F928F929F92AF92BF92CF92DF9251
:10A74000EF92FF920F931F93CF93DF93CDB7DEB7B6
:10A75000A7970FB6F894DEBF0FBECDBF4C013B01EB
:10A76000D0909805DD2009F4BFC080918D068F5FE1
:10A7700080938D06E0919906F0919A06309709F43E
:10A78000ABC046805780A0909906B0909A06A1145D
:10A79000B10409F49DC04114510409F499C0D201D7
:10A7A00018968C918770853091F7C2010E94D697D8
:10A7B000823068F3B201CE0101960E94A51CCE0141
:10A7C00001960E942B13882309F465C040E058E0ED
:10A7D00060E070E0CE0101960E94633B672B682B1E
:10A7E000692B09F458C01E8E1F8E18A219A21AA236
:10A7F0001BA21CA21DA28F8D8F708F8F40E053E093
:10A80000BE016F5F7F4FCE014E960E94A43064EB75
:10A8100079E087E799E00E940C8240E058E060E030
:10A8200070E0CE0101960E945E3A8A859B85009772
:10A8300091F1DC01ED91FC910488F589E02DA12CCA
:10A84000CC24C394F12CE12C0E8D1F8D28A139A1AD
:10A850004AA15BA16CA17DA119958F3F9807D9F002
:10A86000E981FA8160817181892BE9F487E799E0B8
:10A870000E94A68162EB79E087E799E00E940C8252
:10A880006AEA79E087E799E00E940C8287E799E01D
:10A890000E941581D12CF20142805380CE01019695
:10A8A0000E94611370CF87E799E00E94A68168EA51
:10A8B00079E087E799E00E940C8264EA79E087E713
:10A8C00099E00E940C8287E799E00E941581E3CF0E
:10A8D00087E799E00E94158180918D0681508093D1
:10A8E0008D06D1101092980565E0D4018D919C9150
:10A8F0000E949F936C01009709F4C0C0FC01A084E2
:10A90000A694A694A694FA2DFF70BF2EDC0119968A
:10A910002D903D904D905C901C970E94BEA2BB2054
:10A9200009F4ACC0261A370A480A590A1E8E1F8E2F
:10A9300018A219A2BE8E1F8D1F70106A1F8F2AA227
:10A940003BA24CA25DA2B4E06B16710439F5E12C78
:10A9500020E2F22E0B2D28A139A14AA15BA16CA106
:10A960007DA1C4010E94A7A3C201B10128EE33E07A
:10A9700040E050E00E94ABCDBA01A9012AE030E0EE
:10A9800087E799E00E94208162EE79E087E799E00D
:10A990000E940C8287E799E00E94158157FE6EC0E5
:10A9A000E2E02E1631044104E0E85E060CF466C0D5
:10A9B0000E94BF261B017FA36EA3E12C90E2F92E1B
:10A9C0000E8D1F8D28A139A14AA15BA16CA17DA18B
:10A9D000C4010E94A7A38EA19FA1883C910554F5B4
:10A9E00069EC79E080ED98E00E940C82B10180ED85
:10A9F00098E00E94CE9780ED98E00E9415818FEF3D
:10AA00009FEFA7960FB6F894DEBF0FBECDBFDF91C4
:10AA1000CF911F910F91FF90EF90DF90CF90BF905B
:10AA2000AF909F908F907F906F905F904F903F90EE
:10AA30002F900895D60118968C91189787701896C4
:10AA40008C9319821A821B821C821D821E821F8295
:10AA500018861A811F701A83B982A2948FE0A822E7
:10AA6000CC24C394F12CE12C0B2D2B813C8140E0B4
:10AA70005E816F817885C4010E94F33BB1E06B1663
:10AA80007104E9F440E053E060E070E0C4010E942A
:10AA9000633B611571058105910589F02091970649
:10AAA000309198062630310551F4C4010E94873B4D
:10AAB00040E053E060E070E0C4010E945E3AF401BF
:10AAC00081859285009719F490E080E09ACFDC01AF
:10AAD000ED91FC910484F585E02D1995892BA1F366
:10AAE000F40181859285DC01ED91FC910480F58172
:10AAF000E02DB301199585CFAF92BF92CF92DF922F
:10AB0000EF92FF920F931F93CF93DF93CDB7DEB7F2
:10AB10006D970FB6F894DEBF0FBECDBF0E94BEA2E8
:10AB20009B01AC016091AA057091AB058091AC05C9
:10AB30009091AD05A12CB12C650118EEE12E13E02A
:10AB4000F12E00E010E00E942825F82E882351F015
:10AB50000E94BEA26093AA057093AB058093AC05DA
:10AB60009093AD0580918D068F5F80938D06E09167
:10AB70009906F0919A060681178194E0C92ED12C8E
:10AB8000F11003C082E0C82ED12CA0909906B0909D
:10AB90009A06A114B10429F10115110511F1F8016A
:10ABA000808587708530A9F7C8010E94D6978230CA
:10ABB00080F3B801CE0101960E94A51CCE0101963A
:10ABC0000E942B13882329F0B601CE0101960E9422
:10ABD0009453F80102811381CE0101960E94611302
:10ABE000D4CF80918D06815080938D0680919706F9
:10ABF000909198060597D9F1FF20C9F110E0609176
:10AC0000B2057091B3056115710589F111112FC05D
:10AC1000FB0180858770853091F4CE0101960E94FA
:10AC2000A51C61E070E0CE0101960E94945311E0F2
:10AC3000892B09F410E0CE0101960E946113E09186
:10AC4000B205F091B305309791F082819381909392
:10AC5000B3058093B205892B91F6E0919906F091A6
:10AC60009A06868197819093B3058093B2056D967D
:10AC70000FB6F894DEBF0FBECDBFDF91CF911F910D
:10AC80000F91FF90EF90DF90CF90BF90AF9008951D
:10AC90002F923F924F925F926F927F928F929F92EC
:10ACA000AF92CF92DF92EF92FF920F931F93CF93C9
:10ACB000DF93CDB7DEB76D970FB6F894DEBF0FBE4A
:10ACC000CDBF009709F4A9C0FC013085377035303D
:10ACD00009F0A3C0D22E1A014B01668077808091C3
:10ACE0008D068F5F80938D066114710409F490C006
:10ACF000F30180858770843009F086C06185728594
:10AD00008091990690919A060E9427932C010097B2
:10AD100009F47AC0FC0180858770853009F074C021
:10AD2000B201CE0101960E94A51C81149104B1F0DC
:10AD3000CE0101960E942B13882381F0AD2CC12CEB
:10AD40007101F40100811181228133814481558197
:10AD500066817781CE0101960E94F33B60E0C201DB
:10AD60000E949F930097E9F1FC0120852770223013
:10AD7000C1F581859285A385B4850797A105B105A5
:10AD800081F561E0C2010E949F932D2DA101B401C4
:10AD90000E9448568114910499F5882389F1809185
:10ADA0008D06815080938D06CE0101960E9461131D
:10ADB00081E06D960FB6F894DEBF0FBECDBFDF9178
:10ADC000CF911F910F91FF90EF90DF90CF90AF90B8
:10ADD0009F908F907F906F905F904F903F902F90BB
:10ADE00008958114910461F4CE0101960E942B1301
:10ADF000882331F0CE0101960E940F57892B79F6F6
:10AE0000CE0101960E946113F301628073806CCFC2
:10AE100080918D06815080938D0680E0CACFDF92AD
:10AE2000EF92FF920F931F93CF93DF9300D000D048
:10AE30001F921F92CDB7DEB77C0119821A821B8246
:10AE40001C821D821E821F8218868A818F708A83CF
:10AE5000D701ED91FC916081718187E799E00E94B3
:10AE6000A68162EA79E087E799E00E940C82C70137
:10AE70000E942B1381111BC069E979E087E799E0F3
:10AE80000E940C8287E799E00E9415810FEF1FEF67
:10AE9000C80128960FB6F894DEBF0FBECDBFDF9174
:10AEA000CF911F910F91FF90EF90DF900895C70110
:10AEB0000E94EB18D82EF70181859285009791F0BA
:10AEC000DC01ED91FC910688F789E02D19958C0144
:10AED00097FD08C081E00115110509F480E00E948A
:10AEE000DD15D6CFF7018085873009F42EC0EFEF4E
:10AEF000ED0DE43150F5F0E08827EE57F84A8F4F1A
:10AF00000C9414CE96579F57A557A5579F57965701
:10AF1000A557A557A557A557A557A557A557965760
:10AF2000A557A557A557A557965796576AE779E0AD
:10AF300087E799E00E940C8201E010E0A9CF80E051
:10AF40000E94DD1510E000E0A3CF40E052E0B70121
:10AF5000CE0101960E94A430D70118968C911897C3
:10AF6000873071F160F4833009F454C0843061F0AB
:10AF70006AE879E087E799E00E940C82E3CF8830A5
:10AF800009F448C08930A1F7CE0101960E94AE9322
:10AF90008C016FE779E087E799E00E940C82B801A5
:10AFA00087E799E00E94CE9787E799E00E94158194
:10AFB00091E080E0012B09F490E0092F182F68CF71
:10AFC0001296ED91FC918085877010E000E085304D
:10AFD00001F767E979E087E799E00E940C8220E0B9
:10AFE00050E040E070E060E0F701828193810E94D0
:10AFF0004856F82E082F10E064E979E087E799E0D9
:10B000000E940C828F2D0E94DD1587E799E00E9437
:10B0100015813ECFCE0101960E94B4318B01B9CF8C
:10B020002F923F924F925F926F927F928F929F9258
:10B03000AF92BF92CF92DF92EF92FF920F931F9346
:10B04000CF93DF93CDB7DEB760970FB6F894DEBF2E
:10B050000FBECDBF6130710509F494C0DC011296BA
:10B060006D917C916115710509F48CC04C011982B8
:10B070001A821B821C821D821E821F8218868A8170
:10B080008F708A8340E052E0CE0101960E94A43086
:10B09000CE0101960E94AE931C01F401828193813E
:10B0A0000E94A0182B013C01D40117962D913D91CF
:10B0B0004D915C911A97D1010E94D5CD2FEF30E0D0
:10B0C00040E050E00E9489CD29873A874B875C8712
:10B0D0000E94BEA29B01AC0189859A85AB85BC8587
:10B0E0000097A105B10509F468C0A12CB12C650138
:10B0F0007C018D01C301B2010E942825898741147A
:10B10000510461047104F1F1D40117968D919D9160
:10B110000D90BC91A02D8D879E87AF87B88B0E9424
:10B12000BEA29B01AC018D859E85AF85B889009735
:10B13000A105B10561F0A12CB12C65017C018D0147
:10B14000C301B2010E942825882309F451C0D4010B
:10B1500012966D907C9080E00E943015AB01BC018E
:10B16000C3010E943C1B232869F0F40184810E94E2
:10B170004112D40116969C91891304C061E0C40168
:10B180000E94F81890E080E060960FB6F894DEBF59
:10B190000FBECDBFDF91CF911F910F91FF90EF9028
:10B1A000DF90CF90BF90AF909F908F907F906F90E7
:10B1B0005F904F903F902F90089591E099879FCF97
:10B1C000B985BB23F1F060E0C4010E94F818F401D6
:10B1D000828193810E940F57892BA1F640E050E0B5
:10B1E000BA01D40112968D919C910E943C1BCACF4A
:10B1F000F40184810E944112D40116969C91891316
:10B20000DFCF232809F4BECFF40184810E944112CC
:10B21000D40116969C918913B5CFB985B111B2CFDF
:10B22000ADCFCF93DF93EC0161EF75E187E799E054
:10B230000E940C826C817D8187E799E00E94CE9705
:10B240006BEE75E187E799E00E940C8287E799E051
:10B250000E94158161E08C810E94089F6E818C8123
:10B260000E94DA9E8A819B81009729F040E050E09D
:10B27000BA010E943C1B81E090E09093B605809358
:10B28000B5058A819B810E940F57181619065CF438
:10B290000A80DB81C02D80E00E943015AB01BC012B
:10B2A000CE010E943C1B81E090E0DF91CF91089598
:10B2B0002F923F924F925F926F927F928F929F92C6
:10B2C000AF92BF92CF92DF92EF92FF920F931F93B4
:10B2D000CF93DF93CDB7DEB7C955D1090FB6F89438
:10B2E000DEBF0FBECDBF0E94BEA29B01AC0160912C
:10B2F000A6057091A7058091A8059091A905A12C9C
:10B30000B12C650110E3E12E15E7F12E00E010E00D
:10B310000E942825882309F422C2E0919906F09121
:10B320009A06309709F41BC280918D068F5F809337
:10B330008D062680378010E02114310409F434C1D1
:10B34000F101808587708530F9F460E0C1010E94C9
:10B350009F93FC0181859285A385B4850597A105FE
:10B36000B10591F4B101CE0101960E94A51CCE0158
:10B3700001960E942B1366968FAF6697811108C0C5
:10B38000CE0101960E946113F10122803380D4CF57
:10B3900025961CAE1DAE1EAE1FAE259729961CAE7F
:10B3A0001DAE1EAE1FAE299740E052E0BE016F5F9A
:10B3B0007F4FCE018F5B9F4F0E94A430CE0101963C
:10B3C0000E94A0186B017C0169966FAF69976A961D
:10B3D000DFAE6A97CE0101960E94E6974C01CE013E
:10B3E0008F5B9F4F0E94C21265966CAF7DAF8EAF90
:10B3F0009FAF6597CE0101960E94EB18182FB601FA
:10B40000DD0C880B990B0E9446CC20E030E048EC24
:10B4100052E40E949FCE2B013C01CE0101960E9476
:10B420000F5768969FAF8EAF689768E475E187E71E
:10B4300099E00E940C8242E065966CAD7DAD8EADC8
:10B440009FAD65970E94B99B62E475E187E799E03B
:10B450000E940C8242E0C301B2010E94B99B6CE3DE
:10B4600075E187E799E00E940C82612F70E087E721
:10B4700099E00E94CE97E114F10409F48EC088E0AF
:10B480000E9430159B01AC0144275527B70190E07D
:10B4900080E0AA24AA94BA2CC12CD12C17E2E12E68
:10B4A00019E0F12E00E010E00E942825882371F1B8
:10B4B000F1016081718180ED98E00E94A6816CE2CB
:10B4C00075E180ED98E00E940C82F101608171814C
:10B4D00085E794E00E948CA690E080E0BC0169962C
:10B4E0004FAD69976A965FAD6A97CE0101960E944B
:10B4F0003C1B62E070E0C4010E94FD17CE01019682
:10B500000E94611366961FAD66973ECF20E030E043
:10B5100048E152E4C301B2010E9447CF18163CF43F
:10B52000F1016081718181E894E00E948CA66896A7
:10B530008EAD9FAD6897892B19F461E070E0DBCF89
:10B5400020E030E040E85FE365966CAD7DAD8EAD08
:10B550009FAD65970E9432CE9B01AC01C301B20141
:10B560000E943FCC70E060E087FDC5CFA30192014F
:10B5700065966CAD7DAD8EAD9FAD65970E943FCC5D
:10B580001816DCF66DE175E187E799E00E940C8200
:10B5900087E799E00E941581B1CF63E175E187E704
:10B5A00099E00E940C82AACF80918D0681508093F1
:10B5B0008D060E94BEA26093A6057093A705809396
:10B5C000A8059093A9050E94BF262B013C010E946B
:10B5D000BEA26B017C010E944593882309F489C0B7
:10B5E00080910408811185C030E020E041E050E006
:10B5F00060E4CE0101960E948A254FE350E063E3A8
:10B600007BE1CE0101960E9463C662EC73E0CE013D
:10B6100001960E945FD24FE350E06AEE74E1CE01E2
:10B6200001960E9463C62AE0AE014F5B5F4FC301E3
:10B63000B2010E94EEC6BE016F5B7F4FCE01019644
:10B640000E948CA330E020E041E050E060E4CE01B5
:10B6500001960E948A254FE350E063E37BE1CE012F
:10B6600001960E9463C662EC73E0CE0101960E94CF
:10B670005FD24FE350E063EE74E1CE0101960E9489
:10B6800063C6C701B60128EE33E040E050E00E94F7
:10B6900089CDCA01B9012AE0AE014F5B5F4F0E941C
:10B6A000EEC6BE016F5B7F4FCE0101960E948CA358
:10B6B00030E020E041E050E060E4CE0101960E94DD
:10B6C0008A254FE350E063E67BE1CE0101960E94BC
:10B6D00063C64FE050E06DE57BE1CE018F5B9F4F8D
:10B6E0000E9481C6BE016F5B7F4FCE0101960E9412
:10B6F0008CA3112309F44DC06DE075E187E799E053
:10B700000E940C820E94BF26AB01BC0187E799E032
:10B710000E94C49765E075E187E799E00E940C827A
:10B7200060918D06062E000C770B87E799E00E944A
:10B73000CE9763EF74E187E799E00E940C82409115
:10B74000A2055091A3056091A4057091A50587E716
:10B7500099E00E94C49787E799E00E941581C75A33
:10B76000DF4F0FB6F894DEBF0FBECDBFDF91CF9194
:10B770001F910F91FF90EF90DF90CF90BF90AF900F
:10B780009F908F907F906F905F904F903F902F9001
:10B79000089563E075E187E799E00E940C820E94BA
:10B7A000BF26AB01BC0187E799E00E94C4976BEF0D
:10B7B00074E1B2CF3F924F925F926F927F928F92DD
:10B7C0009F92AF92BF92CF92DF92EF92FF920F9330
:10B7D0001F93CF93DF93CDB7DEB7CE56D1090FB607
:10B7E000F894DEBF0FBECDBFDC0114962D913C91C5
:10B7F000232B09F422C69B01225031092230310546
:10B8000008F091C23B014C01FC018281803409F4B3
:10B81000F7C208F04AC0843008F085C280919705CD
:10B820008F5F80939705A3016FEFC4010E9485513C
:10B83000D40112960C9112970695017013961C91E3
:10B8400013978AEC810F803108F043C06EE874E0F2
:10B850008D919C910E9427937C010097D1F1FC016E
:10B86000808587708530A9F58091B609181324C0AA
:10B870008091B709803401F58091B8099091B90998
:10B880005C01990FCC08DD0860E0C7010E949F931E
:10B89000FC0181859285A385B485A816B906CA06E0
:10B8A000DB060CF065C0512C3EC0823409F4A8C2FE
:10B8B00008F439C28058AFCF1093B60980E4809362
:10B8C000B709812F0E94449F9093B9098093B809CA
:10B8D000D7CF212F30E0F901EB55F34E8491F901D8
:10B8E000EB5FF24E1491F901E55BF24EF490FF200C
:10B8F00009F43BC081110E94739EEF2DF0E0EE0F22
:10B90000FF1FE95AF94FA591B491EC911E2331E044
:10B9100020E009F430E0832F922F55245394081728
:10B92000190609F0C0CFF3E06F16710409F488C05E
:10B93000D4011496ED91FC91E181EF70E150EC306F
:10B9400008F07EC0F0E08827E755F34A8F4F0C944B
:10B9500014CECA5C465E005D365D465E4F5D465E57
:10B96000835DB05DC95D0B5E2D5E90E080E0D5CF5C
:10B9700061E0C7010E949F9355245394FC01818587
:10B980009285A385B4858A159B05AC05BD050CF091
:10B99000CACF89CF0E94BEA29B01AC014427552784
:10B9A000D4011496ED91FC916281738190E080E066
:10B9B000AA24AA94BA2CC12CD12C18EEE12E13E0A3
:10B9C000F12E00E010E00E9428258823C9F1F4013F
:10B9D0000081118160E574E0C8010E942793892BE2
:10B9E00041F465E574E0C8010E942793892B09F4AE
:10B9F0000EC142E050E063E0C4010E94855120C0C6
:10BA00000E94BEA29B01AC0144275527D401149685
:10BA1000ED91FC916281738190E080E0AA24AA9468
:10BA2000BA2CC12CD12C1CE2E12EFF24F39400E0AF
:10BA300010E00E94282542E050E064E0811184C0BB
:10BA4000D4011496ED91FC91808183FB992790F9A4
:10BA5000951509F4D2C1982F907E09F439C1982F19
:10BA6000907E90528F71892B808358C10E94BEA214
:10BA70009B01AC0144275527D4011496ED91FC910C
:10BA80006281738190E080E0AA24AA94BA2CC12C30
:10BA9000D12C16E9E12EF12C00E010E0CACF0E9473
:10BAA000BEA29B01AC0144275527D4011496ED9109
:10BAB000FC916281738190E080E0AA24AA94BA2C60
:10BAC000C12CD12C18EEE12E13E0F12E00E010E095
:10BAD0000E942825882309F4B3CFF4010081118145
:10BAE0006BE574E0C8010E942793892B41F461E65D
:10BAF00074E0C8010E942793892B09F488C042E0B2
:10BB000050E068E079CF0E94BEA29B01AC014427BF
:10BB10005527D4011496ED91FC916281738190E0D8
:10BB200080E0AA24AA94BA2CC12CD12C1CE2E12ECC
:10BB3000FF24F39400E010E00E94282542E050E04A
:10BB400069E0882309F47CCFC4010E9485510E94DA
:10BB5000BEA2D4011496ED91FC917383628370CFE1
:10BB60000E94BEA29B01AC0144275527D401149624
:10BB7000ED91FC916281738190E080E0AA24AA9407
:10BB8000BA2CC12CD12C16E9E12EF12C00E010E0EA
:10BB9000D3CF0E94BEA29B01AC0144275527D401FC
:10BBA0001496ED91FC916281738190E080E0AA246B
:10BBB000AA94BA2CC12CD12C18EEE12E13E0F12E50
:10BBC00000E010E00E942825882309F439CFF40111
:10BBD0000081118168E674E0C8010E942793892BD7
:10BBE00039F46EE674E0C8010E942793892B21F096
:10BBF00042E050E06BE000CF6AE474E0C8010E94CC
:10BC0000279342E050E066E0892B09F4F5CE42E04C
:10BC100050E06DE0F1CE0E94BEA29B01AC01442732
:10BC20005527D4011496ED91FC916281738190E0C7
:10BC300080E0AA24AA94BA2CC12CD12C1CE2E12EBB
:10BC4000FF24F39400E010E00E942825882309F4E3
:10BC5000F7CE42E050E06CE077CF0E94BEA29B019D
:10BC6000AC0144275527D4011496ED91FC916281D3
:10BC7000738190E080E0AA24AA94BA2CC12CD12C24
:10BC800016E9E12EF12C00E010E0DECF0E94BEA20A
:10BC90009B01AC0144275527D4011496ED91FC91EA
:10BCA0006281738190E080E0AA24AA94BA2CC12C0E
:10BCB000D12C18E5E12E12E0F12E00E010E00E94F8
:10BCC0002825882309F4BCCE42E050E060E094CE01
:10BCD0000E94BEA2D4011496ED91FC911597738336
:10BCE0006283E181EF70552009F445C0E230F1F044
:10BCF00050F4EE23E9F1D4011496ED91FC9180818A
:10BD000050FA83F9B1CEE53089F0A3016AE0E7305B
:10BD100091F7C4010E9485518111EDCF8091970563
:10BD200081508093970590E080E089C3F401008101
:10BD3000118164E474E0C8010E942793892BA9F45F
:10BD40006BE574E0C8010E942793892B71F461E6CA
:10BD500074E0C8010E942793892B39F46CE274E0E7
:10BD6000C8010E942793892B19F0A30166E0D1CF67
:10BD7000A30161E0CECFE150ED3008F0BCCFF0E0A0
:10BD80008827EA53F14A8F4F0C9414CED35E7B5E22
:10BD9000D65ED65E7B5ED95E7B5EFA5EFA5EFA5E4A
:10BDA000FA5EFA5ED65EA30162E0B3CFA30165E05E
:10BDB000B0CF0D911C9164E474E0C8010E942793F8
:10BDC000892BA9F46BE574E0C8010E942793892BA5
:10BDD00071F461E674E0C8010E942793892B39F45D
:10BDE0006CE274E0C8010E942793892B19F0A3012B
:10BDF00067E08FCFA30160E08CCF8F71806434CE79
:10BE0000B3E06B16710409F48ECF6EE874E0F401B0
:10BE1000808191810E9427938C01D40113968C918B
:10BE20009091B6098913EBC09091B709903409F04D
:10BE3000E6C08091B8099091B9093C01011511053E
:10BE400009F40DC1F80120852770253009F007C1DC
:10BE5000C8010E94D697382EF3E0F81708F0DBC02F
:10BE600063E0C8010E949F93DC0119968D919C911B
:10BE70003AE0E32EE89E6001E99ED00C1124A396DF
:10BE8000DFAECEAEA39762E0C8010E949F93DC01B3
:10BE900019968D919C91E89E2001E99E500C1124E9
:10BEA0006201052C000CEE08FF08AF96CCAEDDAEAB
:10BEB000EEAEFFAEAF9761E0C8010E949F935C01B8
:10BEC00060E0C8010E949F93DC011996CD90DD903F
:10BED000ED90FC901C97A796CCAEDDAEEEAEFFAE1B
:10BEE000A7979301072C000C440B550B2C193D0907
:10BEF0004E095F09A396CEACDFACA397B601DD0C6B
:10BF0000880B990BAF96CCACDDACEEACFFACAF9729
:10BF10006C197D098E099F090E9479CDD50119966A
:10BF20002D913D914D915C911C97A796CCACDDACC9
:10BF3000EEACFFACA7972C193D094E095F09A796F7
:10BF40002CAF3DAF4EAF5FAFA7970E94ABCDAF9682
:10BF5000ACACBDACCEACDFACAF97A20EB31EC41E72
:10BF6000D51E45E0E42E3E1409F468C081E090E05F
:10BF7000A396EEACFFACA397A701FF0C660B770B63
:10BF80004A155B056C057D050CF461C0B601A50181
:10BF90006201052C000CEE08FF084C155D056E05CE
:10BFA0007F050CF459C06A017B0122E032126BC09C
:10BFB0006301770CEE08FF0860E0C8010E949F93C0
:10BFC000FC0181859285A385B485C816D906EA0649
:10BFD000FB060CF44DC261E0C8010E949F93FC0176
:10BFE00081859285A385B4858C159D05AE05BF0519
:10BFF0000CF099CE81E090E0A0E0B0E03CC28093EC
:10C00000B60990E49093B7090E94449F9093B909B0
:10C010008093B80912CF8AE0869D5001879DB00CAD
:10C0200011240B2C000CCC08DD08512C412C20E0F5
:10C0300038E2A3963FAF2EAFA39798CF64E0C80134
:10C040000E949F93DC0119968D919C9191CF66245B
:10C050006A9423E0722E9CCF712C612CA6CF2AE02B
:10C06000289F6001299FD00C11240D2C000CEE0894
:10C07000FF08512C412C20E038E2A3963FAF2EAFB1
:10C08000A39781E090E0D4011496ED91FC91628138
:10C090007381A301461B570B57FF03C05195419570
:10C0A0005109841795070CF4C1C08081982F92958F
:10C0B00096959770963008F0BCC09F5F9295990F47
:10C0C000907E8F71892BB4C0F70161857285DB0189
:10C0D0008C9181115DC2A114B10409F473C0D50122
:10C0E00018968C9118978770843009F06BC0199658
:10C0F0006D917C91CE0101960E948938CE01019606
:10C100000E942B13882309F459C06114710409F4A7
:10C1100060C0E114F10431F0F7018085877084304C
:10C1200009F442C025961CAE1DAE1EAE1FAE25976B
:10C1300029961CAE1DAE1EAE1FAE299723961FADCD
:10C1400023971F7023961FAF239781E022968FAF0E
:10C150002297A12CCC24C394F12CE12C01E024964D
:10C160002FAD249725963FAD259740E027965FADEC
:10C17000279728966FAD289729967FAD2997CE01EE
:10C1800001960E94F33B1AC00115110529F0F80130
:10C1900080858770843019F065E974E0F9C16185A4
:10C1A0007285FB01808195CF61857285FB0180815D
:10C1B000882321F0CE0101960E949B98CE01019622
:10C1C0000E946113D4011496ED91FC9173826282F6
:10C1D000AACD0115110531F0D80118968C91877000
:10C1E0008430F1F025961CAE1DAE1EAE1FAE259715
:10C1F00029961CAE1DAE1EAE1FAE299723961FAD0D
:10C2000023971F7023961FAF239782E022968FAF4C
:10C210002297A12CCC24C394F12CE12C02E09FCFD7
:10C22000F80161857285DB018C91C2CF80818F71AD
:10C2300080838081803AB8F0C201550CAA0BBB0BF9
:10C24000C816D906EA06FB0671F0A396EEADFFAD5F
:10C25000A397CF01FF0FAA0BBB0BC816D906EA069E
:10C26000FB0609F060CD6616770609F45CCD6D9685
:10C270001CAE1DAE1EAE1FAE6D976B968FAD6B974D
:10C280008F7080666B968FAF6B976D968CAD9DAD02
:10C29000AEADBFAD6D9765968CAF9DAFAEAFBFAF86
:10C2A0006597AAE0B0E0A70196010E94CACD699601
:10C2B0006CAF7DAF8EAF9FAF699766E476E087E79E
:10C2C00099E00E940C82D40113966C9187E799E063
:10C2D0000E94C79764E476E087E799E00E940C82A9
:10C2E000CE018F5A9F4F0E94A22F6AE074E0F401A2
:10C2F000808191810E942793B12CA12CD12CC12C3B
:10C300006296EFAC62976396FFAC639764960FAD4D
:10C31000649765961FAD659766962FAD669767968D
:10C320003FAD679768964FAD689769965FAD69971F
:10C330006FEF0E94614ED4010D911C916EE074E08C
:10C34000C8010E9427937C0163E174E0C8010E9448
:10C3500027938C010097E1F1FC0180858770843080
:10C36000B9F56185728540E450E0CE0101960E94E6
:10C37000A3D26FE270E0CE0101960E946AD2892BAF
:10C3800059F4D80119962D913C9143E050E060E4B6
:10C39000CE0101960E948A2500E020E032E040E1D3
:10C3A00050E0BE016F5B7F4FCE018F5A9F4F0E94BE
:10C3B000812D0E944593882359F0809104088111B2
:10C3C00007C0BE016F5B7F4FCE0101960E948CA318
:10C3D000E114F10409F4F6CEF7018085877084300A
:10C3E00009F0F0CE61857285CE0101960E948938F0
:10C3F000CE0101960E942B13882309F4DFCEA12CD5
:10C40000CC24C394F12CE12C62960FAD6297639615
:10C410001FAD639764962FAD649765963FAD6597A2
:10C4200066964FAD669767965FAD679768966FADF6
:10C43000689769967FAD6997A2CE8FEF9FEFC2593B
:10C44000DF4F0FB6F894DEBF0FBECDBFDF91CF91A7
:10C450001F910F91FF90EF90DF90CF90BF90AF9022
:10C460009F908F907F906F905F904F903F90089536
:10C4700080E090E0DC01F40124813581F901428102
:10C480005381052E000C660B770B84179507A607C2
:10C49000B70709F448CC3C01D4010D911C916EE022
:10C4A00074E0C8010E9427935C0163E174E0C80155
:10C4B0000E9427936C01A114B10419F4892B09F48B
:10C4C00081CE6FE374E0C8010E9427937C016AE388
:10C4D00074E0C8010E9427938C016CE476E087E742
:10C4E00099E00E940C82F401638187E799E00E9441
:10C4F000C7976AE476E087E799E00E940C82B3016F
:10C5000087E799E00E94CE9787E799E00E9415811E
:10C51000C114D10409F4DFCDD60118968C91189777
:10C520008770843009F0D7CD19966D917C9140E4E5
:10C5300050E0CE0101960E94A3D20E944593882329
:10C5400009F4C9CD809104088111C5CD6FE270E076
:10C55000CE0101960E946AD2892B51F4F601218501
:10C56000328543E050E060E4CE0101960E948A25C6
:10C570006114710409F408CEE114F10439F0D70113
:10C5800018968C918770843009F49ECD62E974E02E
:10C59000CE0101960E948CA39ECD8F929F92AF9266
:10C5A000BF92CF92DF92EF92FF920F931F93CF93A0
:10C5B000DF9300D000D0CDB7DEB72091AE0530912B
:10C5C000AF05232B09F4C5C02091A1052111C1C0DD
:10C5D0004C018091A1058F5F8093A10580918D060C
:10C5E0008F5F80938D060E94BEA29B01AC0160917B
:10C5F0009D0570919E0580919F059091A005A12CAD
:10C60000B12C65011BE0E12EF12C00E010E00E944E
:10C610002825882309F452C0E091AE05F091AF05BA
:10C620000681178101151105B9F1F8018085877020
:10C63000863071F56AE074E0C8010E942793009784
:10C64000D1F0FC01208527702530A9F4E680F78021
:10C65000E114F104E9F0FA82E982B801CE01019611
:10C660000E94BB1CB401CE0101960E94DA5BF70167
:10C67000E280F380EDCF1A83098370E060E0CE01A1
:10C6800001960E94BB1CB401CE0101960E94DA5BA8
:10C69000F80102811381C6CFF3E08F16910451F0A7
:10C6A0000E94BEA260939D0570939E0580939F0596
:10C6B0009093A0051092B6091092B70983E08816EE
:10C6C0009104E9F10E94BEA29B01AC016091990521
:10C6D00070919A0580919B0590919C05A12CB12C9D
:10C6E000650118E8E12E13E1F12E00E010E00E9450
:10C6F0002825882321F1E091AE05F091AF05068150
:10C7000017810115110589F0F80180858770863041
:10C7100041F41A83098370E060E0CE0101960E9423
:10C72000BB1CF80102811381ECCF0E94BEA2609372
:10C73000990570939A0580939B0590939C05809131
:10C740008D06815080938D068091A1058150809344
:10C75000A10526960FB6F894DEBF0FBECDBFDF91C0
:10C76000CF911F910F91FF90EF90DF90CF90BF90EE
:10C77000AF909F908F9008954F925F926F927F92AB
:10C78000AF92BF92CF92DF92EF92FF920F931F93DF
:10C79000CF93DF93CDB7DEB76D970FB6F894DEBFBA
:10C7A0000FBECDBF66ED75E187E799E00E940C8270
:10C7B00087E799E00E9415810E94BEA22B013C01EF
:10C7C00080918D06882371F10E94BEA29B01AC016D
:10C7D000A12CB12C650110E1E12E17E2F12E00E051
:10C7E00010E0C301B2010E94282581111BC00E94E4
:10C7F000578380919D0681116BC08091970690911F
:10C800009806059741F08091990690919A06892B98
:10C8100011F00E947C550E94585982E090E00E94DD
:10C82000CD62CECF80918D06FF24F394882359F0FA
:10C8300063EB75E180ED98E00E940C8280ED98E05A
:10C840000E941581F12C6DE975E187E799E00E945E
:10C850000C8287E799E00E9415818091B4058F5F73
:10C860008093B405E0919906F0919A063097D1F142
:10C870000681178101151105A9F1D80118968C912F
:10C8800087708530B9F7C8010E94D697882391F345
:10C89000F80160817181CE0101960E948938CE0134
:10C8A00001960E942B13882359F08A859B85009757
:10C8B00039F0DC01ED91FC910284F385E02D1995AE
:10C8C000CE0101960E946113F80102811381D2CF3B
:10C8D00080919B0690919C06892B09F48ECF0E9433
:10C8E00041288BCF1092B3051092B20565E975E12E
:10C8F00087E799E00E940C8287E799E00E94158102
:10C9000064E670E080E090E00E9479A01092190641
:10C9100010928E066DE775E187E799E00E940C8220
:10C920000E94BF26AB01BC0187E799E00E94C49733
:10C930008091B0059091B105009711F00E949B9CE9
:10C940001092B1051092B0051092AF051092AE058D
:10C9500010929A061092990610921B0610921A06CF
:10C9600010928B0610928A06109289061092880601
:10C9700010929C0610929B0668E775E187E799E0A4
:10C980000E940C820E94BF26AB01BC0187E799E0A0
:10C990000E94C49787E799E00E94158110928C0647
:10C9A0008091B40581508093B4058F2D6D960FB69C
:10C9B000F894DEBF0FBECDBFDF91CF911F910F91D5
:10C9C000FF90EF90DF90CF90BF90AF907F906F90EF
:10C9D0005F904F900895809104088F5F80930408C2
:10C9E000A89583E090E00E94CD620E9457838091D9
:10C9F00004088150809304080895CF92DF92EF924B
:10CA0000FF920F931F93CF93DF93FC012485243073
:10CA100059F090E080E0DF91CF911F910F91FF904E
:10CA2000EF90DF90CF9008956A018B01EC01F12C1B
:10CA30008F2D0E949E8F811127C0FC868C858430AB
:10CA400041F320910202309103022F5F3F4F21F109
:10CA5000309303022093020240910202509103029C
:10CA600020E061E00E94EF8EF80182818F3FB9F4EF
:10CA700083818F3FF9F484818F3FE1F485818F3F7B
:10CA8000C9F484E08C87C5CF8B7F8831B1F2F394F1
:10CA9000F4E0FF12CDCFD2CF20E030ECD9CF81111E
:10CAA00009C08381811106C08481811103C0858101
:10CAB000882339F3C114D10421F3FC8480E590E08C
:10CAC0000E94E59CB8016E5F7F4F8F2D0E94521E21
:10CAD000B6018F2D0E94411E64E070E08F2D0E94F0
:10CAE000449D0E94BEA26B017C01F4E9CF0EF1E1EE
:10CAF000DF1EE11CF11CCE010E945B1E873149F153
:10CB000061E070E080E090E00E9479A00E94EB6418
:10CB1000CE010E945B1E882309F4B3CF0E94BEA2FF
:10CB2000C616D706E806F90630F78C850E94DB8E1C
:10CB3000EC85F0E0EE0FFF1FE157F94F11821082F4
:10CB400084E08C876DE278E18AED98E00E94308283
:10CB500060CF62E278E18AED98E00E94308281E065
:10CB600090E059CFA89583E090E00C94CD625F925D
:10CB70006F927F928F929F92AF92BF92CF92DF92ED
:10CB8000EF92FF920F931F93CF93DF93CDB7DEB752
:10CB9000A3970FB6F894DEBF0FBECDBF8091B0054E
:10CBA0009091B105892B09F429C480918D068111DA
:10CBB00025C480918D068F5F80938D0667E770E1B5
:10CBC00086EC98E00E940C8286EC98E00E94158129
:10CBD0000091B0051091B10569E974E0C8010E94A7
:10CBE000279390939A06809399066FE974E0C801A1
:10CBF0000E94279390931B0680931A066AED74E0B7
:10CC0000C8010E9427939093AF058093AE0566EA12
:10CC100074E0C8010E94279390938B0680938A0644
:10CC20000E94B82C6BEA74E08091B0059091B10538
:10CC30000E94279390939C0680939B06009709F48B
:10CC4000BBC120919D062111B7C1DC011696ED9064
:10CC5000FC908091860690918706892B51F081E0A7
:10CC600080939D0667E670E186EC98E00E940C8256
:10CC700055C06EE270E187E799E00E940C8287E779
:10CC800099E00E94158168E270E187E799E00E94CF
:10CC90000C820E94BF26AB01BC0187E799E00E948D
:10CCA000C49787E799E00E9415818FE090E00E9489
:10CCB00011C48C0188E1F8018183128210821686EA
:10CCC000158610926506109264061092E107109284
:10CCD00003080E94A9158AEBA82E81E1B82EB09214
:10CCE0003E06A0923D069BEBC92E91E1D92ED09233
:10CCF0004206C09241061093870600938606012BD8
:10CD000009F0B1C066E170E180ED98E00E940C820C
:10CD100080ED98E00E94158110929D061092C0054A
:10CD20001092BF05CC24C394D12CE114F10409F472
:10CD300043C180919D06882309F43EC1D70118960E
:10CD40008C9118978770863009F089C00D911C91DD
:10CD5000FE0131965F014801F0E18F0E911C350113
:10CD6000D8018C910E949612582EF80181810E9460
:10CD700096125294A0EF5A22582AD5015D925D0175
:10CD80000E5F1F4F8016910659F763E97FE086EC2E
:10CD900098E00E940C826091BF057091C00586ECFE
:10CDA00098E00E94CE976CE87FE086EC98E00E94C5
:10CDB0000C828091BF059091C005F3E0880F991F08
:10CDC000FA95E1F72091BD053091BE05820F931FC2
:10CDD0000E94659B86EC98E00E9415812091BF051A
:10CDE0003091C00521313105D4F56091BD057091B8
:10CDF000BE0548E0C901E3E0880F991FEA95E1F715
:10CE0000860F971F415058F1FC01E40FF11D50812E
:10CE10005523C1F3220F331F4091B7055091B80538
:10CE2000240F351FF901D182C08228E0F301DC0113
:10CE300001900D922A95E1F7DC018C91883231F452
:10CE400080918606909187060E944B228091BF05B3
:10CE50009091C00501969093C0058093BF05F7019E
:10CE6000E280F38062CF88E890E00E9411C4909342
:10CE7000BE058093BD056AE070E187E799E00E94F6
:10CE80000C820E94BF26AB01BC0187E799E00E949B
:10CE9000C49787E799E00E94158182E290E00E94A2
:10CEA00011C49093B8058093B7056DEF7FE087E7D5
:10CEB00099E00E940C820E94BF26AB01BC0187E76B
:10CEC00099E00E94C49787E799E00E9415818091BC
:10CED000BD059091BE05892B31F08091B7059091E9
:10CEE000B805892B79F465EE7FE080ED98E00E942B
:10CEF0000C820E94BF26AB01BC0180ED98E00E942D
:10CF0000C49706CF8AEB90E59093BA058093B90554
:10CF100010926506109264061092E10710920308C1
:10CF20000E94A915B0923E06A0923D06D0924206FC
:10CF3000C092410680918606909187060E948711D3
:10CF400081E00E94869F811130C062ED7FE087E71B
:10CF500099E00E9430820091860610918706C801F0
:10CF60000E94871140E060EFC8010E9457220E9492
:10CF700076A0E0918606F091870681E0808362EBDF
:10CF80007FE087E799E00E94308280918606909149
:10CF900087060E940A22882309F461CE66EA7FE0B0
:10CFA00087E799E00E9430825ACE68E97FE087E700
:10CFB00099E00E943082B0CE1092B3051092B20573
:10CFC000E0919906F0919A06309709F4F8C0E6804E
:10CFD000F7800091990610919A060115110509F440
:10CFE000E7C0E114F10409F4E3C0D70118968C916D
:10CFF0008770853091F7C7010E94D697823068F319
:10D00000B701CE0101960E94A51CCE0101960E9497
:10D010002B13882309F466C08A859B85009759F5F0
:10D02000CE0101960E94E6978C01912C812C97FFEE
:10D0300006C011950195110988248394912CCE0185
:10D0400001960E94EB18C82ED12C8985853009F4F1
:10D0500052C0863009F046C0B02E61E0802F0E9499
:10D06000089F61E0892809F481C0CA94CD2809F09D
:10D0700081C060E07FC0DC01ED91FC910484F58506
:10D08000E02D1995892B49F08A859B85DC01ED916E
:10D09000FC910284F385E02D19958A859B85DC013E
:10D0A000ED91FC910680F781E02D1995892BD1F047
:10D0B000CE0101960E94EB18882341F040E051E038
:10D0C00060E070E0CE0101960E94873A8D819E81DA
:10D0D000892B41F040E052E060E070E0CE01019623
:10D0E0000E94873AD7011296ED90FC90CE010196EE
:10D0F0000E9461136ECFCD2829F462E0CE01019623
:10D100000E94BC1840E051E060E070E0CE01019662
:10D110000E94873A8D819E81892B41F040E052E048
:10D1200060E070E0CE0101960E94873A61E0802FB6
:10D130000E94089F60E0802F0E94DA9E6FE570E1F8
:10D1400087E799E00E940C82B80187E799E00E9486
:10D15000CE976AE570E187E799E00E940C8268E566
:10D1600070E187E799E00E940C82BCCFCA94CD2879
:10D1700009F07FCFC62ED12C8B2D0E94DA9E63E55D
:10D1800070E187E799E00E940C82B80187E799E097
:10D190000E94CE9761E570E187E799E00E940C82DA
:10D1A000B60187E799E00E94CE976FE470E1D9CF8E
:10D1B000F801868197819093B3058093B20587E744
:10D1C00099E00E941581E091AE05F091AF0530978E
:10D1D00009F48AC080918D068F5F80938D06068149
:10D1E00017810115110509F47AC0D80118968C91A0
:10D1F0008770863009F069C01F8F0E8F70E060E085
:10D20000CE014E960E94BB1C8AA19BA1892B09F4DA
:10D210005CC08091B0059091B105892B09F455C08F
:10D22000EE8CFF8CF70180858770863099F56AE077
:10D2300074E0C7010E9427930097F1F0DC01189673
:10D240002C91189727702530B9F41696CD90DC9064
:10D25000C114D104F9F0DA82C982B701CE01019676
:10D260000E94BB1CED81FE8110821182128213820A
:10D27000F601C280D380ECCFFA82E98270E060E0F0
:10D28000CE0101960E94BB1C62E070E0CE010196C7
:10D290000E94DA5BEAA1FBA1108211821282138242
:10D2A00088A1843068F462E0823008F060E089A1EF
:10D2B0000E94089FEAA1FBA18181807F818305C034
:10D2C000803441F060E0823431F0D80112960D9143
:10D2D0001C9187CF62E089A10E94089FF6CF8091C0
:10D2E0008D06815080938D066FE77FE086EC98E095
:10D2F0000E940C8267E77FE086EC98E00E940C8237
:10D3000081E02091990630919A06232B09F480E060
:10D310000E94C7156EE67FE086EC98E00E940C82C2
:10D3200081E02091AE053091AF05232B09F480E018
:10D330000E94C71567E67FE086EC98E00E940C82A9
:10D3400081E020918A0630918B06232B09F480E03E
:10D350000E94C7156EE57FE086EC98E00E940C8283
:10D3600081E020919B0630919C06232B09F480E0FC
:10D370000E94C71565E57FE086EC98E00E940C826C
:10D38000809119060E94C71586EC98E00E941581CD
:10D3900060E57FE086EC98E00E940C820E94BF2648
:10D3A000AB01BC0186EC98E00E94C49786EC98E043
:10D3B0000E94158181E080938E0685E998E00E94A5
:10D3C000631E882351F085E998E00E94081F84E0DD
:10D3D00090E090939806809397068091970690919D
:10D3E0009806079731F484E090E090939806809334
:10D3F000970680918D06815080938D06A3960FB677
:10D40000F894DEBF0FBECDBFDF91CF911F910F917A
:10D41000FF90EF90DF90CF90BF90AF909F908F9054
:10D420007F906F905F900895CF93DF93EC01FB01A5
:10D430002481358140815181628173810E942081E4
:10D44000CE01DF91CF910895AF92BF92CF92DF923C
:10D45000EF92FF921F93CF93DF9300D000D0CDB710
:10D46000DEB76C017C0110E08AE0A82EB12C1330ED
:10D4700061F1F701828190E0B0E0A0E089839A83B6
:10D48000AB83BC83BE82AD82BE016F5F7F4F86ECF3
:10D4900098E00E94146A60ED76E10E940C821F5FA2
:10D4A000FFEFEF1AFF0A143011F726960FB6F89423
:10D4B000DEBF0FBECDBFDF91CF911F91FF90EF90E8
:10D4C000DF90CF90BF90AF900895F601858190E0F6
:10D4D000B0E0A0E089839A83AB83BC83BE82AD8237
:10D4E000BE016F5F7F4F86EC98E00E94146A6EEC7D
:10D4F00076E1D3CF0F931F93CF93DF9300D000D06B
:10D50000CDB7DEB70E94E02B67EC7CE086EC98E0BC
:10D510000E940C82CE0101960E94E89CCE010196E9
:10D520000E94246A0DEA13E01A830983809133086C
:10D5300090913408A0913508B09136088B839C8374
:10D54000AD83BE83CE0101960E94246A1A830983AB
:10D550001B821C821D821E8280E590E00E94E59C59
:10D5600044E050E0BE016D5F7F4F81E090E00E949B
:10D570002687CE0101960E94246A1A8309831B82A2
:10D580001C821D821E8280E590E00E94E59C44E0A2
:10D5900050E0BE016D5F7F4F85E090E00E942687DE
:10D5A000CE0101960E94246A6DEE7CE086EC98E044
:10D5B0000E940C8288EC90E026960FB6F894DEBFAD
:10D5C0000FBECDBFDF91CF911F910F910895CF92E4
:10D5D000DF92EF92FF921F93CF93DF9300D000D0A2
:10D5E000CDB7DEB763E97CE086EC98E00E940C8260
:10D5F0008AEAE82E88E0F82E10E090E1C92ED12CBE
:10D60000F70181917F01803130F46EEA74E086EC9D
:10D6100098E00E94A681153041F1F7013197808191
:10D6200090E0B0E0A0E089839A83AB83BC83DE8284
:10D63000CD82BE016F5F7F4F86EC98E00E94146A36
:10D6400061E97CE00E940C821F5F1630C9F62696C5
:10D650000FB6F894DEBF0FBECDBFDF91CF911F9103
:10D66000FF90EF90DF90CF9008958091AF0890E009
:10D67000B0E0A0E089839A83AB83BC83DE82CD8255
:10D68000BE016F5F7F4F86EC98E00E94146A0E9493
:10D690001581DACFEF92FF920F931F93CF93DF9311
:10D6A00000D000D01F92CDB7DEB77B01CE01079628
:10D6B0009F938F9301979F938F9301979F938F933E
:10D6C00001979F938F9301979F938F9301979F93B8
:10D6D0008F938E010F5F1F4F1F930F9380EB94E08A
:10D6E0009F938F93DB0113968C9113978F931296D0
:10D6F0008C918F930E942AD30FB6F894DEBF0FBE91
:10D70000CDBF0697ECF46BE771E180ED98E00E94E5
:10D710000C82D70112966D917C9180ED98E00E9469
:10D72000A68180E991E027960FB6F894DEBF0FBE80
:10D73000CDBFDF91CF911F910F91FF90EF90089592
:10D740008091A2089091A308892BA9F10E94899445
:10D75000882389F182E70E9474948091A2089091B5
:10D76000A308DC01ED91FC910088F189E02D64E0D3
:10D7700070E019958091A2089091A308DC01ED91C9
:10D78000FC910280F381E02D46E050E0B80119954C
:10D7900086E0F801AAEAB8E001900D928A95E1F7D7
:10D7A0008091A2089091A308DC01ED91FC9104887E
:10D7B000F589E02D19950E94E76A6DE871E186EC24
:10D7C00098E00E940C8288EC90E0ADCFAF92BF92BF
:10D7D000DF92EF92FF920F931F93CF93DF9300D0CE
:10D7E00000D0CDB7DEB78C017B01D42EFB01848144
:10D7F0009581892BF9F0A080B1806FE370E0C501BD
:10D800000E946AD20097B1F09C012A193B0937FDAA
:10D8100011C050E040E0B701CE0101960E941E8089
:10D82000BE016F5F7F4FC7010E94D47ECE0101967B
:10D830000E94CE7F64EC74E0C7010E944F7E882373
:10D8400021F1F801128A118A80E090E1958784879E
:10D8500084E890E0948B838B81E0868780E090E27F
:10D86000908B8787D58A81E090E026960FB6F89452
:10D87000DEBF0FBECDBFDF91CF911F910F91FF9003
:10D88000EF90DF90BF90AF90089561ED74E0C70115
:10D890000E944F7E882369F0F801128A118A148A47
:10D8A000138A84E890E095878487168680E090E369
:10D8B000D7CF90E080E0D9CFEF92FF920F931F93E4
:10D8C000CF93DF9300D000D0CDB7DEB78091A20810
:10D8D0009091A308892B09F46CC087E70E94749487
:10D8E0008091A2089091A308DC01ED91FC91008841
:10D8F000F189E02D70E060E0199510E000E0809182
:10D90000A2089091A308DC01ED91FC9111971C965F
:10D910002D913C910217130740F40190F081E02D06
:10D9200060E019950F5F1F4FEACF0088F189E02D65
:10D9300070E060E0199506EC12E08AECE82E82E0D7
:10D94000F82E8091A2089091A308F80161918F01AF
:10D95000DC01ED91FC910190F081E02D1995E0162C
:10D96000F10679F78091A2089091A308DC01ED916E
:10D97000FC910488F589E02D19956AE275E0CE01E5
:10D9800001960E940D80CE0101960E94E0A8CE0172
:10D9900001960E94CE7F87E090E00E94909787E0FA
:10D9A00090E00E949A976EE371E186EC98E00E9405
:10D9B0000C821092C2081092C10880E090E190930E
:10D9C000BD088093BC0884E890E09093C4088093DD
:10D9D000C30881E08093BE0880E090E29093C00885
:10D9E0008093BF0882E78093C50880EB98E00E948F
:10D9F000AB1380EB98E00E94E71588EC90E0269648
:10DA00000FB6F894DEBF0FBECDBFDF91CF911F914F
:10DA10000F91FF90EF900895CF93DF93CDB7DEB7CE
:10DA20002E970FB6F894DEBF0FBECDBF80918D0646
:10DA3000811178C062ED70E186EC98E00E940C8262
:10DA400086EC98E00E9415811092C2081092C108DD
:10DA500080E090E19093BD088093BC0884E890E05A
:10DA60009093C4088093C30881E08093BE0880E04F
:10DA700090E29093C0088093BF0882E78093C50826
:10DA800080EB98E00E946B1D8B37910509F0B9C0BF
:10DA900064EC70E187E799E00E940C8287E799E0E7
:10DAA0000E9415811C821B828FE792E09A838983F2
:10DAB00080EB98E09E838D838FEF9FEF98878F8315
:10DAC0008091B0059091B105892B11F00E94BC6343
:10DAD000CE0101960E94C79C9093B1058093B0053A
:10DAE00080EB98E00E94E7158091B0059091B10518
:10DAF000892BD9F468EB70E180ED98E00E940C82EC
:10DB000080ED98E00E9415816AE275E0CE010996E9
:10DB10000E940D80CE0109960E94E0A8CE010996D0
:10DB20000E94CE7F90E080E014C065EA70E186EC50
:10DB300098E00E940C8286EC98E00E9415810E9479
:10DB4000B7658091A2089091A308892B59F481E0D0
:10DB500090E02E960FB6F894DEBF0FBECDBFDF91DA
:10DB6000CF9108950E948994882389F382E70E94C7
:10DB700074948091A2089091A308DC01ED91FC912E
:10DB80000088F189E02D60E670E019956091A208A7
:10DB90007091A30840E0CE0109960E949280BE01D8
:10DBA000675F7F4F84EA98E00E94D47ECE01099699
:10DBB0000E94CE7F8091A2089091A308DC01ED9194
:10DBC000FC910488F589E02D199567E870E187E7F5
:10DBD00099E00E940C8264EA78E0CE0109960E94E6
:10DBE0000480BE01675F7F4F87E799E00E94FE8156
:10DBF00087E799E00E941581CE0109960E94CE7FA9
:10DC0000A6CF80EB98E00E948113892BA1F080EBD6
:10DC100098E00E94AB136AE275E0CE0101960E9483
:10DC20000D80CE0101960E94E0A8CE0101960E94CF
:10DC3000CE7F0E944FA980EB98E00E94E71564E92F
:10DC400070E186EC98E00E940C8286EC98E00E94DD
:10DC5000158168CF0E940C6D892B49F486EF9FEFE8
:10DC6000909398068093970684EF91E0089588EC4E
:10DC700090E00895FF920F931F93CF93DF9300D00E
:10DC800000D0CDB7DEB78C01BC01CE0101960E9459
:10DC90000480BE016F5F7F4F87E799E00E94FE819D
:10DCA00087E799E00E941581CE0101960E94CE7F00
:10DCB00060EF71E1CE0101960E94D67FBE016F5FD9
:10DCC0007F4FC8010E94347EF82ECE0101960E943B
:10DCD000CE7FFF2069F0B801CE0101960E9404803A
:10DCE000CE0101960E94E0A8CE0101960E94CE7F4F
:10DCF00026960FB6F894DEBF0FBECDBFDF91CF9151
:10DD00001F910F91FF9008955F926F927F928F9273
:10DD10009F92AF92BF92CF92DF92EF92FF920F93BA
:10DD20001F93CF93DF93CDB7DEB7CF56D1090FB690
:10DD3000F894DEBF0FBECDBF4C018B01F42E642FD3
:10DD400087E799E00E94C79765E27CE087E799E062
:10DD50000E940C82B801CE0101965C010E940480F1
:10DD6000B50187E799E00E94FE8187E799E00E946C
:10DD70001581C5010E94CE7F92E0F9126BC263E269
:10DD80007CE0C5010E94D67FB501C8010E94647E77
:10DD9000F82EC5010E94CE7FFF2009F4D0C220E0FA
:10DDA0004DE251E0B40183E798E00E94B882E09030
:10DDB0008806F09089066CE17CE0CE0186599F4F81
:10DDC0000E94D67F65E17CE0CE018C599F4F0E9476
:10DDD000D67FCE01885A9F4F0E94E89C6E961FAD59
:10DDE0006E976D960FAD6D976C96DFAC6C976B96DA
:10DDF000CFAC6B976AE275E0CE0181960E940D80F0
:10DE0000BE016F5D7F4FC5010E9404806C2DC5016E
:10DE10000E941F7F6DED74E00E94507F6D2D0E9467
:10DE20001F7F6DED74E00E94507F602F0E941F7F66
:10DE30006DED74E00E94507F612F0E941F7FBC0136
:10DE4000CE01825A9F4F0E940480C5010E94CE7F5E
:10DE5000CE0181960E94CE7F60E17CE0CE018E5A99
:10DE60009F4F0E94D67F6AE275E0CE01845B9F4F90
:10DE70000E940D8002EA18E0D80118966C9170E0BB
:10DE800084E0759567958A95E1F7C5010E944894ED
:10DE90004D815E8169817A81CE01845B9F4F0E94B2
:10DEA000947EC5010E94CE7FF80160856F7070E09E
:10DEB000C5010E9448944D815E8169817A81CE01BD
:10DEC000845B9F4F0E94947EC5010E94CE7F0F5FAE
:10DED0001F4FF8E0083A1F0779F66AE07CE0CE01B0
:10DEE0008A5B9F4F0E94D67F69EE7BE0CE018196D0
:10DEF0000E94D67FBE016F5D7F4FCE01CE960E94FD
:10DF00000480BE016A5B7F4FCE01CE960E946A7F7D
:10DF1000BE01645B7F4F0E946A7FBE016E5A7F4FD5
:10DF20000E946A7FBE01625A7F4F0E946A7FBE01D3
:10DF30006C597F4F0E946A7F8C014AE0B50180E5F1
:10DF400090E00E94C6C6F50101900020E9F73197E4
:10DF5000AF014A195B09B501C8010E94947E811185
:10DF600003C0C8010E940D7FBE0166597F4FC801E2
:10DF70000E946A7FB7010E94507FBC01C4010E94C9
:10DF8000FE81C4010E941581CE01CE960E94CE7FF3
:10DF9000CE0181960E94CE7FCE018A5B9F4F0E9468
:10DFA000CE7FCE01845B9F4F0E94CE7FCE018E5AE2
:10DFB0009F4F0E94CE7FCE01825A9F4F0E94CE7FFC
:10DFC000CE018C599F4F0E94CE7FCE0186599F4F24
:10DFD0000E94CE7FC4010E94158164E670E080E05B
:10DFE00090E00E9479A0D401ED91FC910488F5891C
:10DFF000E02DC401199501E010E088C028966EADAF
:10E000007FAD2897CE0181960E949B98892B09F4B9
:10E0100050C122961CAE1DAE1EAE1FAE2297269694
:10E020001CAE1DAE1EAE1FAE26978FAD8F708FAF8C
:10E0300040E053E0BE016F5D7F4FCE01CE960E945F
:10E04000A43000E020E033E040E250E0B501CE0132
:10E05000CE960E94812DBC01C6010E94A87F08ECCB
:10E0600010E129C1EE2009F4F3C046E050E070E071
:10E0700060E0C8010E94D17DD8016D917C91CE01F4
:10E0800081960E948938CE0181960E942B1300E967
:10E0900011E08823B9F189A5873061F4CE0181961A
:10E0A0000E940F5761E0892B09F462E0CE0181964E
:10E0B0000E94BC1822961CAE1DAE1EAE1FAE22974B
:10E0C00026961CAE1DAE1EAE1FAE26978FAD8F706E
:10E0D0008FAF40E053E0BE016F5D7F4FCE01CE9623
:10E0E0000E94A43000E020E033E040E250E0B501BF
:10E0F000CE01CE960E94812DBC01C6010E94A87F50
:10E1000008EC10E1CE0181960E946113C801C1594B
:10E11000DF4F0FB6F894DEBF0FBECDBFDF91CF91BA
:10E120001F910F91FF90EF90DF90CF90BF90AF9035
:10E130009F908F907F906F905F900895F80160811D
:10E1400071810E9427937C01892B09F040C104E969
:10E1500011E0DCCFEE2009F47BC049E050E070E034
:10E1600060E0C8010E94D17D4AE0B401C5010E946F
:10E17000928041E050E06FEC73E0C8010E94947E11
:10E180004D815E8169817A81C8010E94947E65EC2F
:10E190007BE087E799E00E940C82B801CE0181966E
:10E1A0000E940480BE016F5D7F4F87E799E00E9467
:10E1B000FE8187E799E00E941581CE0181960E9439
:10E1C000CE7F6DEB7BE0CE0181960E94D67FF80179
:10E1D000848195812DA13EA182179307E1F4892BBB
:10E1E000A1F1E080F18069A07AA0D7018D917D0135
:10E1F000882359F1082E000C990B0E94FAD16C016A
:10E20000F30181913F01082E000C990B0E94FAD175
:10E21000C816D90651F3CE0181960E94CE7F5520B3
:10E2200041F021E048EC50E0B40183E798E00E941F
:10E23000B882D8018D919C910E94E682009711F4DA
:10E2400084E991E08C01C5013DC055245394E3CF8E
:10E2500001E97ECFB1E0FB1270C062EE7BE0C50148
:10E260000E94D67FB501C8010E94347E582EC50198
:10E270000E94CE7F552049F1EE2051F346E050E058
:10E2800070E060E0C8010E94D17D4AE0B401CE0197
:10E290008A5B9F4F0E949280F80160817181CE015C
:10E2A00081960E948938CE0181960E942B1381119C
:10E2B000A5CE00E911E0CE0181960E946113CE0146
:10E2C0008A5B9F4F0E94CE7F21CF6BEC7BE0C50124
:10E2D0000E94D67FB501C8010E94347EF82EC50188
:10E2E0000E94CE7FF11036CF60EB7BE0C5010E942B
:10E2F000D67FB501C8010E94347E182FC5010E9447
:10E30000CE7F00E0112309F401CF80E00E948697C0
:10E3100068E87BE086EC98E00E940C8286EC98E04E
:10E320000E9415816AE275E0C5010E940D80C50159
:10E330000E94E0A8C5010E94CE7F00E05DCE6BED9B
:10E340007BE0C5010E94D67FB501C8010E94347EE2
:10E35000F82EC5010E94CE7FF11084CE65ED7BE0E2
:10E36000C5010E94D67FB501C8010E94347EF82EF7
:10E37000C5010E94CE7FFF2001F3EE2009F468CF93
:10E3800045E050E070E060E0C8010E94D17D6DED95
:10E3900074E0C8010E944F7E882339F0E09099060E
:10E3A000F0909A06E114F10491F46AE275E0C80174
:10E3B0000E944F7E811107C08091990690919A0624
:10E3C000009709F0BBCEE090B005F090B10520E0D9
:10E3D00048EC50E2B40183E798E00E94B882C4019F
:10E3E0000E9415811C821B828FE792E09A838983A9
:10E3F0009E828D828FEF9FEF98878F83B701C50133
:10E400000E940F84EACD4F925F926F927F928F921B
:10E410009F92AF92BF92CF92DF92EF92FF920F93B3
:10E420001F93CF93DF93CDB7DEB7C659D1090FB68F
:10E43000F894DEBF0FBECDBF8E010F5B1F4FD8011A
:10E440001D921C92FE01ED5BFF4F8EE1DF011D92DC
:10E450008A95E9F78091A2089091A308892B09F485
:10E46000CAC10E948994882309F4C5C182E70E9429
:10E4700074948091A2089091A308DC01ED91FC9125
:10E480000088F189E02D60E270E019954FE150E0DD
:10E49000B8018091A2089091A3080E94CE947C01BB
:10E4A0008091A2089091A308DC01ED91FC91048871
:10E4B000F589E02D1995E114F10409F49CC1F801E6
:10E4C000EE0DFF1D10828091AF081F928F938091F7
:10E4D000AE081F928F938091AD081F928F93809109
:10E4E000AC081F928F938091AB081F928F938091FD
:10E4F000AA081F928F938FED94E09F938F931F92A2
:10E5000080E48F93FE0131966F01FF93EF930E9499
:10E51000BDD263ED72E186EC98E00E940C82B801F6
:10E5200086EC98E00E94A681B60186EC98E00E94F5
:10E53000A68186EC98E00E9415817E01F1E6EF0E3F
:10E54000F11CD70113961C921E92129788EE93E04D
:10E55000A0E0B0E0F70184839583A683B78384E0CD
:10E56000848785E393E09183808316861586108BDC
:10E570000787128A118A80E590E0948B838B178A33
:10E5800067EF71E187E799E00E940C8264EA78E026
:10E59000CE0187589F4F0E940480BE0167587F4F6D
:10E5A00087E799E00E94FE8187E799E00E94158144
:10E5B000CE0187589F4F0E94CE7F6EE075E0CE015E
:10E5C00085579F4F0E940D806EE075E0CE01875801
:10E5D0009F4F0E940D80BE0167587F4FCE018D571F
:10E5E0009F4F0E94048064EA78E0CE018D579F4FD0
:10E5F0000E946A7FBE0165577F4F0E946A7FBC01FF
:10E60000CE018F569F4F0E940480CE018D579F4FA1
:10E610000E94CE7FCE0187589F4F0E94CE7FCE01B1
:10E6200085579F4F0E94CE7F80E195E0CD57DF4F09
:10E6300099838883C358D040C957DF4F1982188205
:10E64000C758D040C757DF4F19821882C958D040E9
:10E65000CF56DF4F88819981C159D040CB57DF4FCA
:10E6600099838883C558D0406DEC72E187E799E0C3
:10E670000E940C820E94BF26AB01BC0187E799E093
:10E680000E94C49787E799E00E94158164E670E0D4
:10E6900080E090E00E9479A08AE39EE6D7011E9672
:10E6A0009C938E931D976CEC7AE782E596E80E9426
:10E6B00054C78C010FB6F894DEBF0FBECDBF892BB7
:10E6C00009F4F4C083E090E00E9411C4D8011D96C3
:10E6D0009C938E931C97FC01F182E0821282C70109
:10E6E0000E94631E882319F0C7010E94081FD701EA
:10E6F00051966D917C9152975396AD90BC90611557
:10E70000710509F48FC0CE0187589F4F0E944C823B
:10E71000A501BE0167587F4FC7010E94FD6418160E
:10E7200019060CF0C0C0D7011F96BC901F975096D9
:10E73000AC90DF92CF9282E592E19F938F931F93EB
:10E740000F930E94DBC7DF92CF928DE492E19F93FB
:10E750008F931F930F930E94DBC7D8011C96ED91F6
:10E76000FC9181E08283DF92CF928AE492E19F93D1
:10E770008F931F930F930E94DBC7D8011C96ED91D6
:10E78000FC911282AF92BF9284E192E19F938F93AA
:10E790001F930F930E94DBC70FB6F894DEBF0FBE26
:10E7A000CDBFB12C8BE0C82E82E1D82E8B2D94E00A
:10E7B0008902F0011124A3E8B0E0AC0FBD1FEA0FFD
:10E7C000FB1F808191810097A9F12281338121155E
:10E7D0003105C9F33F932F939F938F93DF92CF928D
:10E7E0001F930F930E94DBC7B3940FB6F894DEBF5C
:10E7F0000FBECDBFDBCF40E250E065E073E1C80162
:10E800000E9481C667EE72E186EC98E00E940C825D
:10E81000B80186EC98E00E94A68186EC98E00E9400
:10E82000158151CEF70167857089A501C7010E9446
:10E830007B1475CF8FE492E19F938F931F930F9377
:10E840000E94DBC7D70156961C921E925597D8019D
:10E850001C96ED91FC91C080D1800F900F900F908D
:10E860000F9033E3A32EB12CD601ED91FC910084DF
:10E87000F185E02DC601199541975CF4B1E0AB1A22
:10E88000B10839F064E170E080E090E00E9479A086
:10E89000EBCFD601ED91FC910084F185E02DC6010E
:10E8A0001995419734F4C8010E942B8610E000E0CE
:10E8B0005AC06AE275E0CE0185579F4F0E940D80D5
:10E8C000912CA12CD601ED91FC910688F789E02DC1
:10E8D000C60119958823E1F1BDE0AB1201C0A92C56
:10E8E000D601ED91FC910688F789E02DC6011995B6
:10E8F0008111D7C0D601ED91FC910084F185E02D06
:10E90000C6011995892B09F4DEC0D601ED91FC9161
:10E910000284F385E02DC6011995B82EBAE08B1755
:10E9200009F4D3C0EDE08E1709F4CFC0FFEF8F17C5
:10E9300009F4C9C0682FCE0185579F4F0E94C07E41
:10E940009A2CAB2CBFCFBAE0BB12FACFAB12F8CFE8
:10E95000CC24C394D12CCE0185579F4F0E94CE7FEB
:10E96000CD2809F4A3CFD7015596ED90FC906FEB1D
:10E9700072E187E799E00E940C82B70187E799E08E
:10E980000E94CE9787E799E00E94158164E670E0C7
:10E9900080E090E00E9479A00115110509F454C1AE
:10E9A000B8ECEB16F10409F02DC163EB72E186ECD3
:10E9B00098E00E940C8264EF71E080E090E00E9499
:10E9C00079A0ED961FAE1EAEED97EF961FAE1EAE70
:10E9D000EF978FEF9FEFC158DF4F99838883CF5711
:10E9E000D04089E692E0EB969FAF8EAFEB97CF5782
:10E9F000DF4F19830883C158D040F8948091B00547
:10EA00009091B105892B11F00E94BC63CE0187580B
:10EA10009F4F0E94C79C9093B1058093B005789456
:10EA2000C8010E942B868091B0059091B105892B79
:10EA300009F0D6C06AE275E0CE0185579F4F0E946B
:10EA40000D80CE0185579F4F0E94E0A8CE018557CB
:10EA50009F4F0E94CE7F6CE972E180ED98E00E94AA
:10EA60000C82F12CE12CCE018F569F4F0E94CE7F5D
:10EA7000C701CA56DF4F0FB6F894DEBF0FBECDBF39
:10EA8000DF91CF911F910F91FF90EF90DF90CF908A
:10EA9000BF90AF909F908F907F906F905F904F90BE
:10EAA0000895D601ED91FC910084F185E02DC60119
:10EAB0001995892B09F01ECF64E670E080E090E0A4
:10EAC0000E9479A00DCFBB24BA946EE175E08AED67
:10EAD00098E00E94A681BE0165577F4F8AED98E0BD
:10EAE0000E94FE818AED98E00E94158162E072E149
:10EAF000CE0187589F4F0E94D67FBE0167587F4F37
:10EB0000CE0185579F4F0E94347E982ECE018758A4
:10EB10009F4F0E94CE7F992099F1C157DF4F2881E6
:10EB20003981CF58D04049E050E0BE0165577F4F52
:10EB3000CE0187589F4F0E941E80EB968EAD9FADF1
:10EB4000EB97412C512C3201009719F00E94FCC523
:10EB50002B014201CE0187589F4F0E94CE7F411466
:10EB6000510429F0D70156965C924E925597B40104
:10EB70008AED98E00E94CE978AED98E00E94158178
:10EB8000F7018584968481149104D1F0C157DF4F39
:10EB900088819981CF58D040892B91F0BE0165576B
:10EBA0007F4FCE0187589F4F0E940480CE01875827
:10EBB0009F4FF4011995CE0187589F4F0E94CE7F39
:10EBC0006AE275E0CE0185579F4F0E949E7FFFEF5E
:10EBD000BF12B9CEC8010E942B86D12CC12CBBCE4E
:10EBE0000E94B76580918E06882329F00E94E896DE
:10EBF00067FF0E943C1865E972E186EC98E00E948C
:10EC00000C8231CFE0E3EE16E1E0FE0651F461E85C
:10EC100072E186EC98E00E940C82C8010E942B866B
:10EC200022CF69E672E180ED98E00E940C82C80173
:10EC30000E942B86B70180ED98E00E94CE9780ED70
:10EC400098E00E9415810FCF66E572E187E799E0B1
:10EC50000E940C82EE24EA94FE2C05CF0F931F93A2
:10EC6000CF93DF93EB0102970CF485C00A811B81DF
:10EC700069EE71E1C8010E942CC6892B51F481E034
:10EC80000E94869788EC90E0DF91CF911F910F91C1
:10EC9000089565EE71E1C8010E942CC6892B11F41C
:10ECA00080E0EECF65EC71E186EC98E00E940C828A
:10ECB0000E94E89663FB662760F981E0682770E0B0
:10ECC00086EC98E00E94CE9786EC98E00E94158131
:10ECD0008091A2089091A308892BE9F10A811B81F8
:10ECE0000E9489948823B9F1F80101900020E9F786
:10ECF0003197E01BF10BB09770F582E70E94749496
:10ED00008091A2089091A308DC01ED91FC9100880C
:10ED1000F189E02D60E270E01995B8018091A208B8
:10ED20009091A3080E94A6818091A2089091A308C7
:10ED3000DC01ED91FC910190F081E02D60E01995EE
:10ED40008091A2089091A308DC01ED91FC910488C8
:10ED5000F589E02D19956A817B8186EC98E00E9407
:10ED6000A6816EEB71E186EC98E00E940C8286EC45
:10ED700098E00E94158180919706909198060297DD
:10ED80007CF10E940372883C910539F424E030E064
:10ED9000309398062093970677CF8F3F9807C9F452
:10EDA00063EA71E187E799E00E940C8287E799E0C6
:10EDB0000E94158110928C0683E090E09093980653
:10EDC0008093970685E998E00E94081F89EC90E0FF
:10EDD0005BCF20918E062111D9CF2FE030E0D8CF24
:10EDE00066E971E180ED98E00E940C8280ED98E088
:10EDF0000E94158184EF91E047CF0895FC012481A2
:10EE000035816217730748F480819181009729F05A
:10EE1000860F971FFC018081089580E00895089572
:10EE2000AF92BF92CF92DF92EF92FF920F931F9318
:10EE3000CF93DF936C017B018B01040F151FEB0156
:10EE40005E01AE18BF08C017D10759F06991D6010D
:10EE5000ED91FC910190F081E02DC6011995892B6F
:10EE600079F7C501DF91CF911F910F91FF90EF903E
:10EE7000DF90CF90BF90AF900895FC01538D448DEB
:10EE8000252F30E0842F90E0821B930B541710F055
:10EE9000CF96089501970895FC01918D828D981762
:10EEA00061F0A28DAE0FBF2FB11D5D968C91928D3A
:10EEB0009F5F9F73928F90E008958FEF9FEF08956B
:10EEC000FC01918D828D981731F0828DE80FF11D34
:10EED000858D90E008958FEF9FEF0895FC01918D4F
:10EEE000228D892F90E0805C9F4F821B91098F7348
:10EEF000992708958AED98E00E946E7721E0892B8A
:10EF000009F420E0822F0895FC01A48DA80FB92FE9
:10EF1000B11DA35ABF4F2C91848D90E001968F7341
:10EF20009927848FA689B7892C93A089B1898C9160
:10EF3000837080648C93938D848D981306C00288AF
:10EF4000F389E02D80818F7D80830895EF92FF9279
:10EF50000F931F93CF93DF93EC0181E0888F9B8DFC
:10EF60008C8D98131AC0E889F989808185FF15C0B6
:10EF70009FB7F894EE89FF896083E889F9898081D9
:10EF80008370806480839FBF81E090E0DF91CF91A8
:10EF90001F910F91FF90EF900895F62E0B8D10E0CA
:10EFA0000F5F1F4F0F731127E02E8C8D8E110CC039
:10EFB0000FB607FCFACFE889F989808185FFF5CF84
:10EFC000CE010E948477F1CFEB8DEC0FFD2FF11D68
:10EFD000E35AFF4FF0829FB7F8940B8FEA89FB89C1
:10EFE00080818062CFCFCF93DF93EC01888D88231F
:10EFF000B9F0AA89BB89E889F9898C9185FD03C09C
:10F00000808186FD0DC00FB607FCF7CF8C9185FF80
:10F01000F2CF808185FFEDCFCE010E948477E9CFCA
:10F02000DF91CF91089580E090E0892B29F00E9434
:10F030007A7781110E94000080E090E0892B49F0EE
:10F0400080E090E0892B29F00E94000081110E944D
:10F05000000080E090E0892B49F080E090E0892B6F
:10F0600029F00E94000081110E94000080E090E0E1
:10F07000892B49F080E090E0892B29F00E94000064
:10F0800081110C94000008950F931F93FC01628579
:10F090007385848595850281138124813581601B68
:10F0A000710B820B930B0685178520893189601BB4
:10F0B000710B820B930B1F910F910895DC01ED9161
:10F0C000FC910190F081E02D19948FEF9FEF08954E
:10F0D000FC0162897389848995890895EF920F9361
:10F0E0001F93CF93DF93FC01248D222341F0213025
:10F0F00051F1DF91CF911F910F91EF9008952289E7
:10F1000033894489558986899789A08DB18D821B61
:10F11000930BA40BB50B892F9A2FAB2FBB278C0118
:10F120000F5F1F4F6281738184819581CFB7F894FF
:10F13000DCB7E1E0ECBFEE24E394E2E0FEEF1995EA
:10F14000DCBFCFBFD6CFF0E0E0E0DF91CF911F91E1
:10F150000F91EF901994FC01138E128E41110CC087
:10F1600082899389A489B589868B978BA08FB18F6B
:10F17000148E81E090E0089590E080E00895CF92B1
:10F18000DF92EF92FF92CF93DF93DC01CB01642FEC
:10F19000CFB7F8946D01EE24FF24CBBEDCB741E07D
:10F1A0004CBFA901E1E0FEEF1995DCBFCFBFDF91B5
:10F1B000CF91FF90EF90DF90CF900895CF93DF93A2
:10F1C000FC01248D211110C0EC01828D938D892BBF
:10F1D00049F066897789808D918D30E020E045E0A7
:10F1E0000E94BF781B8E1A8EDF91CF9108951F93D6
:10F1F000CF93DF93FC01248D211145C0162FEC0124
:10F20000828D938D892B49F466897789808D918DC4
:10F2100030E020E043E00E94BF784A8D5B8DCA0158
:10F2200081709927FE01E80FF91F158F892B69F06E
:10F230002D8D3E8D6E897F89888D998D640F751F08
:10F24000811D911D41E00E94BF788A8D9B8D0196A2
:10F250009B8F8A8F81159140B1F46E897F89888D4B
:10F26000998D30E020E045E00E94BF781B8E1A8E19
:10F270008E899F89A88DB98D9F5FAF4FBF4F8E8BB1
:10F280009F8BA88FB98F81E090E0DF91CF911F9184
:10F290000895DC01ED91FC910280F381E02D40E0C6
:10F2A0001994FB0144815581228133812150310918
:10F2B0004217530750F4A081B181A40FB51F8C935E
:10F2C0008481958101969583848380E00895CF930E
:10F2D000DF93EC01E881F9810284F385E02DCE0112
:10F2E00019950196B9F7DF91CF910895CF92DF92EA
:10F2F000EF92FF920F931F93CF93DF937C016A01EC
:10F300008B01D0E0C0E0CC15DD0581F0D701ED9197
:10F31000FC910284F385E02DC70119958F3F980772
:10F3200029F0F80181938F012196EDCFCE01DF9175
:10F33000CF911F910F91FF90EF90DF90CF900895A4
:10F34000CF93C62FDC01ED91FC910088F189E02D6F
:10F350001995DC01ED91FC910190F081E02D6C2F6D
:10F36000CF911994062E000C770BFC0177836683EE
:10F370000895CF93DF93EC018E819F81019611F563
:10F38000E881F9810088F189E02DCE011995DC0131
:10F39000ED91FC910084F185E02D1995892BB1F058
:10F3A000E881F9810284F385E02DCE01199581323F
:10F3B000910534F3E881F9810684F785E02D682F03
:10F3C000CE01199581E0DF91CF91089580E0FBCFC8
:10F3D000CF93DF931F92CDB7DEB76983DC01ED9148
:10F3E000FC910280F381E02D41E050E0BE016F5FAF
:10F3F0007F4F19950F90DF91CF910895EF92FF9273
:10F400000F931F93CF93DF93EC018B017A010E943E
:10F41000BEA2688B798B8A8B9B8B8C819D81DC0152
:10F42000ED91FC910280F381E02DA701B801DF91FD
:10F43000CF911F910F91FF90EF9019941F93CF934D
:10F44000DF93EC01162F0E94BEA2688B798B8A8B0A
:10F450009B8B8C819D81DC01ED91FC910190F08171
:10F46000E02D612FDF91CF911F911994CF92DF9200
:10F47000EF92FF92CF93DF93EC018E819F818F3FBC
:10F48000980759F02FEF3FEF3F832E83DF91CF9105
:10F49000FF90EF90DF90CF9008950E94BEA26B0185
:10F4A0007C01A4EFCA0EA1E0DA1EE11CF11CE88188
:10F4B000F9810088F189E02DCE011995DC01ED91EB
:10F4C000FC910084F185E02D1995892B39F40E9477
:10F4D000BEA26C157D058E059F0548F3E881F98174
:10F4E0000088F189E02DCE011995DC01ED91FC91A8
:10F4F0000284F385E02DDF91CF91FF90EF90DF90B4
:10F50000CF9019940E94F5D10F931F93CF93DF935F
:10F51000D0E0C0E0009791F08C01C0EED6E06881A9
:10F5200079816115710529F0C8010E9475D2892B76
:10F5300029F00B80DC81C02D209789F7CE01DF9167
:10F54000CF911F910F9108950F931F93CF93DF9346
:10F55000EC0188819981009759F02A813B81261717
:10F56000370730F081E0DF91CF911F910F9108951F
:10F570008B016F5F7F4F0E9414D1009759F09983E0
:10F5800088831B830A832C813D81232B59F7FC013F
:10F590001082E8CF80E0E7CFEF92FF920F931F93A6
:10F5A000CF93DF93009751F4CFEFDFEFCE01DF91E0
:10F5B000CF911F910F91FF90EF900895DC011C9661
:10F5C000ED90FC90F70100811181D801ED91FC9143
:10F5D0000688F789E02DC8011995882329F3D801F9
:10F5E000ED91FC910084F185E02DC8011995D801B9
:10F5F000ED91FC91892B61F30284F385E02DC80124
:10F600001995EC01019681F2F8018789882329F088
:10F610006C2F8AED98E00E94C797D70112968C91C3
:10F62000882321F2C532D10509F6D801ED91FC916C
:10F630000084F185E02DC801199502975CF0D8018E
:10F64000ED91FC910688F789E02DC801199581118B
:10F65000ECCFAACFD1E0C0E0D801ED91FC910284BB
:10F66000F385E02DC80119958F3F980709F49CCFC9
:10F670009C01215431092A31310570F48D2F829576
:10F68000807F829FC00D1124D11104C00C2E000C6C
:10F69000DD0B8CCFD0E0E0CF9C01215631092A311F
:10F6A000310560F3C0978A30910570F79D2F9295D0
:10F6B000907F989FC00D1124E7CFCF92DF92EF92F9
:10F6C000FF920F931F93CF93DF936C018B0186E022
:10F6D00090E00E9411C4EC019093220780932107CF
:10F6E000F60101900020E9F7CF018C199D090E94D5
:10F6F00011C47C01B6010E947ED2F6010190002067
:10F70000E9F73197EC19FD09EE0DFF1D1082F98222
:10F71000E8821B830A8380912307909124079D83AD
:10F720008C83D0932407C0932307DF91CF911F913F
:10F730000F91FF90EF90DF90CF900895FC018681AC
:10F7400097818F3F980729F02FEF3FEF378326836C
:10F750000895808591850C949FC71F93CF93DF9365
:10F76000182F66E270E00E94231EC82F67E270E047
:10F77000812F0E94231E9C2FDF91CF911F9108950E
:10F78000CF93FC01C08D80E590E00E94E59C60E293
:10F7900070E08C2F0E94449D62E070E08C2F0E94EC
:10F7A000231E84FD1AC062E070E08C2F0E94231E8D
:10F7B00083FF0CC048E162E070E08C2F0E94191EAC
:10F7C0000E949B1E90E080E0CF9108950E949B1EB6
:10F7D00080E590E00E94E59CDFCF40E162E070E0D0
:10F7E0008C2F0E94191E0E949B1E81E090E0ECCF9E
:10F7F000FF920F931F93CF93DF93EB01FC01178AC6
:10F80000168A2A81211109C02B81211106C02C8161
:10F81000211103C02D812223F1F041155105D9F0AA
:10F820008A01FC01F08C80E590E00E94E59CBE011D
:10F830006E5F7F4F8F2D0E94521EB8018F2D0E9448
:10F84000411E0E949B1E81E090E0DF91CF911F91AD
:10F850000F91FF90089590E080E0F7CFAF92BF92B4
:10F86000CF92DF92FF920F931F93CF93DF938C0180
:10F870005B01EA01FC01C688D788F08C80E590E046
:10F880000E94E59C8F2D0E94FC9D8C179D0720F403
:10F890008F2D0E94FC9DEC019E01A501B6018F2DCC
:10F8A0000E949C9D0E949B1EF801868997898C0F5F
:10F8B0009D1F978B868BCE01DF91CF911F910F916A
:10F8C000FF90DF90CF90BF90AF9008957F928F927E
:10F8D0009F92AF92BF92CF92DF92EF92FF920F93DF
:10F8E0001F93CF93DF93CDB7DEB7A6970FB6F894EB
:10F8F000DEBF0FBECDBF8C01762E942E852E20E26A
:10F90000A22ECE0101967C01DC01EA2D1D92EA9522
:10F91000E9F76801F3E4CF0ED11C8DEA93E09AA3D6
:10F9200089A38FEF8BA38CA38DA38EA343E450E018
:10F93000BE016F5D7F4FC6010E94F87B019609F4FE
:10F94000BFC081E089838A8386E0B82EBB821C8297
:10F95000D80114966D917D918D919C9117970E947D
:10F960001CCE6D837E838F83988789869A8680E8F4
:10F9700090E09C878B874CE150E0B701C6010E9464
:10F980002E7CFE0137968AE1DF011D928A95E9F708
:10F990004801B8E08B0E911CF401D70101900D9243
:10F9A000BA94E1F740E150E0B701C6010E942E7C15
:10F9B000F7011192AA94E9F796E0A92EB12C40E242
:10F9C00050E0B701C6010E942E7CF1E0AF1AB108E9
:10F9D000B1F783E6898392E89A8393E59B838C83CE
:10F9E00085E38D8381E08E837F829DE3988797E016
:10F9F00099878A8786E0F401DE011B9601900D92BB
:10FA00008A95E1F78CE0898B8A8B61E275E0CE0103
:10FA100043960E947ED2D8011B966C91CE014996E6
:10FA20000E94189EF8016485CE014B960E94189E94
:10FA3000D8011D966C91CE014D960E94189E4EE104
:10FA400050E0B701C6010E942E7CB3E07B121EC0BD
:10FA500082E3898384E08A83F80196859B83978576
:10FA60009C8390899D8391899E8396E39F83888759
:10FA7000828D8987838D8A87848D8B87858D8C87FE
:10FA80004CE050E0B701C6010E942E7C87E38983D9
:10FA900086E08A8391E09B8393E09C838D838FE053
:10FAA0008E838AE38F838BE388878FEF898749E092
:10FAB00050E0B701C6010E942E7CC6010E94C07BA7
:10FAC000A6960FB6F894DEBF0FBECDBFDF91CF91E3
:10FAD0001F910F91FF90EF90DF90CF90BF90AF906C
:10FAE0009F908F907F900895AF92BF92CF92DF92B8
:10FAF000EF92FF920F931F93CF93DF93DC01CD9092
:10FB0000DC901197C114D10439F01496CD91DC9199
:10FB10008C017601209761F4DF91CF911F910F91B5
:10FB2000FF90EF90DF90CF90BF90AF900895750158
:10FB30005701BFEFAB1ABB0AF7018081082E000CFA
:10FB4000990B0E9423C6892B91F72197CC0DDD1DBF
:10FB50008881082E000C990B0E9423C6892B29F05E
:10FB6000CE15DF0510F02197F3CFAE014F5F5F4F49
:10FB70004E195F09D80115965C934E931497CE14D5
:10FB8000DF0420F4B701C6010E9431D2D801ED9103
:10FB9000FC91119714968D919C91E80FF91F10829A
:10FBA000BBCFCF93DF93DC011496ED91FC916E17E0
:10FBB0007F0728F54115510511F19F01261B370BD1
:10FBC0004217530708F49A01DB01EC0188819981FF
:10FBD000E21BF30BFD83EC83AF01461B570B260F93
:10FBE000371FBC01620F731F8A0F9B1F0E94A3D295
:10FBF000E881F9818C819D81E80FF91F1082DF91E6
:10FC0000CF910895DF92EF92FF920F931F93CF93BE
:10FC1000DF93FC01E480F580E114F10451F48FEFEF
:10FC20009FEFDF91CF911F910F91FF90EF90DF90A9
:10FC30000895EC010190F081E02DEE0DFF1DD080C4
:10FC4000108208811981062E000C770BC8010E94D2
:10FC5000B2D20E0D1F1DF801D082009701F328814A
:10FC60003981821B930BDDCFFB0144815581FC015F
:10FC7000248135812417350778F0808191810097A0
:10FC800059F0FB01608171816115710529F00E94B5
:10FC900095D221E0892B09F020E0822F0895FC0104
:10FCA00024813581232B39F421E0FB0180818823D5
:10FCB00049F020E007C0808191810E9475D221E047
:10FCC000892BB9F7822F0895FC0124813581FB012E
:10FCD0004481558124173507E1F4FC01808191812D
:10FCE000FB01608171810097D1F061157105A1F46C
:10FCF000232BC1F0FC01808190E008C0232B91F000
:10FD0000FB01808190E091958195910921E0892BFB
:10FD100009F020E0822F08950E9475D2F7CF611577
:10FD2000710561F721E0F6CFEF92FF920F931F93D9
:10FD3000CF93DF936115710541F480E0DF91CF919E
:10FD40001F910F91FF90EF90089541155105B1F06B
:10FD50007B01EC010C811D81040F151FB8010E946D
:10FD6000A47A882351F3288139818C819D81B70140
:10FD7000820F931F0E947ED21D830C8381E0DECF11
:10FD8000CF93DF931F921F92CDB7DEB769831A829C
:10FD900041E050E0BE016F5F7F4F0E94947E0F9064
:10FDA0000F90DF91CF9108950F931F93CF93DF931F
:10FDB0008C01EB01FC01808191810097E1F0688169
:10FDC000798161157105A9F0428153812C813D81B2
:10FDD0004217530770F00E947ED28C819D81F801FA
:10FDE000958384831D821C82DF91CF911F910F9197
:10FDF00008950E94ADC488819981F8019183808320
:10FE00008A819B81938382838C819D819583848366
:10FE1000198218821B821A82E5CFCF93DF93EC01FF
:10FE200088819981009711F00E94ADC419821882CF
:10FE30001D821C821B821A82DF91CF910895EF925E
:10FE4000FF920F931F93CF93DF9300D01F92CDB7F4
:10FE5000DEB77C01862F4AE08E010F5F1F4FB8018D
:10FE600090E00E94C6C6F80101900020E9F73197A2
:10FE7000AF01401B510BB801C7010E94947E811154
:10FE800003C0C7010E940D7FC7010F900F900F9014
:10FE90000F90DF91CF911F910F91FF90EF900895F8
:10FEA000CF93DF93EC016115710539F4CE010E9407
:10FEB0000D7FCE01DF91CF910895FB0101900020CD
:10FEC000E9F73197AF01461B570B0E94947E8823B8
:10FED00069F3EFCFCF93DF93EC01FB0144815581B0
:10FEE000608171810E94947E811103C0CE010E94C5
:10FEF0000D7FCE01DF91CF910895EF92FF920F9386
:10FF00001F93CF93DF93EC017B018A01BA010E941A
:10FF1000A47A81110BC0CE010E940D7FCE01DF912A
:10FF2000CF911F910F91FF90EF9008951D830C8347
:10FF3000B701888199810E947ED2F0CFFB010190A8
:10FF40000020E9F73197AF01461B570B0C947D7FDA
:10FF5000CF93DF93EC016115710531F00E949E7F14
:10FF6000CE01DF91CF9108950E940D7FF9CFCF93FD
:10FF7000DF93EC01FB018617970749F060817181DF
:10FF80006115710541F0448155810E947D7FCE014C
:10FF9000DF91CF9108950E940D7FF9CFFC01808100
:10FFA0009181009711F00C94ADC40895EF92FF92E7
:10FFB0000F931F93CF93DF93EC018B01198218826B
:10FFC0001B821A821D821C82CB010E945AC67C01B0
:10FFD000BC01CE010E94A47A811109C0CE01DF913B
:10FFE000CF911F910F91FF90EF900C940D7FFD82A8
:10FFF000EC82B80188819981DF91CF911F910F9197
:020000021000EC
:10000000FF90EF900C9453C6FC0111821082138272
:100010001282158214820C94B77FFC011182108227
:100020001382128215821482FB0101900020E9F7ED
:100030003197AF01461B570B0C947D7FAF92BF9257
:10004000CF92DF92EF92FF920F931F93CF93DF93A4
:100050005C016B017A0189012417350720F48F2D8B
:100060007901042F182F6AE275E0C5010E940D8006
:10007000D6011496CD91DC91EC16FD06C8F40C1750
:100080001D0708F4E801D601ED91FC911197EC0FE2
:10009000FD1F108110826D917C916E0D7F1DC50139
:1000A0000E94A87FF60180819181C80FD91F188313
:1000B000C501DF91CF911F910F91FF90EF90DF90DD
:1000C000CF90BF90AF9008950F931F93CF93DF937E
:1000D000EC010E94BEA2688779878A879B87E881A6
:1000E000F9810284F385E02DCE01199597FF15C0A3
:1000F0000E94BEA2088519852A853B85601B710B6D
:10010000820B930B0C811D812E813F81601771073B
:100110008207930720F38FEF9FEFDF91CF911F911D
:100120000F910895EF92FF920F931F93CF93DF9358
:10013000EC017B01042F6AE275E00E940D80C7018B
:100140000E946480002E000C110B97FD0BC0081755
:10015000190741F0682FCE010E94C07EC7010E949E
:100160006480F3CFCE01DF91CF911F910F91FF906B
:10017000EF900895FB0101900020E9F73197AF015E
:10018000461B570BDC01ED91FC910280F381E02DC1
:1001900019948F929F92AF92BF92EF92FF920F931A
:1001A0001F93CF93DF93CDB7DEB7A1970FB6F89427
:1001B000DEBF0FBECDBF7C01FA01CB0119A22230F8
:1001C00008F42AE08E010F5D1F4F822E912CB12C76
:1001D000A12CBF01A50194010E9489CDF901CA019A
:1001E0006A300CF5605DD8016E938D01232B242BB2
:1001F000252B79F790E080E0109721F0BD01C70131
:100200000E94BA80A1960FB6F894DEBF0FBECDBF94
:10021000DF91CF911F910F91FF90EF90BF90AF9022
:100220009F908F900895695CDECF68E275E00C9432
:10023000BA80DC01ED91FC910190F081E02D1994E0
:10024000CF92DF92EF92FF920F931F93CF93DF93A2
:100250002115310581F4DC01ED91FC910190F081D3
:10026000E02D642FDF91CF911F910F91FF90EF90C0
:10027000DF90CF9019942A30310501F52AE077FFFD
:100280001DC06A017B01EC016DE20E9419818C01A5
:1002900044275527BA014C195D096E097F092AE0E8
:1002A000CE010E94C980800F911FDF91CF911F91D5
:1002B0000F91FF90EF90DF90CF900895DF91CF9155
:1002C0001F910F91FF90EF90DF90CF900C94C98019
:1002D0008F929F92AF92BF92CF92DF92EF92FF9256
:1002E0000F931F93CF93DF937C018B014C0182E02E
:1002F000880E911C5701E5E0AE0EB11CD0E0C0E0C5
:10030000F40161914F01C8010E94C7976C016EE230
:10031000C8010E9419818C0D9D1DC80FD91F8A1418
:100320009B0471F7F7016581C8010E94C7978C0F84
:100330009D1FDF91CF911F910F91FF90EF90DF9064
:10034000CF90BF90AF909F908F90089561157105E9
:1003500011F00C94BA8090E080E008950F931F9301
:10036000CF93DF93EC018B016EE075E00E94A681D4
:1003700001151105C1F1F80161918F01662399F111
:10038000603240F0623231F06C3521F0CE010E94D3
:100390001981F1CF6CE5CE010E941981F8013197E6
:1003A00080818C30D1F044F48930D9F08A30B9F0B2
:1003B000883009F762E6EACF823259F024F462E726
:1003C0008D3021F3D8CF8F3231F06CE58C35F1F2DE
:1003D000D2CF62E2DBCF6FE2D9CF66E6D7CF6EE64F
:1003E000D5CF64E7D3CF62E2CE010E94198190E0BD
:1003F00080E0DF91CF911F910F910895DB0114965A
:100400004D915C9115976D917C91DC01ED91FC9182
:100410000280F381E02D1994EF92FF920F931F93C6
:10042000CF93DF938C017B01D0E0C0E0F701EC0FAC
:10043000FD1F6491662361F0D801ED91FC9101905C
:10044000F081E02DC8011995892B11F02196EECF8E
:10045000CE01DF91CF911F910F91FF90EF90089502
:100460000F931F93CF93DF93EC010E940C828C01BA
:10047000CE010E941581800F911FDF91CF911F91B6
:100480000F9108958AED98E00E9415816BE378E161
:100490008AED98E00C940C82DC018DEA93E08D9358
:1004A0009D9384E0FB0101900D928A95E1F70895F8
:1004B0001F920F920FB60F9211240BB60F922F932B
:1004C0003F934F935F936F937F938F939F93AF93DC
:1004D000BF93EF93FF938AED98E00E948477FF919A
:1004E000EF91BF91AF919F918F917F916F915F91AC
:1004F0004F913F912F910F900BBE0F900FBE0F9019
:100500001F9018951F920F920FB60F9211240BB6E1
:100510000F922F938F939F93EF93FF93E091EA08AD
:10052000F091EB088081E091F008F091F10882FDF4
:100530001DC090818091F3088F5F8F732091F40824
:10054000821741F0E091F308F0E0E652F74F958F03
:100550008093F308FF91EF919F918F912F910F90CE
:100560000BBE0F900FBE0F901F9018958081F2CF99
:10057000DF92EF92FF920F931F93CF93DF9300D000
:1005800000D0CDB7DEB78B017A01D22E6AE275E0DA
:10059000CE0101960E940D809E012F5F3F4F4D2D91
:1005A000B701C8010E94C6A9CE0101960E94CE7F64
:1005B00026960FB6F894DEBF0FBECDBFDF91CF9168
:1005C0001F910F91FF90EF90DF900895CF92DF92EF
:1005D000EF92FF920F931F93CF93DF93CDB7DEB7C8
:1005E000EC970FB6F894DEBF0FBECDBFDC012C91A7
:1005F000222309F459C06FEC73E00E9490C69A83DD
:1006000089837E01B3E0EB0EF11C01E010E0D02EF7
:10061000C12E6FEC73E090E080E00E9490C6F7017D
:10062000819391937F010E31110521F00F5F1F4FD0
:10063000892B69F70091210710912207E980FA8040
:100640000115110549F1D8016D917C91C7010E94F6
:1006500075D2892BE9F4D8011296ED91FC91BE0177
:100660006F5F7F4F8D2D9C2D19958C010E944282CA
:10067000C801EC960FB6F894DEBF0FBECDBFDF9178
:10068000CF911F910F91FF90EF90DF90CF90089541
:10069000F80104811581D4CF6FE378E18AED98E009
:1006A0000E9430820E94428210E000E0E1CFCF93AE
:1006B0008AED98E00E946E77892BE9F18AED98E047
:1006C0000E944C77C82F8A3089F08D3079F08830BD
:1006D00001F568E08AED98E00E9419818091250774
:1006E000882331F3815080932507E2CFE0912507DD
:1006F000F0E0EB51F94F108268E275E08AED98E086
:100700000E94A68185EE96E00E94E682109225075F
:10071000CFCF682F8AED98E00E941981E0912507DC
:10072000EB3330F681E08E0F80932507F0E0EB513C
:10073000F94FC083BDCFCF910895CF93DF930E942F
:10074000847AEC01892B99F08A8181508A83811106
:100750000EC0888199810E94ADC419821882E091EF
:10076000E306F091E406C0EED6E0309719F4DF918D
:10077000CF9108959381848120813181232B41F48D
:100780009B838C83CF010E94ADC49B818C81FE0131
:10079000EF01E92FF82FE9CFEF92FF920F931F930C
:1007A000CF93DF937C010E94847AFC01892B61F056
:1007B00082818F5F828380819181DF91CF911F91B0
:1007C0000F91FF90EF900895C0EED6E08881998157
:1007D000892B51F4C7010E940AD29983888321E0B2
:1007E0002A83EBCFEC01F2CF8B819C810097D1F76C
:1007F00085E090E00E9411C48C0190E080E001153A
:100800001105D9F21C830B83C7010E940AD2F8019B
:100810009183808321E0228314821382CECF8F9232
:100820009F92AF92BF92CF92DF92EF92FF920F937F
:100830001F93CF93DF936115710509F48FC0DB011E
:100840001896EC911897E770E73008F087C0EC0134
:10085000F0E08827E15DFB478F4F0C9414CE36847F
:10086000478450846784B184C384FC846BE275E060
:10087000CE01DF91CF911F910F91FF90EF90DF900C
:10088000CF90BF90AF909F908F900C94BA801996A4
:100890008C9165E375E0882359F360E375E0E8CF58
:1008A00019964D915D916D917C911C972AE030E0F5
:1008B000CE01DF91CF911F910F91FF90EF90DF90CC
:1008C000CF90BF90AF909F908F900C9420811996FD
:1008D000CD90DD90ED90FC901C9720E030E0A901D8
:1008E000C701B6010E943FCC87FF09C064EC73E0EA
:1008F000CE010E94A681F7FAF094F7F8F094C701B0
:10090000B6010E9418CF4B015C01BC01A401CE01CD
:100910000E94C4976DED74E0CE010E94A681C501CE
:10092000B4010E9444CC9B01AC01C701B6010E94F6
:1009300032CE2DEC3CEC4CE45DE30E9433CE20E063
:1009400030E040E251E40E94A5CC0E9418CFAB01F8
:1009500070E060E02AE0CE010E94C98090E080E073
:100960001DC019966D917C91CE01DF91CF911F91A1
:100970000F91FF90EF90DF90CF90BF90AF909F903E
:100980008F900C94AE8116960D911C916BE5CE0163
:100990000E941981019679F48FEF9FEFDF91CF913B
:1009A0001F910F91FF90EF90DF90CF90BF90AF908D
:1009B0009F908F9008950115110579F0B801CE012F
:1009C0000E940F84019641F3D80112960D911C915B
:1009D0000115110511F06CE2DACF6DE5CE010E9430
:1009E000198121E030E0019611F030E020E0882705
:1009F0009927821B930BD2CF16960D911C916BE712
:100A0000CE010E941981019639F20115110529F1D3
:100A1000D8016D917C91CE010E94AE81019609F4BE
:100A2000BBCF6AE3CE010E941981019609F4B4CFCD
:100A3000B801CE010E940F84019609F4ADCFD80110
:100A400012960D911C910115110539F06CE2CE0141
:100A50000E9419810196C9F69FCF6DE7BFCF0F9312
:100A60001F93CF93DF93EC01E881F9810284F38532
:100A7000E02D199500E011E08F3F9807D1F0813209
:100A80009105E4F401501109E881F9810F3F100745
:100A900031F00284F385E02DCE011995EDCFE88188
:100AA000F9810684F785E02D682FCE01199590E035
:100AB00080E0DF91CF911F910F910895012B79F77D
:100AC0008FEF9FEFF6CFCF92DF92EF92FF920F93CF
:100AD0001F93CF93DF937C016B01DC01ED91FC91BF
:100AE0000284F385E02D1995829761F0CFEFDFEF57
:100AF000CE01DF91CF911F910F91FF90EF90DF908A
:100B0000CF900895F6018085887F8460808786E095
:100B100090E00E9411C48C01009741F3E0EAF6E0F6
:100B2000DC01ED93FC9380E4DF011D928A95E9F7E7
:100B300080E490E0F8019383828315821482D701C8
:100B4000ED91FC910284F385E02DC7011995EC012C
:100B50000196C9F0C232D10509F44DC0C032D105A9
:100B60000CF449C0B8018C2FCC35D10549F5D7011B
:100B7000ED91FC910284F385E02DC7011995EC01FC
:100B80008F3F980721F4C8010E94ADC4B1CF8236CF
:100B9000910541F15CF48F32910509F18C35910595
:100BA000D9F0829761F6B80182E20AC08E369105CB
:100BB000E1F04CF4B8018CE0C636D10509F0BFCFA6
:100BC0000E945179BCCF8237910591F0B80189E03C
:100BD000C437D105A9F3B3CFB8018CE5F1CFB80183
:100BE0008FE2EECFB80188E0EBCFB8018AE0E8CF22
:100BF000B8018DE0E5CFF80184819581009749F037
:100C00000190F081E02DE80FF91F31978081882352
:100C100021F0B80180E00E94517980EA96E00E94BC
:100C2000CC83EC01892B19F0C8010E94ADC4D60118
:100C30001A96DC93CE931997D0E0C0E059CF8DE09F
:100C400090E00E9411C4009729F02DE0FC01119260
:100C50002A95E9F708950F931F93CF93DF93009799
:100C6000E1F0EC010C851D850115110579F0D80125
:100C70008D919C91009739F0DC01ED91FC910488F5
:100C8000F589E02D1995C8010E94ADC4CE01DF9110
:100C9000CF911F910F910C942AC7DF91CF911F9193
:100CA0000F910895AF92BF92CF92DF92EF92FF9291
:100CB0000F931F93CF93DF9300D01F92CDB7DEB772
:100CC00061157105B1F06B01182FDB011C96AD9019
:100CD000BC90F501E080F180D701ED91FC91068890
:100CE000F789E02DC7011995811106C0C6010E9440
:100CF0002B868FEF9FEF13C0F5019281911124C0D5
:100D0000D701ED91FC910190F081E02D612FC70199
:100D10001995F7018789811111C090E080E00F904B
:100D20000F900F900F90DF91CF911F910F91FF9037
:100D3000EF90DF90CF90BF90AF900895612F8AED34
:100D400098E00E941981E9CF812F8F7D81548A31EB
:100D5000B8F280ED810F8A3098F283ED810F8230F6
:100D600078F21F3569F21E3759F21132B1F086EC74
:100D7000810F823090F08AED810F873070F01D3343
:100D800061F0812F8F7E8F3241F08DED810F8230A7
:100D900020F01B3511F01D3511F491FFB1CF1982F0
:100DA0001A821B821C82812F012E000C990B9F93AB
:100DB0001F938BE395E09F938F938E010F5F1F4FDF
:100DC0001F930F930E94FAD26E01F4E0CF0ED11C54
:100DD0000F900F900F900F900F900F90D8016D9182
:100DE0008D01D701ED91FC910190F081E02DC701BB
:100DF0001995F7018789882339F0F80131976081C7
:100E00008AED98E00E9419810C151D0539F785CFF0
:100E10002C9A08952C9808951F93CF93DF93182F41
:100E200060E270E00E94231EC82F61E270E0812F13
:100E30000E94231E9C2FDF91CF911F9108958EBD9C
:100E400000000DB407FEFDCF8EB50895CF92DF925E
:100E5000EF92FF920F931F93CF93DF93EC017A01F0
:100E60008B016C01C40ED51ECC15DD05A9F00E94C6
:100E70000A878FE00E941F878D2F0E941F878C2F6B
:100E80000E941F87219680E00E941F87F8018193AE
:100E90008F010E940887E8CFC701DF91CF911F9192
:100EA0000F91FF90EF90DF90CF900895CF92DF9257
:100EB000EF92FF920F931F93CF93DF93EC017A0190
:100EC0008B016C01C40ED51ECC15DD05A1F00E946E
:100ED0000A8780EF0E941F878D2F0E941F878C2F0B
:100EE0000E941F872196F80181918F010E941F8720
:100EF0000E940887E9CFC701DF91CF911F910F9121
:100F0000FF90EF90DF90CF9008951F93CF93DF93E2
:100F1000D82F192FC62F0E940A8780EF0E941F87A3
:100F2000812F0E941F878D2F0E941F878C2F0E9468
:100F30001F870E94088781E0DF91CF911F9108955C
:100F4000EF92FF920F931F93CF93C82F7B0180E501
:100F500090E00E94E59C68E270E08C2F0E94231EC6
:100F6000082F69E270E08C2F0E94231E282F302F5B
:100F7000B90121E030E0A7018C2F0E94549D0E940E
:100F80009B1E81E090E0CF911F910F91FF90EF9019
:100F90000895CF93DF931F92CDB7DEB7FC01218D6B
:100FA000328D8FEF9FEF232B41F0BE016F5F7F4F9C
:100FB000808D0E94A087898190E00F90DF91CF9172
:100FC0000895FF920F931F93CF93DF93F82E80E540
:100FD00090E00E94E59C10E000E08F2D0E94AD7B28
:100FE000EC01892B21F08F2D0E94AD7B8C01C01765
:100FF000D10799F70E949B1ECE01DF91CF911F91DF
:101000000F91FF900895AF92BF92CF92DF92EF922F
:10101000FF921F93CF93DF93182F6B017A0180E526
:1010200090E00E94E59CB12CA12C812F0E94AD7B09
:10103000EC01892B21F0812F0E94AD7B5C01CA1548
:10104000DB0599F72097F9F463E070E0812F0E94A7
:10105000231E843159F0882349F0C1E0D0E08C315F
:1010600011F4D0E0C0E0D195C195D1090E949B1E3A
:10107000CE01DF91CF911F91FF90EF90DF90CF9045
:10108000BF90AF900895EC16FD060CF4E7011C1616
:101090001D0664F768E270E0812F0E94231EE82E8F
:1010A00069E270E0812F0E94231E282F3E2D7901D6
:1010B0009E01A601B701812F0E94549DEC0EFD1EDA
:1010C0004F2D68E270E0812F0E94191E4E2D69E2BB
:1010D00070E0812F0E94191E60E470E0812F0E9451
:1010E000449DC4CFCF93DF93FC01218D328D211518
:1010F000310529F48FEF9FEFDF91CF910895EC0137
:10110000808D4217530708F0A9010E940388181622
:10111000190684F7298D3A8D281B390B3A8F298FB0
:10112000EBCF0F931F93CF93DF931F92CDB7DEB713
:10113000FC01218D328D232B41F48FEF9FEF0F9017
:10114000DF91CF911F910F9108958C0141E050E004
:10115000BE016F5F7F4FFC01808D0E9403881816CF
:1011600019065CF7F801818D928D0197928F818F1E
:10117000898190E0E4CF0F931F93CF93DF9300D04A
:1011800000D01F921F92CDB7DEB78C01D8015996BF
:101190008D919C915A97892B41F0ED91FC9102849D
:1011A000F385E02DC8011995F1CFF801808D0E94DB
:1011B000E18718161906B4F548E050E0BE016F5FEC
:1011C0007F4FD80158968C910E94038818161906F3
:1011D000F4F4D801509684E0FE01319601900D920E
:1011E0008A95E1F78D8190E0982F88272E81820FD4
:1011F000911DF801958B848B8F81282F30E0322F41
:1012000022278885820F932F911D928F818F289698
:101210000FB6F894DEBF0FBECDBFDF91CF911F9107
:101220000F91089590E080E0F2CF4F925F926F921D
:101230007F928F929F92AF92BF92CF92DF92EF9266
:10124000FF920F931F93CF93DF93CDB7DEB76397D2
:101250000FB6F894DEBF0FBECDBF7C016B013A0123
:10126000FB0120E090E080E06AE03191332309F453
:1012700061C040ED430F4A3008F04DC0689FA001A7
:10128000699F500D1124CA01C097830F911D37FD2E
:101290009A958F3F910549F340F3F70142815381BD
:1012A0006481758180912D0890912E08A0912F085E
:1012B000B0913008481759076A077B0709F42EC216
:1012C0008701085F1F4F0E94BEA26F7077277C5F67
:1012D000C8010E940315813009F025C28DEA93E010
:1012E0009A838983F70182819381A481B5818B835D
:1012F0009C83AD83BE8345E350E0BE016F5F7F4FAB
:10130000C8010E94F87B892BA9F5D12CC12CC801FA
:101310000E94EE1417C03E3209F0BFCF233009F40B
:10132000BCCFD301A20FB11D12968C932F5F90E01A
:1013300080E09BCF233009F0B0CFF3018583CC242C
:10134000C394D12CC60163960FB6F894DEBF0FBECE
:10135000CDBFDF91CF911F910F91FF90EF90DF9064
:10136000CF90BF90AF909F908F907F906F905F9045
:101370004F9008950E94BEA2F70177836683762777
:10138000672776277A83698342E050E0BE016F5F6A
:101390007F4FC8010E942E7C81E090E09E878D8760
:1013A00042E050E0BE01635F7F4FC8010E942E7C87
:1013B00080E091E09E878D8742E050E0BE01635F50
:1013C0007F4FC8010E942E7C1E861D8642E050E0A1
:1013D000BE01635F7F4FC8010E942E7C42E050E057
:1013E000BE01635F7F4FC8010E942E7C42E050E047
:1013F000BE01635F7F4FC8010E942E7C5601F6013B
:101400008081882301F16501F60181912F018823F4
:1014100011F08E32B1F446018A189B081814190491
:1014200074F48F8641E050E0BE01615F7F4FC801D8
:101430000E942E7CA401B501C8010E942E7C52019D
:10144000DECF6201E1CF1F8641E050E0BE01615F67
:101450007F4FC8010E942E7CC12CDD24D394DE86F0
:10146000CD8642E050E0BE01635F7F4FC8010E941D
:101470002E7CDE86CD8642E050E0BE01635F7F4F6A
:10148000C8010E942E7CC8010E94C07B892B09F4F0
:101490003CCFF3E0AF2EB12C230122E0420E511CD1
:1014A000EEC0F7014281538164817581808D918DF9
:1014B000A28DB38D481759076A077B0709F024C12D
:1014C000848D958DC59709F01FC181A192A15DEF13
:1014D000C52EDD24DA940C970CF4C5C04CE050E026
:1014E000BE016F5F7F4FC8010E9472888B819C8113
:1014F0009827892798279A8B898B29813A813227C7
:1015000023273227F701468157814217530709F0F5
:1015100000C197FFFEC08F7092703BEFC32EDD2499
:10152000DA94892B09F09FC06F8078847624672431
:1015300076242AEFC22EDD24DA946114710409F4B2
:1015400092C0D12CC12C8D819E8198278927982704
:10155000C816D90640F541E050E0BE01635F7F4FF9
:10156000C8010E9472888D85882351F08D859FEF78
:10157000980F9D87882321F0C8010E949188F6CF9B
:101580008D858111E8CFC8010E949188C8010E9411
:101590009188C8010E949188C8010E949188FFEF3C
:1015A000CF1ADF0AD0CF912C812C41E050E0BE0150
:1015B0006D5E7F4FC8010E9472888B89982F907C46
:1015C00061F4882389F08B899FEF980F9B8B882388
:1015D00041F0C8010E949188F6CFC8010E9491880D
:1015E0001B8A8B898111E1CF42E050E0BE01615F2F
:1015F0007F4FC8010E94728842E050E0BE01635FE5
:101600007F4FC8010E947288C8010E949188C8015A
:101610000E949188C8010E949188C8010E94918807
:1016200042E050E0BE016F5E7F4FC8010E947288A9
:101630008F8598898115914009F040C0CD84DE8462
:10164000DC24CD24DC2481E0C816D104B9F58989D5
:101650009A898115944009F04EC044E050E0B201EF
:10166000C8010E9472880E94EB6481E0A81AB10848
:1016700009F44DCEFFEFCF16DF0609F048CE0E94E9
:10168000BEA23B014C01C8010E94BB881816190676
:101690000CF407CF0E94BEA2661977098809990940
:1016A000613A7F408105910558F50E94EB6461E045
:1016B00070E080E090E00E9479A0E5CFD12CC12CB1
:1016C00089899A89982789279827C816D90638F4CE
:1016D000C8010E949188FFEFCF1ADF0AF1CF2FEFE8
:1016E000821A920A6814790409F05FCF96EFC92E26
:1016F000DD24DA94B8CFE7EFCE2EDD24DA94B3CF31
:10170000CC24CA94DC2CAFCF6EEFC62EDD24DA9445
:10171000AACF4CEFC42EDD24DA94A5CF8EEFC82ECD
:10172000DD24DA940FCED12CC12C0CCE2F923F9217
:101730004F925F926F927F928F929F92AF92BF92E1
:10174000DF92EF92FF920F931F93CF93DF93CDB76A
:10175000DEB7E4970FB6F894DEBF0FBECDBF7C01B5
:101760004A015B0119010E94BEA22B013C018701C5
:101770000D5B1F4FC8010E94BB88181619069CF00C
:101780000E94BEA2641975098609970986169706F4
:10179000A806B90608F488C162E370E080E090E032
:1017A0000E9479A0E7CF42E250E0BE016F5F7F4F19
:1017B000C8010E94728889818230D1F0D12C8D2D90
:1017C000E4960FB6F894DEBF0FBECDBFDF91CF9188
:1017D0001F910F91FF90EF90DF90BF90AF909F907F
:1017E0008F907F906F905F904F903F902F900895D3
:1017F000F801848995898334910501F76D817E8193
:101800008F8198850E941CCE2B013C01F101408202
:1018100051826282738246E050E0B701685F7F4F79
:10182000CE014D960E9424D2892B41F6F70180818A
:101830009181A281B381481659066A067B0608F495
:10184000BDCF84819581A681B78184159505A605B4
:10185000B70508F4B3CF89899A89AB89BC89868793
:101860009787A08BB18B8EECA82EB12CC8010E945B
:101870009188F1E0AF1AB108C9F7D12CC70182965F
:101880009AA789A7F701B696FCA7EBA708969EA78B
:101890008DA73C974F01899698AB8FA73897FAABE5
:1018A000E9AB1701F6E12F0E311CC5979CAB8BAB52
:1018B000F801818D928D181619060CF080CFC801A1
:1018C0000E9491888333910509F4D4C0A4F5813036
:1018D000910509F474C074F4892B51F3C8010E9476
:1018E0009188B82EBA94FFEFBF1611F3C8010E9479
:1018F0009188F8CF8330910509F46CC0069771F791
:10190000C8010E949188A82E44E050E06BA97CA9F0
:10191000C8010E947288712C612CEA2DE450FF0BE3
:101920005F016A147B0424F6C8010E949188FFEFCE
:101930006F1A7F0AF6CF8A33910509F46FC074F5E8
:1019400085339105A1F1C69749F6C8010E94918897
:10195000B82EF701828D811109C0838D811106C0D7
:10196000848D811103C0858D8823A1F0EFA5F8A98E
:101970004080518062807380B401CE0183960E94C2
:101980004C828DA19EA1AFA1B8A584159505A60591
:10199000B705D9F544E050E0B40118C08B33910588
:1019A00009F452C08F3F910509F482CF97CFC80147
:1019B0000E949188C8010E949188D82E79CFC801D1
:1019C0000E94918844E050E069A97AA9C8010E9468
:1019D00072886ECFC8010E949188A82E44E050E022
:1019E000B101C8010E947288712C612C8A2D84502B
:1019F000990B5C016A147B040CF05ACFC8010E9459
:101A000091889FEF691A790AF5CFBA94FFEFBF1654
:101A100009F44ECFC8010E949188F7CFC8010E94F7
:101A2000918844E050E06BA57CA5C8010E947288B3
:101A3000F70166A177A180A591A50E941CCE66A39F
:101A400077A380A791A734CFC8010E94918844E072
:101A500050E06DA57EA5C8010E947288F70162A5BD
:101A600073A584A595A50E941CCE62A773A784A721
:101A700095A71ECFC8010E94918844E050E069A557
:101A80007AA5C8010E947288F70162A173A184A19E
:101A900095A10E941CCE62A373A384A395A366A7FD
:101AA00077A780AB91AB04CFDD24DA9488CE2F9258
:101AB0003F924F925F926F927F928F929F92AF92DE
:101AC000BF92CF92DF92EF92FF920F931F93CF932B
:101AD000DF9300D000D0CDB7DEB78C010E9482C565
:101AE0002FEC37E040E050E00E94ABCDDC01CB01B1
:101AF0000196A11DB11DF80184839583A683B78348
:101B000080839183A283B3835801F3E4AF0EB11CA9
:101B1000C5010E94EE1464E470E0C5010E94031543
:101B2000882309F445C10E94BEA22B013C01480153
:101B300082E4880E911C48EEC42E43E0D42EE12CA2
:101B4000F12C52E0252E1E821D82D4018C9183300F
:101B5000B1F1811166C0F80184819581A681B781B8
:101B60000196A11DB11D84839583A683B7830E942E
:101B7000BEA26419750986099709A70196010E94FA
:101B800089CDA90161E0C8010E94667C81E0D40191
:101B90008C938D819E810197C1F20E94BEA264192F
:101BA000750986099709D801D6962D913D914D91D9
:101BB0005C91D997261737074807590720F6C501C2
:101BC0000E94EE14F80184819581A681B781019667
:101BD000A11DB11D84839583A683B7830E94BEA2F5
:101BE000F801FE9660837183828393838D819E8149
:101BF00026960FB6F894DEBF0FBECDBFDF91CF9112
:101C00001F910F91FF90EF90DF90CF90BF90AF901A
